:020000040800F2
:1000000000040020E10100081D0F0008210F000876
:10001000750F0008210F0008490F0008E3010008D0
:10002000E3010008E3010008E301000809280008D3
:10003000E3010008E3010008E3010008E301000810
:10004000E3010008E3010008E3010008E301000800
:10005000E3010008E3010008713900089D39000838
:10006000C9390008F5390008213A0008E301000801
:10007000E3010008E3010008E3010008E3010008D0
:10008000E3010008E3010008E3010008E3010008C0
:10009000E3010008E3010008E30100084D3A00080D
:1000A000E3010008E3010008E3010008E3010008A0
:1000B000E3010008E3010008E3010008E301000890
:1000C000E3010008E3010008E3010008E301000880
:1000D000E3010008E30100082511000839110008B8
:1000E000B53A0008E3010008E3010008E301000855
:1000F000E3010008E3010008E3010008E301000850
:10010000E3010008E301000881370008E30100086B
:10011000E3010008E3010008E3010008E30100082F
:10012000E3010008E3010008E3010008E30100081F
:10013000E3010008E3010008E3010008E30100080F
:10014000E3010008E3010008E3010008F52E0008C0
:10015000E3010008E3010008E3010008E3010008EF
:10016000E3010008E3010008E3010008E3010008DF
:10017000E3010008E3010008E3010008E3010008CF
:10018000E3010008E30100084D110008E301000845
:10019000E3010008E3010008E3010008E3010008AF
:1001A000E3010008E3010008E3010008E30100089F
:1001B000E3010008E3010008E3010008E30100088F
:1001C000E3010008E3010008E3010008E30100087F
:1001D000E3010008E3010008E3010008E30100086F
:1001E00002E000F000F8FEE772B6394880F30888B4
:1001F000384880F3098838484EF60851CEF200019D
:10020000086040F20000CCF200004EF63471CEF2ED
:1002100000010860BFF34F8FBFF36F8F40F2000003
:10022000C0F2F0004EF68851CEF200010860BFF334
:100230004F8FBFF36F8F4FF00000E1EE100A4EF6C4
:100240003C71CEF200010860062080F31488BFF3F1
:100250006F8F02F017FB03F029FA4FF055301F495A
:100260001B4A91423CBF41F8040BFAE71C49194A6A
:1002700091423CBF41F8040BFAE71A491A4A1B4B5A
:100280009A423EBF51F8040B42F8040BF8E70020F5
:100290001749184A91423CBF41F8040BFAE702F0B3
:1002A000F5FA03F05FFA144C144DAC4203DA54F83B
:1002B000041B8847F9E700F03FF8114C114DAC42A0
:1002C00003DA54F8041B8847F9E702F0DDBA0000AE
:1002D000000400200024002000000008000000208E
:1002E00000040020583F000800240020282400209B
:1002F00028240020903D0020E0010008E0010008D3
:10030000E0010008E00100082DE9F04F2DED108A12
:10031000C1F80CD0C3689D46BDEC108ABDE8F08FD3
:10032000002383F311882846A047002001F0ECFE4B
:1003300001F09CFE00DFFEE770B5204C092300258C
:1003400023706FF03F061F236570A570E57025715F
:100350006571A571E57125726672A372E57200F090
:10036000FFFC20B10F2325726672A372E57202F0C2
:100370001DFA044602F042FA0546D8B9104B9C42D9
:100380001AD001339C4218BF054641F2883404BF9D
:1003900001250024002002F013FA0DB100F0B6F898
:1003A00000F062FD00F01AFC204600F00DF900F0AC
:1003B000ADF8F9E70024EDE70446EBE72824002038
:1003C000010007B008B500F087FBA0F120035842F8
:1003D000584108BD07B5054B02211B88ADF8043014
:1003E00001A800F0E5FB03B05DF804FB9C3B0008AE
:1003F000064991F8243033B100230822086A81F8B5
:10040000243000F00DBC0120704700BF48240020BC
:100410002DE9F84F234C94F82430054688461746BA
:100420008BBB2E46DFF87C90002F38D094F824A0A8
:10043000BAF1000F05D12022FF214846266200F0C4
:1004400001FDCAF10805BD4228BF3D465FFA85FBA4
:10045000AD0041462A4604EB8A0000F0C9FC94F83E
:100460002430A7EB0B079B445FFA8BFBBBF1080F13
:100470002E44A844FFB284F824B0D5D1FFF7B8FFCA
:100480000028D1D108E0266A06EB8306B042C9D025
:10049000FFF7AEFF0028C4D10020BDE8F88F01208F
:1004A000BDE8F88F4824002010B5202383F311887D
:1004B0001248C3680BB101F0ADFE0023104A0F488B
:1004C0004FF47A7101F06AFE002383F311880D4C1A
:1004D000236813B12368013B2360636813B1636829
:1004E000013B6360084B1B7833B9636823B9022072
:1004F00000F074FC3223636010BD00BF3424002080
:10050000A9040008782500207024002010B5254B90
:10051000254953F8042F013200D110BD8B42F8D188
:10052000224C234B22689A423AD9224B9B6803F112
:10053000006303F580439A4232D2002000F068FB4A
:100540001D4B0220187000F03FFC1C4B1A6C00225F
:100550001A64196E1A66196E596C5A64596E5A6685
:100560005A6E5A6942F080025A615A6922F080023A
:100570005A615A691A6942F000521A611A6922F0E6
:1005800000521A611B6972B60D4A0E4B13601B684C
:100590002268202181F311889D4683F30888104743
:1005A00010BD00BFFC3F00081C40000804400008CC
:1005B000FF3F00082824002070240020003802405B
:1005C00008ED00E0004000082DE9F04F99B0B34C71
:1005D00001902022FF2110A8A66800F033FCB04A49
:1005E0001378A346A3B9AF480121C360117020233B
:1005F00083F31188C3680BB101F00CFE0023AA4AF3
:10060000A8484FF47A7101F0C9FD002383F31188E3
:10061000019B13B1A54B019A1A60A54AA349019FFA
:100620000292002313704B6099461C461D46984663
:10063000012000F0C9FB002F00F012829B4B1B68C9
:10064000002B40F00D8219B0BDE8F08F0220FFF7BB
:10065000B9FE002840F0FB81019BB9F1000F08BFF3
:100660001F46944B1B88ADF82C3002210BA800F0DC
:100670009FFADDE74FF47A7000F02EFA031E039321
:10068000EADB0220FFF79EFE82460028E4D0039BAF
:10069000581E042800F2DD81DFE800F0030E11147B
:1006A000170018A8052340F8343D042100F080FA13
:1006B00054464FF0000856E004217848F6E704213C
:1006C0007D48F3E704217D48F0E71C24204600F034
:1006D000A1FA04340B9004210BA800F069FA2C2C29
:1006E000F4D1E5E7002DB7D0002CB5D00220FFF7FC
:1006F00069FE0546002800F0AF8101206C4C00F037
:1007000087FA0220207000F05FFB4FF000095FFACB
:1007100089FA504600F08CFA074658B1504600F06E
:1007200097FA09F101090028F1D12C46A9460027C2
:10073000634B97E701230220237000F03BFB3E460A
:10074000DBF808309E4206D2304600F063FA0130F2
:10075000EBD10436F4E7029B00261E70534BA946EA
:100760005E602C46374600F075FB15B1002C18BFB3
:100770000027FFF72FFE5BE7002D3FF46DAF002C45
:100780003FF46AAF029B0220187000F01DFB32207C
:1007900000F0A2F9B0F1000AC0F25E811AF0030580
:1007A00040F05A81DBF8082006EB0A03934200F27E
:1007B0005381BAF5807F00F24F8155450DDA4FF431
:1007C0007A7000F089F90490049B002BC0F24481F8
:1007D0003C4A049BAB540135EFE7C820FFF7F2FD1C
:1007E0000546002800F038811F2E11D8C6F12004DC
:1007F000544528BF544610AB26F003002246314929
:10080000184400F0F5FA2246FF212E4800F01AFBAA
:100810004FEAAA0A5FFA8AF22A493046FFF7F8FD42
:100820000446002800F01A8106EB8A0605469AE77E
:100830000220FFF7C7FD00283FF40EAFFFF7D8FDF9
:1008400000283FF409AF4FF0000A5346DBF80820B8
:1008500092451CD2BAF11F0F12D8109A01320FD054
:100860002AF0030218A90A4452F8202C0B921846C9
:1008700004220BA900F092FB0AF1040A0346E5E703
:100880005046039300F0C6F9039B0B90EFE718A8BE
:10089000042140F84C3D00F08BF964E72824002047
:1008A0007425002034240020A904000878250020A5
:1008B000702400209E3B00082C24002030240020BF
:1008C000A03B00087424002018A8002340F8343D01
:1008D000642100F039F900287FF4BEAE0220FFF752
:1008E00071FD00283FF4B8AE0B9800F0C3F918ABC7
:1008F00043F8480D04211846CDE718A8002340F816
:10090000343D642100F020F900287FF4A5AE0220D8
:10091000FFF758FD00283FF49FAE0B9800F0B8F9A0
:1009200018AB43F8440DE5E70220FFF74BFD002824
:100930003FF492AE00F0B2F918AB43F8400DD9E79E
:100940000220FFF73FFD00283FF486AE0BA91420DC
:1009500000F0AAF9824618A8042140F83CAD00F046
:1009600027F951460BA896E7322000F0B5F8B0F110
:10097000000AFFF671AE1AF0030F7FF46DAEDBF8DC
:1009800008200AEB080393423FF666AE0220FFF709
:1009900019FD00283FF460AE2AF0030AC244D04596
:1009A0003FF4E1AE404600F035F904210A900AA870
:1009B00000F0FEF808F10408F1E74FF47A70FFF751
:1009C00001FD00283FF448AEFFF712FD00283FF478
:1009D000AFAE109B01330CD0082210A90020FFF706
:1009E00017FD00283FF4A4AE2022FF2110A800F03C
:1009F00029FAFFF7EFFC374801F08CFB23E6002DC6
:100A00003FF42AAE002C3FF427AE18A8002340F88C
:100A1000343D642100F098F8824600287FF41CAE33
:100A20000220FFF7CFFC00283FF416AE0390FFF73B
:100A3000D1FC41F2883001F06DFB0B9800F04EFACA
:100A400000F008FA039B57461C461D46F0E5054694
:100A500089E64FF00008FFE52546FDE52C4667E6F0
:100A6000002000F039F80490049B002BFFF6E3AD62
:100A7000012000F09FF9049B213B122B3FF6D8ADDB
:100A800001A252F823F000BF4D06000875060008C9
:100A9000E5060008310600083106000831060008A6
:100AA000790700086909000831080008C90800082A
:100AB000FB08000829090008310600084109000860
:100AC00031060008BB090008670700083106000866
:100AD000FF090008A08601002DE9F34702AE0024BB
:100AE0004FF47A7506F8014D144FDFF858804543EE
:100AF00097F900305A1C5FFA84F901D0A34212D151
:100B000058F8240003680122D3F820A031462B4670
:100B1000D047012807D10A4B9DF8070083F80090C1
:100B200002B0BDE8F0870134042CE1D14FF4FA7033
:100B300001F0F0FA4FF0FF30F2E700BF0024002090
:100B400098250020F43B00082DE9F0474FF47A7512
:100B5000144FDFF8588006464D43002497F90030C3
:100B60005A1C5FFA84F901D0A34210D158F824002E
:100B700003680422D3F820A031462B46D04704282E
:100B800005D1094B83F800900020BDE8F0870134BF
:100B9000042CE3D14FF4FA7001F0BCFA4FF0FF30AF
:100BA000BDE8F0870024002098250020F43B0008D1
:100BB00030B4074B1A78074B53F822402368DD699D
:100BC000054B0A46AC460146204630BC604700BF94
:100BD00098250020F43B0008A086010070B501F0C4
:100BE000E1FC094C094E20700025306823788342CF
:100BF00008D901F0D1FC336805440133B5F5804FC5
:100C00003360F2D370BD00BF9925002080250020FD
:100C100001F07EBD00F1006000F580400068704783
:100C200000F10060920000F5804001F009BD000075
:100C3000054B1A68054B1B789B1A834202D9104456
:100C400001F0AABC002070478025002099250020D3
:100C500038B5074D04462868204401F0A5FC28B9A2
:100C600028682044BDE8384001F0B6BC38BD00BF5C
:100C70008025002010F0030308D1B0F5007F05D8CF
:100C800000F10050A0F50840006870470020704750
:100C9000014BC058704700BF107AFF1F014B186806
:100CA000704700BF002004E070B52A4B1C68C4F3F5
:100CB0000B03240C63B140F21342934231D040F253
:100CC000194293422FD040F2214293422DD1032367
:100CD000214A0C2505FB03235D6893F9082042F2A5
:100CE00001039C4224D0B4F5805F23D041F201037C
:100CF0009C4221D041F203039C421FD041F20703E2
:100D00009C4208BF3122441E0C44013D0B46A342C5
:100D10001ED215F9016F581C96B1034600F8016CFC
:100D2000F5E70123D4E70223D2E73F220B4DD6E7B4
:100D30003322E3E74122E1E75A22E4E75922E2E7DE
:100D40002C2584421D7001D9981C5A70401A70BD20
:100D50001846FBE7002004E0C43B0008A43B000861
:100D6000124B5A8842F201018A4293B214D0B3F571
:100D7000805F13D041F20102934211D041F203028D
:100D800093420FD041F2070293420DD10423084A47
:100D900002EB8303D87870470023F8E70123F6E7D6
:100DA0000223F4E70323F2E700207047002004E069
:100DB000B03B0008022802BF024B4FF480529A61F8
:100DC000704700BF00100240022802BF024B4FF0E4
:100DD00080529A61704700BF00100240022801BF94
:100DE000024A536983F480535361704700100240F4
:100DF00010B50023934203D0CC5CC4540133F9E70F
:100E000010BD000030B5441E14F9010F0B4660B14F
:100E100093F90050854201F1010106D11AB993F905
:100E20000020801A30BD013AEEE7002AF7D11046C3
:100E300030BD000002460346981A13F9011B002931
:100E4000FAD1704702440346934202D003F8011BD3
:100E5000FAE77047024B1A78024B1A70704700BFCE
:100E60009825002000240020F8B5164C1648174D90
:100E7000174E154F00F096FC2146134800F0BEFCBB
:100E800024681448626D936B23F40023936301F08C
:100E900041F92046104900F0BDFD626D936B43F4AB
:100EA000002393634FF4E1332B60002456F82400B1
:100EB000B84202D0294600F0D3FB0134042CF5D10E
:100EC000F8BD00BFDC3C00089433002084250020DE
:100ED000F43B000840420F00043D000838B50B4BBE
:100EE0001A780B4B53F822400A4B9C4205460CD013
:100EF000094B002118461422FFF7A4FF05600146A4
:100F00002046BDE8384000F0ABBB38BD9825002036
:100F1000F43B00089433002084250020FEE7000005
:100F200000B59BB0EFF3098168226846FFF760FFC8
:100F3000EFF30583034B9A6B9A6A9A6A9A6A9A6AE4
:100F40009B6AFEE700ED00E000B59BB0EFF309817E
:100F500068226846FFF74CFFEFF30583044B9A6B5A
:100F60009A6A9A6A9A6A9A6A9A6A9B6AFEE700BFC4
:100F700000ED00E000B59BB0EFF309816822684600
:100F8000FFF736FFEFF30583034B5A6B9A6A9A6AB1
:100F90009A6A9A6A9B6AFEE700ED00E030B5084D58
:100FA0000A4491420BD011F8013B09245840013CFE
:100FB000F7D040F300032B4083EA5000F7E730BD41
:100FC0002083B8ED002304491A465A50C818083344
:100FD000802B4260F9D170479C250020026843684D
:100FE0001143016003B1184770470000024AD368FB
:100FF00043F0C003D360704700440040024AD36806
:1010000043F0C003D360704700480040024AD368F1
:1010100043F0C003D3607047007800402DE9F041F1
:10102000D0F85C64F7683368DA0505469CB20DD5E4
:10103000202383F311884FF400710430FFF7CEFFB3
:101040006FF480733360002383F31188202383F3CC
:10105000118805F1040814F02F0333D183F31188AC
:10106000380615D5210613D5202383F3118805F101
:10107000380000F053FA002846DA0821281DFFF74F
:10108000ADFF4FF67F733B40F360002383F311887D
:101090007A060ED563060CD5202383F31188EA6CFB
:1010A0002B6D9A4202D12B6C002B2FD1002383F39E
:1010B0001188D5F86424D368002B31D01069BDE8BD
:1010C000F0411847230713D014F0080F0CBF00217C
:1010D0008021E00748BF41F02001A20748BF41F04E
:1010E0004001630748BF41F480714046FFF776FF37
:1010F000A406736805D595F860142846194000F0D9
:10110000BDFA3468A4B2A6E77060BEE727F04007D6
:101110003F041021281D3F0CFFF760FFF760C5E773
:10112000BDE8F08108B50348FFF778FFBDE8084047
:1011300001F07ABB1C26002008B50348FFF76EFFBC
:10114000BDE8084001F070BB842A002008B50348C0
:10115000FFF764FFBDE8084001F066BBEC2E0020FD
:1011600010B50E4C0E4A2046002100F057FA0D4BE8
:10117000C4F85C340C4C0D4A2046002100F04EFAB5
:101180000B4BC4F85C340B4C0B4A0021204600F09A
:1011900045FA0A4BC4F85C3410BD00BF1C26002081
:1011A000ED0F000800440040842A0020FD0F0008D5
:1011B00000480040EC2E00200D1000080078004090
:1011C00038B5394D037C002918BF0D46012B044664
:1011D000C0F8645410D1354B984242D1344B1A6C4C
:1011E00042F400321A641A6E42F400321A661B6E20
:1011F0000B21262000F06AF82E4BD4F85C249A428A
:101200002B6802D02C498A424BD12C4901EB530167
:10121000B1FBF3F3A988080442BF23F0070003F0F1
:10122000070343EA40039360EB8843F040039BB21B
:1012300013612B8943F001039BB2536141F40453C2
:1012400043F02C03D36001F4A05100231360B1F5E7
:10125000806F136853680CBF7F23FF2384F86034CA
:1012600038BD174B98420CD1114B1A6C42F48022B6
:101270001A641A6E42F480221A661B6E0B21272014
:10128000B8E7104B9842B7D1094B1A6C42F0804234
:101290001A641A6E42F080421A661B6E0B215220AD
:1012A000A8E70949B2E700BF243C00081C2600203B
:1012B00000380240001001400014014000BD01054B
:1012C000842A0020EC2E002080DE800200F16043A2
:1012D00000F01F02400903F5614309018000C9B213
:1012E00000F1604083F8001300F561400123934052
:1012F000C0F8803103607047F8B51546826806690A
:10130000AA420B46816938BF8568761AB542044601
:1013100007D218462A46FFF76BFDA3692B44A36149
:101320000DE011D932461846FFF762FDAF1B3A4671
:10133000E1683044FFF75CFDE2683A44A261A368CB
:101340005B1BA3602846F8BD18462A46FFF750FDF0
:10135000E368E4E783682DE9F041044693421546CB
:10136000266938BF85684069361AB5420F4606D2ED
:101370002A46FFF73DFD63692B4463610DE012D9F6
:101380003246A5EB0608FFF733FD4246B919E0687F
:10139000FFF72EFDE26842446261A3685B1BA36015
:1013A0002846BDE8F0812A46FFF722FDE368E4E71E
:1013B00010B50A440024C361029B00604060846051
:1013C000C160816141610261036210BD08B582693B
:1013D0004369934201D1826882B982680132826096
:1013E0005A1C42611970426903699A4201D3C36869
:1013F0004361002100F0AAFE002008BD4FF0FF303D
:1014000008BD000070B5202304460E4683F3118802
:10141000A568A5B1A368A269013BA360531CA361A1
:1014200015782269934224BFE368A361E3690BB195
:1014300020469847002383F31188284670BD314623
:10144000204600F073FE0028E2DA85F3118870BDB3
:101450002DE9F74F05460F4690469A46D0F81C9066
:10146000202686F311884FF0000B144664B1224603
:1014700039462846FFF740FF034668B951462846DB
:1014800000F054FE0028F1D0002383F31188A8EB6C
:10149000040003B0BDE8F08FB9F1000F03D0019054
:1014A0002846C847019B8BF31188E41A1F4486F332
:1014B0001188DBE7C16081614161C3611144009B18
:1014C000006040608260016103627047F8B50446C5
:1014D0000E461746202383F31188A568A5B1A3689B
:1014E000013BA36063695A1C62611E7023696269D3
:1014F0009A4224BFE3686361E3690BB120469847D1
:10150000002080F31188F8BD3946204600F00EFE19
:101510000028E2DA85F31188F8BD0000836942698A
:101520009A4210B501D182687AB98268013282602C
:101530005A1C82611C7803699A4201D3C368836193
:10154000002100F003FE204610BD4FF0FF3010BD1B
:101550002DE9F74F05460F4690469A46D0F81C9065
:10156000202686F311884FF0000B144664B1224602
:1015700039462846FFF7EEFE034668B9514628462D
:1015800000F0D4FD0028F1D0002383F31188A8EBEC
:10159000040003B0BDE8F08FB9F1000F03D0019053
:1015A0002846C847019B8BF31188E41A1F4486F331
:1015B0001188DBE7026843681143016003B11847F3
:1015C000704700001430FFF743BF00004FF0FF33B7
:1015D0001430FFF73DBF00003830FFF7B9BF0000FF
:1015E0004FF0FF333830FFF7B3BF00001430FFF780
:1015F00009BF00004FF0FF311430FFF703BF0000B8
:101600003830FFF763BF00004FF0FF323830FFF78C
:101610005DBF000000207047FFF7A2BD37B50F4B3C
:101620000360002343608360C360012304460374A6
:10163000154600900B464FF4007200F15C01143027
:10164000FFF7B6FE00942B464FF4007204F51771B5
:1016500004F13800FFF72EFF03B030BD383C00081E
:1016600010B52023044683F31188FFF7A9FD022358
:101670002374002383F3118810BD000038B5C369BB
:1016800004460D461BB904210844FFF793FF294681
:1016900004F11400FFF79AFE002806DA201D4FF42B
:1016A0008061BDE83840FFF785BF38BD02684368F8
:1016B0001143016003B118477047000013B5446B34
:1016C000D4F894341A681178042915D1217C0229A0
:1016D00012D11979128901238B4013420CD101A92F
:1016E00004F14C0001F056FED4F89444019B21799A
:1016F0000246206800F0DAF902B010BD143001F0A3
:10170000D9BD00004FF0FF33143001F0D3BD00000D
:101710004C3001F0ABBE00004FF0FF334C3001F015
:10172000A5BE0000143001F0A7BD00004FF0FF314E
:10173000143001F0A1BD00004C3001F077BE000074
:101740004FF0FF324C3001F071BE0000D0F894240D
:1017500038B5136819780429054601D0012038BD31
:10176000017C0229FAD112795C8901209040044061
:10177000F4D105F1140001F039FD02460028EDD046
:10178000D5F894544FF480732868697900F07CF997
:10179000204638BD406BFFF7D9BF000000207047DE
:1017A000704700007FB5124B0360002343608360E5
:1017B000C360012502260F4B057404460290019375
:1017C00000F18402294600964FF48073143001F032
:1017D000E9FC094B0193029400964FF4807304F5E1
:1017E0002372294604F14C0001F0B0FD04B070BD35
:1017F000603C000895170008BD1600080B68202201
:1018000082F311880A7903EB820290614A790932E6
:1018100043F822008A7912B103EB82039861022314
:101820000374C0F89414002383F3118870470000F8
:1018300038B5037F044613B190F85430ABB9201D7E
:1018400001250221FFF732FF04F1140025776FF024
:10185000010100F087FC84F8545004F14C006FF053
:101860000101BDE8384000F07DBC38BD10B5012154
:1018700004460430FFF71AFF0023237784F854301E
:1018800010BD000038B504460025143001F0A2FC5C
:1018900004F14C00257701F071FD201D84F85450AF
:1018A0000121FFF703FF2046BDE83840FFF74EBF98
:1018B00090F8443003F06003202B19D190F84520B4
:1018C000212A0AD0222A4FF000030ED0202A0FD15D
:1018D000084A82630722C26304E0064B836307233E
:1018E000C36300230364012070478363C363F9E784
:1018F0000020704701240020D0F8943437B51A68CE
:101900001178042904461AD1017C022917D11979CA
:10191000128901238B40134211D100F14C05284656
:1019200001F0ECFD58B101A9284601F033FDD4F8CF
:101930009444019B21790246206800F0B7F803B077
:1019400030BD000000EB8103F7B59C6905460E46EB
:10195000F4B1202383F3118805EB8607201D0821AD
:10196000FFF7A4FEFB685B691B684C3413B120468B
:1019700001F01EFD01A9204601F00CFD024648B110
:10198000019B3146284600F091F8002383F311882B
:1019900003B0F0BDFB685A691268002AF5D01B8AB3
:1019A000013B1340F1D105F14402EAE7093138B5B2
:1019B00050F82140DCB1202383F31188D4F894241B
:1019C0001368527903EB8203DB689B695D6845B15C
:1019D00004216018FFF76AFE294604F1140001F0A3
:1019E0000FFC2046FFF7B2FE002383F3118838BDB9
:1019F0007047000000F0D0BF012303700023436054
:101A0000C36183620362C3624362036303814381F0
:101A10007047000038B50446202383F31188002561
:101A20004160C56005614561856100F0C5FF022325
:101A3000237085F3118838BD70B500EB810305462E
:101A40005069DA600E46144618B110220021FFF7E3
:101A5000F9F9A06918B110220021FFF7F3F9314616
:101A60002846BDE8704001F071B80000028902F01C
:101A700001020281428902F00102428100220261D8
:101A80004261826101F0F6B8F0B400EB810447894D
:101A9000E4680125A4698D403D434581236000230E
:101AA000A2606360F0BC01F011B90000F0B400EB7B
:101AB00081040789E468012564698D403D430581FF
:101AC00023600023A2606360F0BC01F08BB90000CA
:101AD00070B50223002504460370A0F84C5080F82E
:101AE0004E5080F84F5005814581C56005614561C4
:101AF000856180F8345000F0C5FF63681B6823B12E
:101B000029462046BDE87040184770BD43680278FA
:101B10001B6880F85020052202700BB10421184781
:101B200070470000436890F850201B6802700BB1AA
:101B3000052118477047000090F8343070B504460E
:101B400013B1002380F8343004F14402204601F040
:101B5000B3F863689B6863BB94F8445015F0600663
:101B600015D194F8453005F07F0545EA032540F28C
:101B700002339D4200F00E815BD8022D00F0DC8024
:101B80003FD8002D00F08780012D00F0CF8000218C
:101B9000204601F0E9FA0021204601F0DBFA6368F3
:101BA0001B6813B1062120469847062384F8343079
:101BB00070BD204698470028CED094F84B2094F86A
:101BC0004A3043EA0223E26B934238BFE36394F95D
:101BD0004430E56B002B4FF0200380F2FD80002D98
:101BE00000F0EC80092284F8342083F3118800216E
:101BF000E36BA26B2046FFF759FF002383F31188A4
:101C000070BDB5F5817F00F0B180B5F5407F49D05A
:101C1000B5F5807FBBD194F84630012BB7D1B4F82D
:101C20004C3023F00203A4F84C30A663E66326642C
:101C3000C3E740F201639D421ED8B5F5C06F3BD2A9
:101C4000B5F5A06FA3D1B4F84430B3F5A06F0ED1B1
:101C500094F8463084F84E30204600F06BFF6368FD
:101C60001B6813B1012120469847032323700023EA
:101C7000A363E3632364A0E7B5F5106F32D040F6A9
:101C800002439D4252D0B5F5006F80D104F14F035D
:101C9000A363012324E004F14C03A3630223E36361
:101CA00025648AE794F84630012B7FF470AFB4F8CE
:101CB0004C3043F00203B6E794F84920616894F889
:101CC00048304D6894F8471043EA0223204694F8C0
:101CD0004620A84700283FF45AAF4368A36303682F
:101CE000E363A4E72378042B10D1202383F3118826
:101CF0002046FFF7BBFE86F31188636884F84F60C7
:101D00001B68032121700BB12046984794F8463098
:101D1000002BACD084F84F300423237063681B6819
:101D2000002BA4D0022120469847A0E7374BA3639D
:101D30000223E36300239DE794F8481011F0800F1D
:101D4000204601F00F010ED000F0A8FF012806D0B8
:101D500002287FF41CAF2E4BA363E06367E72D4B93
:101D6000A363E56363E700F08BFFEFE794F8463089
:101D7000002B7FF40CAF94F8483013F00F013FF4C0
:101D800076AF1A06204602D501F002FA6FE701F09D
:101D9000F5F96CE794F84630002B7FF4F8AE94F830
:101DA000483013F00F013FF462AF1B06204602D506
:101DB00001F0DAF95BE701F0CDF958E7142284F875
:101DC000342083F311882B462A4629462046FFF704
:101DD0005BFE85F3118870BD5DB1152284F8342057
:101DE00083F311880021E36BA26B2046FFF74CFEC2
:101DF00003E70B2284F8342083F311882B462A460C
:101E000029462046FFF752FEE3E700BF903C00085A
:101E1000883C00088C3C000838B590F83430044603
:101E2000152B29D8DFE803F03E28282828283E284B
:101E3000280B293928282828282828283E3E90F8C9
:101E40004B1090F84A20C36B42EA01229A4214D9FF
:101E5000C268128AB3FBF2F502FB15356DB9202377
:101E600083F311882B462A462946FFF71FFE85F388
:101E700011880A2384F8343038BD142384F83430B0
:101E8000202383F3118800231A4619462046FFF7C2
:101E9000FBFD002383F3118838BD036C03B1984721
:101EA0000023E7E7002101F05FF90021204601F05F
:101EB00051F963681B6813B1062120469847062331
:101EC000D8E7000090F83420152A38B5044622D807
:101ED0000123934040F6416213421DD113F4801553
:101EE0000FD19B0217D50B2380F83430202383F3C6
:101EF00011882B462A462946FFF7D8FD85F311881D
:101F000038BDC3689B695B682BB9036C03B1984704
:101F1000002384F8343038BD002101F025F9002178
:101F2000204601F017F963681B6813B106212046AB
:101F300098470623EDE70000024B00221B605B6020
:101F40009A60704754330020002303748268054B65
:101F50001B6899689142FBD25A6803604260106026
:101F6000586070475433002008B5202383F311884C
:101F7000037C032B05D0042B0DD02BB983F31188E0
:101F800008BD436900221A604FF0FF334361FFF739
:101F9000DBFF0023F2E790E80C001A600268536050
:101FA000F2E70000002303748268054B1B68996800
:101FB0009142FBD85A6803604260106058607047D5
:101FC00054330020054B19690874186802681A60B8
:101FD0005360186101230374FEF796B9543300204F
:101FE00030B54B1C87B005460A4C10D023690A4A0D
:101FF00001A800F0D3F82846FFF7E4FF049B13B1D3
:1020000001A800F007F92369586907B030BDFFF750
:10201000D9FFF8E754330020691F000838B50C4D8C
:1020200041612B6981689A689142044603D8BDE8F2
:102030003840FFF789BF1846FFF786FF01232C6160
:10204000014623742046BDE83840FEF75DB900BF65
:1020500054330020044B1A681B6990689B689842AF
:1020600094BF0020012070475433002010B5084C65
:10207000236820691A6822605460012223611A745F
:10208000FFF790FF01462069BDE81040FEF73CB91C
:10209000543300208260022202740022427470478E
:1020A0008368A3F17C0243F80C2C026943F83C2CB2
:1020B000426943F8382C074A43F81C2CC26843F89D
:1020C000102C022203F8082C002203F8072CA3F19D
:1020D000180070472103000810B5202383F31188EE
:1020E000FFF7DEFF00210446FFF798FF002383F38C
:1020F0001188204610BD0000024B1B6958610F205B
:10210000FFF760BF54330020202383F31188FFF7CB
:10211000F3BF000008B50146202383F3118808208F
:10212000FFF75EFF002383F3118808BD49B1064B1A
:1021300042681B6918605A60136043600420FFF70F
:102140004FBF4FF0FF307047543300200368984270
:1021500006D01A680260506059611846FFF7F4BE55
:102160007047000038B504460D462068844200D10F
:1021700038BD036823605C604561FFF7E5FEF4E766
:10218000054B03F114025A619A614FF0FF32DA6194
:1021900000221A62704700BF54330020F8B5036173
:1021A0001A4BC2605C6A1A4B1A46022952F8145F35
:1021B00038BF0221954206461F460AD158619861F0
:1021C0001C620560456081600819BDE8F84001F0B7
:1021D000B7B9186AAB68241A0C1902D3E41A2D682F
:1021E00004E09C4202D2204401F0BAF9AB689C4260
:1021F000F4D86B68736035601E606E60B460A96867
:102200004FF0FF33091BA960FB61F8BD000C0040D3
:102210005433002010B41A4C234653F8141F814243
:1022200010D0416802680A60026851609A424FF01B
:102230000001C16003D0936881680B4493605DF82E
:10224000044B70470A68626100209A425360C8607C
:1022500003D15DF8044B01F07DB9936888680344AD
:102260009360084A206A526A121A9342E7D9991A6F
:10227000012998BF931C18445DF8044B01F070B914
:1022800054330020000C004000207047FEE700009F
:10229000704700004FF0FF3070470000022906D061
:1022A000032906D00129064818BF002070470548B9
:1022B0007047032A9ABF044800EBC2000020704711
:1022C000603D0008143D00080824002070B59AB055
:1022D00001AD064608462946144600F095F8284602
:1022E000FEF7A8FDC0B2431C5B0086E8180023700F
:1022F00003236370002302341946DAB2904204F1DA
:10230000020401D81AB070BDEA5C04F8022C04F88B
:10231000011C0133F1E7000008B5202383F3118885
:102320000348FFF7E9FA002383F3118808BD00BFD3
:102330009433002010B50446052916D8DFE801F0D3
:1023400016150316161D202383F311880E4A01214A
:10235000FFF772FB20460D4A0221FFF76DFB0C4888
:10236000FFF790FA002383F3118810BD202383F335
:1023700011880748FFF75CFAF4E7202383F31188FC
:102380000348FFF773FAEDE7943C0008B83C0008F7
:102390009433002038B50C4D0C4C0D492A4604F1FD
:1023A0000800FFF793FF05F1CA0204F11000094984
:1023B000FFF78CFF05F5CA7204F118000649BDE865
:1023C0003840FFF783BF00BF5C380020082400209E
:1023D000E43C0008EE3C0008F93C000870B50446F7
:1023E00008460D46FEF726FDC6B2204601340378A6
:1023F0000BB9184670BD32462946FEF703FD00288A
:10240000F3D1012070BD00002DE9F84F05460C46C0
:10241000FEF710FD2A49C6B22846FFF7DFFF08B1D4
:10242000023EF6B227492846FFF7D8FF08B110361A
:10243000F6B2632E0DD8DFF88890DFF888A0224F1F
:10244000DFF88CB0DFF88C802E7846B92670BDE8B6
:10245000F88F29462046BDE8F84F01F097BB252E9E
:1024600029D1072249462846FEF7CCFC40B9D8F8C6
:102470000030236098F80430237107350534E3E712
:10248000082251462846FEF7BDFCA0B90F4BA21CFE
:1024900013F8011F09095B45C95D02F8021C197890
:1024A00001F00F0102F10202C95D02F8031CEFD135
:1024B00018340835C8E7267001350134C4E700BF79
:1024C000803D0008F93C00088E3D00080F7AFF1F90
:1024D0001B7AFF1F883D0008BFF34F8F024AD36865
:1024E000DB03FCD4704700BF003C024008B5094B39
:1024F0001B7873B9FFF7F0FF074B1A69002ABFBFBB
:10250000064A5A6002F188325A601A6822F48062E0
:102510001A6008BDBA3A0020003C0240230167451A
:1025200008B50B4B1B7893B9FFF7D6FF094B1A6917
:1025300042F000421A611A6842F480521A601A6826
:1025400022F480521A601A6842F480621A6008BD50
:10255000BA3A0020003C0240172870B513D80B4A45
:102560000B4C137863B90B4E4FF0006144F8231005
:1025700056F823500133182B2944F7D10123137047
:1025800054F8200070BD002070BD00BF1C3B00202F
:10259000BC3A0020A03D0008014B53F820007047D2
:1025A000A03D000818207047172810B5044601D92F
:1025B000002010BDFFF7D0FF064B53F8243018441D
:1025C000C21A0BB9012010BD12680132F0D1043BD0
:1025D000F6E700BFA03D0008172810B5044629D82B
:1025E000FFF77AFFFFF782FF1349F323CB600C2339
:1025F000B0FBF3F203FB1200D30143EAC003DBB2EA
:1026000043F4007343F002030B610B6943F480331E
:102610000B61FFF761FF2046FFF79EFF074B53F862
:10262000241000F0DDF8FFF77BFF2046BDE81040E6
:10263000FFF7BABF002010BD003C0240A03D0008DB
:102640002DE9F84312F00103154640D18218B2F18A
:10265000026F3CD22C4B1B6813F0010337D02B4C7C
:10266000FFF744FFF323E360FFF736FF40F2012753
:10267000032D01D9830713D0244C0F46401A40F292
:102680000118EB1B0B44012B00EB0706236924D830
:1026900023F001032361FFF743FF0120BDE8F88326
:1026A000236923F44073236123693B43236151F879
:1026B000046B0660BFF34F8FFFF70EFF03689E4267
:1026C00008D0236923F001032361FFF729FF0020CD
:1026D000BDE8F883043D0430CAE723F44073236166
:1026E000236943EA08032361B94637F8023B338084
:1026F000BFF34F8FFFF7F0FE3688B9F80030B6B25F
:10270000B342BED0DDE700BF00380240003C0240CB
:10271000084908B50B7828B153B9FFF7E7FE012344
:102720000B7008BD23B1BDE808400870FFF7F8BE84
:1027300008BD00BFBA3A002010B50244064B043968
:10274000D2B2904200D110BD441C00B253F8200018
:1027500041F8040FE0B2F4E750280040104B30B5C8
:102760001C6F240407D41C6F44F400741C671C6F96
:1027700044F400441C670B4C236843F480732360CB
:102780000244094B0439D2B2904200D130BD441CFE
:1027900000B251F8045F43F82050E0B2F4E700BF04
:1027A00000380240007000405028004007B5012268
:1027B00001A90020FFF7C0FF019803B05DF804FBFA
:1027C00013B50446FFF7F2FFA04206D002A901228A
:1027D00041F8044D0020FFF7C1FF02B010BD00001A
:1027E00070470000034B1B689B0042BF024B012255
:1027F0001A707047743802401D3B0020014B187856
:10280000704700BF1D3B0020064A536823F00103B8
:102810005360EFF30983683383F30988002383F35C
:102820001188704730EF00E010B5202383F3118842
:10283000104B5B6813F4006318D0F1EE103AEFF31D
:1028400009844FF0807344F84C3C0B4BDB6844F830
:10285000083CA4F1680383F30988FFF7FBFB18B178
:10286000064B44F8503C10BD054BFAE783F3118842
:1028700010BD00BF00ED00E030EF00E031030008C4
:102880003403000870470000FEE70000084A094BC7
:1028900009498B4204D3094A0021934205D370476A
:1028A00052F8040F43F8040BF3E743F8041BF4E772
:1028B0007C3F0008903D0020903D0020903D00208E
:1028C000836D30B500229D68446D11464FF0FF3096
:1028D00004EB421301329542C3F80019C3F81019F2
:1028E000C3F80809C3F8001BC3F8101BC3F8080B92
:1028F000EED24FF00113C4F81C3830BD890141F00D
:102900002001016103699B06FCD4122000F0B4BED3
:10291000204B03EB80022DE9F047D2F80CE05D6D0F
:10292000DEF81420461CD2F800C005EB063605EB95
:102930004018516861450BD3D5F83428012303FAB8
:1029400000F022EA0000C5F834081846BDE8F08718
:10295000BEF81040ACEB0103A34228BF2346D8F8D1
:102960001849A4B2B3EB840F10D894681F46A4F1A1
:10297000040959F804AFC6F800A0042F01D9043F98
:10298000F7E71C440B4494605360D2E70020BDE895
:10299000F08700BF203B002010B5054C2046FFF714
:1029A0002BF84FF0A0436365024BA36510BD00BF39
:1029B000203B0020243E00080378012B70B505461B
:1029C00050D12A4B446D98421BD1294B5A6B42F08F
:1029D00080025A635A6D42F080025A655A6D5A69F4
:1029E00042F080025A615A6922F080025A610E2137
:1029F00043205B69FEF76AFC1E4BE3601E4BC4F884
:102A000000380023C4F8003EC02323606E6D4FF4ED
:102A10005023A3633369002BFCDA012333610C20BC
:102A200000F02AFE3369DB07FCD4122000F024FEFC
:102A30003369002BFCDA0026A6602846FFF740FF2A
:102A40006B68C4F81068DB68C4F81468C4F81C68C4
:102A50004BB90A4BA3614FF0FF336361A36843F0A6
:102A60000103A36070BD064BF4E700BF203B0020CC
:102A7000003802404014004003002002003C30C0F7
:102A8000083C30C0F8B5446D054600212046FFF7EC
:102A900035FFA96D00234FF001128F68C4F8343858
:102AA0004FF00066C4F81C284FF0FF3004EB4312CF
:102AB00001339F42C2F80069C2F8006BC2F80809EE
:102AC000C2F8080BF2D20B686A6DEB6563621023E3
:102AD0001361166916F01006FBD1122000F0CCFD30
:102AE000D4F8003823F4FE63C4F80038A36943F433
:102AF000402343F01003A3610923C4F81038C4F83D
:102B000014380A4BEB604FF0C043C4F8103B084B3D
:102B1000C4F8003BC4F81069C4F80039EB6D03F148
:102B2000100243F48013EA65A362F8BD003E00087A
:102B300040800010426D90F84E10D2F8003823F417
:102B4000FE6343EA0113C2F8003870472DE9F041F3
:102B50000EB200EB86080D46D8F80C100F6807F08F
:102B60000303022B50D0032B50D03D4A3D4F012B85
:102B700018BF1746446D4FEA451E04EB0E030022B2
:102B8000C3F8102B8A6905F1100C002A40D04A8A3C
:102B900005F158035B013A43E2500123D4F81C28A5
:102BA00003FA0CF31343A6444A69C4F81C38002303
:102BB000CEF8103905F13F03002A39D00A8A898BF3
:102BC0009208012988BF4A43C16D04EB830356185C
:102BD00041EA0242C66529465A602046FFF78EFE4A
:102BE000D8F80C301B8A43EA85531F4305F148038C
:102BF0005B01E7500123D4F81C2803FA05F51543BF
:102C0000C4F81C58BDE8F081174FB3E7174FB1E780
:102C100004EB4613D3F8002B22F40042C3F8002B38
:102C2000D4F81C28012303FA0CF322EA0303BAE7C1
:102C300004EB83030E4A5A6004EB461629462046ED
:102C4000FFF75CFED6F8003923F40043C6F80039DC
:102C5000D4F81C38012202FA05F523EA0505CFE76E
:102C600000800010008004100080081000800C100C
:102C700000040002826D1268C265FFF721BE0000E9
:102C80005831436D49015B5813F4004004D013F4EC
:102C9000001F14BF01200220704700004831436D1F
:102CA00049015B5813F4004004D013F4001F14BF13
:102CB000012002207047000000EB8101CB68196AF7
:102CC0000B6813604B6853607047000000EB810392
:102CD00030B5DD68AA691368D36019B9402B84BF89
:102CE000402313606B8A1468426D1C44013CB4FBA2
:102CF000F3F46343033323F0030302EB411043EA8D
:102D0000C44343F0C043C0F8103B2B6803F00303F7
:102D1000012B09B20ED1D2F8083802EB411013F49E
:102D2000807FD0F8003B14BF43F0805343F0005342
:102D3000C0F8003B02EB4112D2F8003B43F00443E1
:102D4000C2F8003B30BD00002DE9F041244D6E6D0E
:102D500006EB40130446D3F8087BC3F8087B38071A
:102D60000AD5D6F81438190706D505EB8403214691
:102D7000DB6828465B689847FA072FD5D6F81438E1
:102D8000DB072BD505EB8403D968CCB98B69488A5E
:102D90005E68B6FBF0F200FB12628AB91868DA6866
:102DA00090420DD2121A83E81400202383F3118875
:102DB0000B482146FFF78AFF84F31188BDE8F081B4
:102DC000012303FA04F26B8923EA02036B81CB68C7
:102DD00023B121460248BDE8F0411847BDE8F08123
:102DE000203B002000EB810370B5DD68436D6C690A
:102DF0002668E6604A0156BB1A444FF40020C2F828
:102E000010092A6802F00302012A0AB20ED1D3F88F
:102E1000080803EB421410F4807FD4F8000914BFB3
:102E200040F0805040F00050C4F8000903EB42121B
:102E3000D2F8000940F00440C2F80009D3F8340881
:102E4000012202FA01F10143C3F8341870BD19B927
:102E5000402E84BF4020206020682E8A841940F0D4
:102E60000050013C1A44B4FBF6F440EAC440C6E703
:102E7000F8B504461E48456D05EB4413D3F80869C0
:102E8000C3F80869F10717D5D5F81038DA0713D554
:102E900000EB8403D9684B691F68DA68974218D23F
:102EA000D21B00271A605F60202383F3118821461C
:102EB000FFF798FF87F31188330617D5D5F8342824
:102EC0000123A340134211D02046BDE8F840FFF78C
:102ED0001FBD012303FA04F2038923EA02030381DD
:102EE0008B68002BE8D021469847E5E7F8BD00BF86
:102EF000203B002096482DE9F84F456D6E69AB697F
:102F00001E4016F4805F6E61044605D0FEF7E0FDBA
:102F1000BDE8F84FFFF788BC002E12DAD5F8003E66
:102F20008B489B071EBFD5F8003E23F00303C5F86E
:102F3000003ED5F8043823F00103C5F80438FEF745
:102F4000F1FD370502D58248FEF7E0FDB0040CD54F
:102F5000D5F8083813F0060FEB6823F470530CBF54
:102F600043F4105343F4A053EB60310704D5636876
:102F7000DB680BB176489847F2025AD4B3020CD5FD
:102F8000D4F85480DFF8C8A100274FF00109A36DE1
:102F90009B68F9B28B4280F08780F70619D5616D86
:102FA0000A6AC2F30A1702F00F0302F4F012B2F534
:102FB000802F00F0A180B2F5402F0AD104EB8303EB
:102FC00001F58051DB68186A00231A469F4240F0E1
:102FD00087803003D5F8184813D5E10302D50020C7
:102FE000FFF7B2FEA20302D50120FFF7ADFE630397
:102FF00002D50220FFF7A8FE270302D50320FFF722
:10300000A3FE750384D5E00702D50020FFF730FF4B
:10301000A10702D50120FFF72BFF620702D502208E
:10302000FFF726FF23077FF573AF0320FFF720FF8D
:103030006EE7D4F85480DFF818A100274FF001099B
:10304000A36D9B685FFA87FB5B4597D308EB4B1337
:10305000D3F8002902F44022B2F5802F22D1D3F810
:103060000029002A1EDAD3F8002942F09042C3F862
:103070000029D3F80029002AFBDB5946606DFFF7D1
:103080003DFC228909FA0BF322EA0303238104EBB6
:103090008B03DB689B6813B15946504698475846E6
:1030A000FFF736FC0137CBE708EB4112D2F8003BC3
:1030B00003F44023B3F5802F10D1D2F8003B002B4E
:1030C0000CDA628909FA01F322EA0303638104EB53
:1030D0008103DB68DB680BB150469847013756E740
:1030E0009C0708BF0A68072B98BF027003F1010311
:1030F0009CBF120A013069E7023304EB830201F539
:103100008051526890690268D0F808C04068A2EB0C
:10311000000E0022104697420AD104EB8304636834
:103120009B699A683A449A605A6817445F6050E70E
:1031300012F0030F08BF0868964588BF8CF800009E
:1031400002F1010284BF000A0CF1010CE3E700BFA9
:10315000203B0020436D03EB4111D1F8003B43F4C9
:103160000013C1F8003B7047436D03EB4111D1F8E8
:10317000003943F40013C1F800397047436D03EB85
:103180004111D1F8003B23F40013C1F8003B704714
:10319000436D03EB4111D1F8003923F40013C1F85A
:1031A0000039704730B5039C0172043304FB0325DA
:1031B000C361049B03630021059B00604060C16004
:1031C000426102618561046242628162C16243635D
:1031D00030BD00000022416A41610161C26082622B
:1031E000C2626FF00101FEF7BDBF000003694269D2
:1031F000934203D1C2680AB100207047181D70477E
:1032000003691960C2680132C260C26913448269ED
:103210000361934224BF436A03610021FEF796BF16
:1032200038B504460D46E3683BB16269131D126868
:10323000A3621344E362002038BD237A33B92946E0
:103240002046FEF773FF0028EDDA38BD6FF001006D
:10325000FBE70000C368C269013BC36043691344D4
:1032600082694361934224BF436A436100238362BE
:10327000036B03B11847704770B52023044683F3EE
:103280001188866A3EB9FFF7CBFF054618B186F371
:103290001188284670BDA36AE26A13F8015BA36235
:1032A000934202D32046FFF7D5FF002383F3118812
:1032B000EFE700002DE9F84F04460E469046994688
:1032C000202787F311880025AA46D4F828B0BBF13F
:1032D000000F09D149462046FFF7A2FF20B18BF32A
:1032E00011882846BDE8F88FA16AE36AA8EB050BB0
:1032F0005B1A9B4528BF9B46BBF1400F1BD9334649
:1033000001F1400251F8040B43F8040B9142F9D14A
:10331000A36A40334036A3624035A26AE36A9A4208
:1033200002D32046FFF796FF8AF311884545D8D28D
:1033300087F31188C9E730465A46FDF759FDA36A5D
:103340005B445E44A3625D44E7E7000010B5029C65
:103350000172043303FB0421C36100238362C3624F
:10336000039B0363049B00604060C4604261026190
:10337000816104624262436310BD0000026AC26060
:10338000426A4261026100228262C2626FF0010100
:10339000FEF7E8BE436902699A4203D1C2680AB1E6
:1033A00000207047184650F8043B0B60704700003F
:1033B000C368C2690133C3604369134482694361CE
:1033C000934224BF436A43610021FEF7BFBE000061
:1033D00038B504460D46E3683BB123691A1DA26265
:1033E000E2691344E362002038BD237A33B92946E9
:1033F0002046FEF79BFE0028EDDA38BD6FF0010095
:10340000FBE7000003691960C268013AC260C26943
:10341000134482690361934224BF436A036100231A
:103420008362036B03B118477047000070B5202317
:1034300004460E4683F31188856A35B91146FFF7B5
:10344000C7FF10B185F3118870BDA36A1E70A36A0F
:10345000E26A01339342A36204D3E169204604394E
:10346000FFF7D0FF002080F3118870BD2DE9F84FE1
:1034700004460D4691469A464FF0200888F311887D
:103480000026B346A76A4FB951462046FFF7A0FF72
:1034900020B187F311883046BDE8F88FA06AE76A4B
:1034A000A9EB06033F1A9F4228BF1F46402F1BD996
:1034B00005F1400355F8042B40F8042B9D42F9D147
:1034C000A36A4033A3624036A26AE36A9A4204D3F5
:1034D000E16920460439FFF795FF8BF311884E45CB
:1034E000D9D288F31188CDE729463A46FDF780FC0A
:1034F000A36A3B443D44A3623E44E5E70269436955
:103500009A4203D1C3681BB9184670470023FBE7F2
:10351000836A002BF8D0043B9B1AF5D01360C36874
:10352000013BC360C3691A44836902619A4224BFA4
:10353000436A0361002383620123E5E700F034B9A5
:10354000034B002258631A610222DA60704700BF01
:10355000000C0040014B0022DA607047000C004074
:10356000014B5863704700BF000C0040FEE70000AD
:1035700010B5174CFEF7E0FCFEF702FE802215495D
:103580002046FEF787FD012344F8180C0374124B04
:10359000124AD96821F4E0610904090C0A43104970
:1035A000DA60CA6842F08072CA600E490A6842F066
:1035B00001020A601022DA77202283F822200023F9
:1035C00083F3118862B60848BDE81040FEF784BD59
:1035D0007C330020303E000800ED00E00003FA05D7
:1035E000F0ED00E0001000E0383E00082DE9F84F53
:1035F0001F4CDFF88090656904F114074FF0000854
:10360000D9F82430266AAA689E1B96421DD34FF033
:10361000200AAA68236AD5F80CB0134423622B68E9
:10362000BB425F60A6EB02066361C5F80C8001D166
:10363000FFF790FF88F311882869D8478AF311882B
:103640006569AB689E42E4D2DAE76269BA420CD09F
:10365000916823628E1B9660A86802282CBF1818F8
:10366000981CBDE8F84FFFF77BBFBDE8F88F00BF9F
:1036700054330020000C0040034B59685A68521A1A
:103680009042FBD8704700BF001000E04B684360D9
:103690008B688360CB68C3600B6943614B690362CD
:1036A0008B6943620B6803607047000008B5224BCA
:1036B00022481A6940F2FF110A431A611A6922F47A
:1036C000FF7222F001021A611A691A6B0A431A6327
:1036D0001A6D0A431A651A4A1B6D1146FFF7D6FF89
:1036E000184802F11C01FFF7D1FF174802F1380119
:1036F000FFF7CCFF154802F15401FFF7C7FF14484C
:1037000002F17001FFF7C2FF124802F18C01FFF7CE
:10371000BDFF114802F1A801FFF7B8FF0F4802F101
:10372000C401FFF7B3FF0E4802F1E001FFF7AEFF5F
:10373000BDE8084000F0A4B8003802400000024094
:10374000583E00080004024000080240000C0240FD
:10375000001002400014024000180240001C024009
:103760000020024008B500F0FFF9FFF701FFFFF766
:1037700039F8BDE80840FEF70DBE000070470000B4
:10378000084B1A69920710B508D500241C61202344
:1037900083F31188FFF72AFF84F31188BDE81040F6
:1037A000FFF742B8000C0040104B1A6C42F00802C0
:1037B0001A641A6E42F008021A660D4A1B6E93686C
:1037C00043F0080393600B4B53229A624FF0FF3291
:1037D000DA6200229A615A63DA605A6001225A6101
:1037E00008211A603220FDF771BD00BF0038024089
:1037F000002004E0000C00401F4B1A696FEAC2521F
:103800006FEAD2521A611A69C2F308021A614FF0C4
:10381000FF301A695A69586100215A6959615A6919
:103820001A6A62F080521A621A6A02F080521A62B0
:103830001A6A5A6A58625A6A59625A6A1A6C42F08B
:1038400080521A641A6E42F080521A661A6E0B4A3F
:10385000106840F480701060186F00F44070B0F58C
:10386000007F1EBF4FF4803018671967536823F438
:103870000073536000F058B90038024000700040F7
:10388000324B4FF080521A64314A4FF4404111607C
:103890001A6842F001021A601A689207FCD59A6809
:1038A00022F003029A60294B19469A6812F00C0222
:1038B000FBD1186800F0F90018609A601A6842F4A9
:1038C00080321A600B689B03FCD54B6F43F00103F9
:1038D0004B671E4B5A6F9007FCD51E4A5A601A68F8
:1038E00042F080721A601A4A53685904FCD5174B8B
:1038F0001A689201FCD5184A9A600322C3F88C20FA
:10390000164B1A68164B9A42164B1BD1164A116871
:10391000164A914216D140F205121A600B4B9A6872
:1039200042F002029A609A6802F00C02082AFAD168
:103930005A6C42F480425A645A6E42F480425A668B
:103940005B6E704740F20572E7E700BF0038024047
:10395000007000401854400700948838002004E0AC
:1039600011640020003C024000ED00E041C20F4124
:10397000084A08B5536911680B4003F0010353610D
:1039800023B1054A13680BB150689847BDE8084059
:10399000FEF74ABF003C01409C250020084A08B5BC
:1039A000536911680B4003F00203536123B1054AC8
:1039B00093680BB1D0689847BDE80840FEF734BF64
:1039C000003C01409C250020084A08B55369116855
:1039D0000B4003F00403536123B1054A13690BB193
:1039E00050699847BDE80840FEF71EBF003C014003
:1039F0009C250020084A08B5536911680B4003F064
:103A00000803536123B1054A93690BB1D069984704
:103A1000BDE80840FEF708BF003C01409C2500209F
:103A2000084A08B5536911680B4003F0100353614D
:103A300023B1054A136A0BB1506A9847BDE80840A4
:103A4000FEF7F2BE003C01409C250020174B10B54C
:103A50005C691A68144004F478725A61A30604D5AC
:103A6000134A936A0BB1D06A9847600604D5104A8E
:103A7000136B0BB1506B9847210604D50C4A936B1E
:103A80000BB1D06B9847E20504D5094A136C0BB112
:103A9000506C9847A30504D5054A936C0BB1D06CC4
:103AA0009847BDE81040FEF7BFBE00BF003C014094
:103AB0009C2500201A4B10B55C691A68144004F468
:103AC0007C425A61620504D5164A136D0BB1506DE4
:103AD0009847230504D5134A936D0BB1D06D9847D1
:103AE000E00404D50F4A136E0BB1506E9847A10441
:103AF00004D50C4A936E0BB1D06E9847620404D57E
:103B0000084A136F0BB1506F9847230404D5054A38
:103B1000936F0BB1D06F9847BDE81040FEF784BE9D
:103B2000003C01409C250020062108B50846FDF711
:103B3000CDFB06210720FDF7C9FB06210820FDF774
:103B4000C5FB06210920FDF7C1FB06210A20FDF770
:103B5000BDFB06211720FDF7B9FB06212820BDE893
:103B60000840FDF7B3BB000008B5FFF745FEFDF7C1
:103B700029FAFDF751FDFDF73DFFFDF711FEFFF7B7
:103B8000FDFDBDE80840FFF7D9BC0000034611F871
:103B9000012B03F8012B002AF9D1704712101213E0
:103BA0001211000053544D3332463F3F3F00000096
:103BB000012033000010410101105A010310590186
:103BC0000710310100000000A43B00083F00000086
:103BD00013040000043C00083F000000190400002A
:103BE0000E3C00083F00000021040000183C0008C3
:103BF0003F000000943300201C260020842A00206F
:103C0000EC2E002053544D33324634307800535458
:103C10004D3332463432780053544D3332463434C7
:103C20003658580000960000000000000000000018
:103C3000000000000000000000000000E115000886
:103C4000CD15000809160008F51500080116000832
:103C5000ED150008D9150008C5150008151600084F
:103C60000000000019170008051700084117000898
:103C70002D1700083917000825170008111700082C
:103C8000FD1600089D17000800000000010000005C
:103C900000000000020000000000000045190008BC
:103CA000AD190008400040002C3800203C380020AE
:103CB00002000000000000000300000000000000FF
:103CC000F119000800000000100000004C3800202E
:103CD000000000000100000000000000203B002068
:103CE000010102004172647550696C6F74002542D5
:103CF0004F415244252D424C002553455249414CD9
:103D000025000000352300089D220008B118000896
:103D100019230008430000001C3D0008090243006D
:103D2000020100C032090400000102020100052462
:103D300000100105240100010424020205240600EC
:103D400001070582030800FF09040100020A0000C0
:103D50000007050102400000070581024000000045
:103D600012000000683D000812011001020000402E
:103D70000912415700020102030100000403090473
:103D800025424F4152442500666D7576330030312F
:103D900032333435363738394142434445460000E2
:103DA0000040000000400000004000000040000013
:103DB00000000100000002000000020000000200FC
:103DC00000000200000002000000020000000200EB
:103DD00000400000004000000040000000400000E3
:103DE00000000100000002000000020000000200CC
:103DF00000000200000002000000020000000200BB
:103E000000000000391B0008191E0008C51E00082C
:103E100040004000803B0020803B0020010000006B
:103E2000903B0020800000004001000003000000E3
:103E30006D61696E00000000503E0008983B002054
:103E4000903D0020010000006D35000800000000DA
:103E500069646C65000000000000802A0002000018
:103E6000AAAAAAAA00000000FFFF000000000000AC
:103E700000A00A000000000000000000AAAAAAAAF0
:103E800000000000FFFF0000000000000000000034
:103E90001400005400000000AAAAAAAA14000054AA
:103EA000FFFF0000000000000000000080699A0190
:103EB00000000000AAAA8AAA40555501FFFF000091
:103EC00000707007777000000081020100000000A0
:103ED000AAAAAAAA00410100FFFF0000000000807A
:103EE000080000000000000000000000AAAAAAAA22
:103EF00000000000FFFF00000000000000000000C4
:103F00000000000000000000AAAAAAAA0000000009
:103F1000FFFF0000000000000000000000000000A3
:103F2000000000000A000000000000000300000084
:103F30000000000000000000000000000000000081
:103F40000000000000000000000000000000000071
:103F50000000000000000000FF00960000000008C4
:103F6000040000007C3D000800000000000000008C
:103F70000000000000000000000000000000000041
:103F8000FFFFFFFFFFFFFFFFFFFFFFFFFFFFFFFF41
:103F9000FFFFFFFFFFFFFFFFFFFFFFFFFFFFFFFF31
:103FA000FFFFFFFFFFFFFFFFFFFFFFFFFFFFFFFF21
:103FB000FFFFFFFFFFFFFFFFFFFFFFFFFFFFFFFF11
:103FC000FFFFFFFFFFFFFFFFFFFFFFFFFFFFFFFF01
:103FD000FFFFFFFFFFFFFFFFFFFFFFFFFFFFFFFFF1
:103FE000FFFFFFFFFFFFFFFFFFFFFFFFFFFFFFFFE1
:103FF000FFFFFFFFFFFFFFFFFFFFFFFFFFFFFFFFD1
:104000000006002015530008992A0E088142000876
:10401000212A0E08192A0E081D2A0E081753000817
:10402000175300081753000817530008C1C8130896
:1040300017530008175300081753000817530008B8
:1040400017530008175300081753000817530008A8
:104050001753000817530008992C1408C12C140892
:10406000E92C1408112D1408392D1408CDD013088B
:10407000F5D0130821D113084DD1130879D11308B5
:10408000A1D11308CDD1130851D01308F91B0E0884
:10409000091C0E081D1C0E0817530008612D14087A
:1040A000AD2E1408B12E1408C52E1408C92E1408FC
:1040B000CD2E140817530008E12E140825DA130832
:1040C00039DA13085DDA130871DA13081753000898
:1040D0001753000817530008352E1408492E1408EA
:1040E000C52D14081753000817530008175300086C
:1040F000175300081753000817530008F9D1130885
:104100001753000869DE1308F52E1408175300082A
:104110005D2E1408175300081753000817530008A2
:1041200025D213084DD2130879D21308A5D213084B
:10413000D1D213081753000817530008311C0E087A
:10414000411C0E08551C0E08175300082928140896
:10415000F9D2130825D3130851D31308712E14086C
:104160001753000817530008175300081753000887
:104170001753000817530008175300081753000877
:104180001753000817530008852E1408992E140899
:104190001753000817530008175300081753000857
:1041A0001753000817530008175300081753000847
:1041B0001753000817530008175300081753000837
:1041C0001753000817530008175300081753000827
:1041D0001753000817530008175300081753000817
:1041E000DD870008B1C10008C90401080D6E01088F
:1041F000F5D70108F98B020821E50208756A030862
:10420000B9C604080DF8060841FE060879900708AB
:104210002D010808F50808082D0C08081D87080856
:10422000E1AE08084DB80808DD460908617D0A08B6
:1042300059150B08B1220B08CD1E0E081D230E08C0
:10424000D93F0E0845B90F08E9FF0F08314910089A
:10425000DD94100829171208DD4D1208A168120814
:10426000D1A51208C1C1120805EC120899F612086E
:1042700079271308992E13080000000000000000A1
:10428000EFF30383EFF30982EFF30881DFF814D033
:104290002DE9FE4F684601F0A9F9BDE8FE4F8D46B5
:1042A0007047000094330020F1EE101AA0EC200AB1
:1042B00001607047A0EC108A704700BF81F0004198
:1042C00002E000BF83F0004330B54FEA41044FEAFB
:1042D000430594EA050F08BF90EA020F1FBF54EA96
:1042E000000C55EA020C7FEA645C7FEA655C00F032
:1042F000E2804FEA5454D4EB5555B8BF6D420CDD03
:104300002C4480EA020281EA030382EA000083EA85
:10431000010180EA020281EA0303362D88BF30BD25
:1043200011F0004F4FEA01314FF4801C4CEA11317B
:1043300002D0404261EB410113F0004F4FEA0333DA
:104340004CEA133302D0524263EB430394EA050F65
:1043500000F0A780A4F10104D5F1200E0DDB02FAD4
:104360000EFC22FA05F2801841F1000103FA0EF268
:10437000801843FA05F359410EE0A5F120050EF12E
:10438000200E012A03FA0EFC28BF4CF0020C43FA5F
:1043900005F3C01851EBE37101F0004507D54FF06C
:1043A000000EDCF1000C7EEB00006EEB0101B1F5BC
:1043B000801F1BD3B1F5001F0CD349085FEA300002
:1043C0004FEA3C0C04F101044FEA445212F5800F0D
:1043D00080F09A80BCF1004F08BF5FEA500C50F1AA
:1043E000000041EB045141EA050130BD5FEA4C0C8D
:1043F000404141EB0101013C28BFB1F5801FE9D2EA
:1044000091F0000F04BF01460020B1FA81F308BF0C
:104410002033A3F10B03B3F120020CDA0C3208DDD8
:1044200002F1140CC2F10C0201FA0CF021FA02F1B3
:104430000CE002F11402D8BFC2F1200C01FA02F123
:1044400020FA0CFCDCBF41EA0C019040E41AA2BF48
:1044500001EB0451294330BD6FEA04041F3C1CDA10
:104460000C340EDC04F11404C4F1200220FA04F030
:1044700001FA02F340EA030021FA04F345EA0301DA
:1044800030BDC4F10C04C4F1200220FA02F001FA9C
:1044900004F340EA0300294630BD21FA04F029461E
:1044A00030BD94F0000F83F4801306BF81F48011B7
:1044B0000134013D4EE77FEA645C18BF7FEA655C2A
:1044C00029D094EA050F08BF90EA020F05D054EAFC
:1044D000000C04BF1946104630BD91EA030F1EBF01
:1044E0000021002030BD5FEA545C05D14000494105
:1044F00028BF41F0004130BD14F580043CBF01F5F8
:10450000801130BD01F0004545F0FE4141F47001DD
:104510004FF0000030BD7FEA645C1ABF19461046B8
:104520007FEA655C1CBF0B46024650EA013406BFB9
:1045300052EA033591EA030F41F4002130BD00BF78
:1045400090F0000F04BF0021704730B54FF4806435
:1045500004F132044FF000054FF0000150E700BFB6
:1045600090F0000F04BF0021704730B54FF4806415
:1045700004F1320410F0004548BF40424FF0000102
:104580003EE700BF42004FEAE2014FEA31014FEA45
:1045900002701FBF12F07F4393F07F4F81F0605194
:1045A000704732F07F4208BF704793F07F4F04BFDF
:1045B00041F40021704730B54FF4607401F00045BC
:1045C00021F000411CE700BF50EA010208BF70471C
:1045D00030B54FF000050AE050EA010208BF70470D
:1045E00030B511F0004502D5404261EB41014FF476
:1045F000806404F132045FEA915C3FF4D8AE4FF07E
:1046000003025FEADC0C18BF03325FEADC0C18BF60
:10461000033202EBDC02C2F1200300FA03FC20FAB1
:1046200002F001FA03FE40EA0E0021FA02F11444FE
:10463000BDE600BF70B54FF0FF0C4CF4E06C1CEA17
:1046400011541DBF1CEA135594EA0C0F95EA0C0F88
:1046500000F0DEF82C4481EA030621EA4C5123EAFB
:104660004C5350EA013518BF52EA033541F480112A
:1046700043F4801338D0A0FB02CE4FF00005E1FBDD
:1046800002E506F00042E0FB03E54FF00006E1FB27
:1046900003569CF0000F18BF4EF0010EA4F1FF046A
:1046A000B6F5007F64F5407404D25FEA4E0E6D41AA
:1046B00046EB060642EAC62141EA55514FEAC520BB
:1046C00040EA5E504FEACE2EB4F1FD0C88BFBCF537
:1046D000E06F1ED8BEF1004F08BF5FEA500E50F1E8
:1046E000000041EB045170BD06F0004646EA0101AE
:1046F00040EA020081EA0301B4EB5C04C2BFD4EBE0
:104700000C0541EA045170BD41F480114FF0000ED8
:10471000013C00F3AB8014F1360FDEBF002001F046
:10472000004170BDC4F10004203C35DA0C341BDCC0
:1047300004F11404C4F1200500FA05F320FA04F092
:1047400001FA05F240EA020001F0004221F00041C6
:1047500010EBD37021FA04F642EB06015EEA430E39
:1047600008BF20EAD37070BDC4F10C04C4F1200569
:1047700000FA04F320FA05F001FA04F240EA02001C
:1047800001F0004110EBD37041F100015EEA430EED
:1047900008BF20EAD37070BDC4F1200500FA05F20D
:1047A0004EEA020E20FA04F301FA05F243EA02038C
:1047B00021FA04F001F0004121FA04F220EA02009B
:1047C00000EBD3705EEA430E08BF20EAD37070BDE1
:1047D00094F0000F0FD101F00046400041EB0101C1
:1047E00011F4801F08BF013CF7D041EA060195F0A3
:1047F000000F18BF704703F00046520043EB03035D
:1048000013F4801F08BF013DF7D043EA0603704749
:1048100094EA0C0F0CEA135518BF95EA0C0F0CD054
:1048200050EA410618BF52EA4306D1D181EA03019A
:1048300001F000414FF0000070BD50EA410606BF94
:104840001046194652EA430619D094EA0C0F02D1D9
:1048500050EA013613D195EA0C0F05D152EA03361E
:104860001CBF104619460AD181EA030101F000413C
:1048700041F0FE4141F470014FF0000070BD41F085
:10488000FE4141F4780170BD70B54FF0FF0C4CF45F
:10489000E06C1CEA11541DBF1CEA135594EA0C0F7E
:1048A00095EA0C0F00F0A7F8A4EB050481EA030ECB
:1048B00052EA03354FEA013100F088804FEA0333B2
:1048C0004FF0805545EA131343EA12634FEA022280
:1048D00045EA111545EA10654FEA00260EF0004141
:1048E0009D4208BF964244F1FD0404F5407402D293
:1048F0005B084FEA3202B61A65EB03055B084FEA24
:1049000032024FF480104FF4002CB6EB020E75EB20
:10491000030E22BFB61A754640EA0C005B084FEA48
:104920003202B6EB020E75EB030E22BFB61A7546C5
:1049300040EA5C005B084FEA3202B6EB020E75EB10
:10494000030E22BFB61A754640EA9C005B084FEA88
:104950003202B6EB020E75EB030E22BFB61A754695
:1049600040EADC0055EA060E18D04FEA051545EA84
:1049700016754FEA06164FEAC30343EA52734FEA2D
:10498000C2025FEA1C1CC0D111F4801F0BD141EAA6
:1049900000014FF000004FF0004CB6E711F4801F0B
:1049A00004BF01430020B4F1FD0C88BFBCF5E06FEB
:1049B0003FF6AFAEB5EB030C04BFB6EB020C5FEAFB
:1049C000500C50F1000041EB045170BD0EF0004E50
:1049D0004EEA113114EB5C04C2BFD4EB0C0541EA82
:1049E000045170BD41F480114FF0000E013C90E67F
:1049F00045EA060E8DE60CEA135594EA0C0F08BF43
:104A000095EA0C0F3FF43BAF94EA0C0F0AD150EA41
:104A100001347FF434AF95EA0C0F7FF425AF1046D4
:104A200019462CE795EA0C0F06D152EA03353FF4FC
:104A3000FDAE1046194622E750EA410618BF52EA79
:104A400043067FF4C5AE50EA41047FF40DAF52EA4D
:104A500043057FF4EBAE12E74FF0FF3C06E000BFEA
:104A60004FF0010C02E000BF4FF0010C4DF804CDF7
:104A70004FEA410C7FEA6C5C4FEA430C18BF7FEAB7
:104A80006C5C1BD001B050EA410C0CBF52EA430CE5
:104A900091EA030F02BF90EA020F0020704710F165
:104AA000000F91EA030F58BF994208BF90422CBFF4
:104AB000D8176FEAE37040F0010070474FEA410CED
:104AC0007FEA6C5C02D150EA013C07D14FEA430C0B
:104AD0007FEA6C5CD6D152EA033CD3D05DF8040B7C
:104AE000704700BF8446104662468C4619466346AE
:104AF00000E000BF01B5FFF7B7FF002848BF10F185
:104B0000000F01BD4DF808EDFFF7F4FF0CBF0120C9
:104B100000205DF808FB00BF4DF808EDFFF7EAFF45
:104B200034BF012000205DF808FB00BF4DF808ED00
:104B3000FFF7E0FF94BF012000205DF808FB00BFF5
:104B40004DF808EDFFF7CEFF94BF012000205DF87F
:104B500008FB00BF4DF808EDFFF7C4FF34BF01208C
:104B600000205DF808FB00BF4FEA410C7FEA6C5C57
:104B700002D150EA013C0AD14FEA430C7FEA6C5C57
:104B800002D152EA033C02D14FF0000070474FF0CF
:104B9000010070474FEA410212F5001215D211D5FB
:104BA0006FF47873B3EB625212D94FEAC12343F02A
:104BB000004343EA505311F0004F23FA02F018BFAC
:104BC000404270474FF00000704750EA013005D175
:104BD00011F0004008BF6FF0004070474FF0000038
:104BE000704700BF4A0011D212F5001211D20DD544
:104BF0006FF47873B3EB62520ED44FEAC12343F0E3
:104C0000004343EA505323FA02F070474FF000008C
:104C1000704750EA013002D14FF0FF3070474FF03B
:104C2000000070474FEA4102B2F1E04324BFB3F500
:104C3000001CDCF1FE5C0DD901F0004C4FEAC00213
:104C40004CEA5070B2F1004F40EB830008BF20F0F7
:104C50000100704711F0804F21D113F13872BCBFB1
:104C600001F00040704741F480114FEA5252C2F106
:104C70001802C2F1200C10FA0CF320FA02F018BF4F
:104C800040F001004FEAC1234FEAD32303FA0CFCA2
:104C900040EA0C0023FA02F34FEA4303CCE77FEA31
:104CA000625307D150EA01331EBF4FF0FE4040F47B
:104CB0004000704701F0004040F0FE4040F400002A
:104CC000704700BF80F0004002E000BF81F000416B
:104CD00042001FBF5FEA410392EA030F7FEA226CA2
:104CE0007FEA236C6AD04FEA1262D2EB1363C1BF32
:104CF000D218414048404140B8BF5B42192B88BFA1
:104D0000704710F0004F40F4000020F07F4018BFC3
:104D1000404211F0004F41F4000121F07F4118BFE3
:104D2000494292EA030F3FD0A2F1010241FA03FC8B
:104D300010EB0C00C3F1200301FA03F100F0004373
:104D400002D5494260EB4000B0F5000F13D3B0F13B
:104D5000807F06D340084FEA310102F10102FE2AAA
:104D600051D2B1F1004F40EBC25008BF20F001001A
:104D700040EA03007047490040EB0000013A28BFB9
:104D8000B0F5000FEDD2B0FA80FCACF1080CB2EB3C
:104D90000C0200FA0CF0AABF00EBC25052421843BA
:104DA000BCBFD0401843704792F0000F81F400015F
:104DB00006BF80F400000132013BB5E74FEA410332
:104DC0007FEA226C18BF7FEA236C21D092EA030F9E
:104DD00004D092F0000F08BF0846704790EA010F18
:104DE0001CBF0020704712F07F4F04D1400028BF45
:104DF00040F00040704712F100723CBF00F5000027
:104E0000704700F0004343F0FE4040F4000070475C
:104E10007FEA226216BF08467FEA23630146420208
:104E200006BF5FEA412390EA010F40F4800070471B
:104E30004FF0000304E000BF10F0004348BF4042C1
:104E40005FEA000C08BF704743F0964301464FF0FD
:104E500000001CE050EA010208BF70474FF0000359
:104E60000AE000BF50EA010208BF704711F000439A
:104E700002D5404261EB41015FEA010C02BF84466A
:104E80000146002043F0B64308BFA3F18053A3F5C9
:104E90000003BCFA8CF2083AA3EBC25310DB01FA10
:104EA00002FC634400FA02FCC2F12002BCF1004F94
:104EB00020FA02F243EB020008BF20F00100704725
:104EC00002F1200201FA02FCC2F1200250EA4C0079
:104ED00021FA02F243EB020008BF20EADC707047BF
:104EE0007BB972B90029BEBF00204FF0004106E037
:104EF00008BF00281CBF6FF000414FF0FF3000F0EA
:104F000007BAADF1080C6DE904CE002909DB002BCE
:104F10001ADB00F095F8DDF804E0DDE9022304B0C7
:104F20007047404261EB4101002B1BDB00F088F829
:104F3000DDF804E0DDE9022304B0404261EB410109
:104F4000524263EB43037047524263EB430300F06A
:104F500077F8DDF804E0DDE9022304B0404261EBBC
:104F600041017047524263EB430300F069F8DDF8FA
:104F700004E0DDE9022304B0524263EB43037047CF
:104F800053B94AB9002908BF00281CBF4FF0FF31B0
:104F90004FF0FF3000F0BCB9ADF1080C6DE904CE64
:104FA00000F04EF8DDF804E0DDE9022304B07047BC
:104FB000430803F05533C01A830803F0333300F07D
:104FC0003330184400EB101000F00F3000EB0020DD
:104FD00000EB0040000E704707EE900AF5EEC07A35
:104FE000F1EE10FA01D400F00BB8F1EE677A08B5D3
:104FF00017EE900A00F004F8404261EB410108BD51
:10500000D0B5FFF7BFFA0C4B002206460F46FFF75C
:1050100011FBFFF7E7FD0446FFF792FA074B00226A
:10502000FFF708FB02460B4630463946FFF74AF9C0
:10503000FFF7D8FD2146D0BD0000F03D0000F04153
:105040002DE9F047089D04468E46002B4DD18A423B
:10505000944669D9B2FA82F252B101FA02F3C2F16E
:10506000200120FA01F10CFA02FC41EA030E9440FF
:105070004FEA1C48210CBEFBF8F61FFA8CF708FB20
:1050800016E341EA034306FB07F199420AD91CEBF8
:10509000030306F1FF3080F01F81994240F21C812A
:1050A000023E63445B1AA4B2B3FBF8F008FB103372
:1050B00044EA034400FB07F7A7420AD91CEB0404A7
:1050C00000F1FF3380F00A81A74240F20781644477
:1050D000023840EA0640E41B00261DB1D4400023FC
:1050E000C5E900433146BDE8F0878B4209D9002D60
:1050F00000F0EF800026C5E9000130463146BDE8EA
:10510000F087B3FA83F6002E4AD18B4202D3824253
:1051100000F2F980841A61EB030301209E46002D02
:10512000E0D0C5E9004EDDE702B9FFDEB2FA82F257
:10513000002A40F09280A1EB0C014FEA1C471FFAB5
:105140008CFE0126200CB1FBF7F307FB131140EA9C
:1051500001410EFB03F0884208D91CEB010103F169
:10516000FF3802D2884200F2CB804346091AA4B22B
:10517000B1FBF7F007FB101144EA01440EFB00FEFF
:10518000A64508D91CEB040400F1FF3102D2A64564
:1051900000F2BB800846A4EB0E0440EA03409CE703
:1051A000C6F12007B34022FA07FC4CEA030C20FAB0
:1051B00007F401FA06F31C43F9404FEA1C4900FAD0
:1051C00006F3B1FBF9F8200C1FFA8CFE09FB18114D
:1051D00040EA014108FB0EF0884202FA06F20BD9C0
:1051E0001CEB010108F1FF3A80F08880884240F210
:1051F0008580A8F102086144091AA4B2B1FBF9F054
:1052000009FB101144EA014100FB0EFE8E4508D94E
:105210001CEB010100F1FF346CD28E456AD90238D3
:10522000614440EA0840A0FB0294A1EB0E01A142B8
:10523000C846A64656D353D05DB1B3EB080261EB26
:105240000E0101FA07F722FA06F3F1401F43C5E900
:10525000007100263146BDE8F087C2F12003D84036
:105260000CFA02FC21FA03F3914001434FEA1C4778
:105270001FFA8CFEB3FBF7F007FB10360B0C43EA6A
:10528000064300FB0EF69E4204FA02F408D91CEB1A
:10529000030300F1FF382FD29E422DD90238634418
:1052A0009B1B89B2B3FBF7F607FB163341EA0341B8
:1052B00006FB0EF38B4208D91CEB010106F1FF3807
:1052C00016D28B4214D9023E6144C91A46EA0046FE
:1052D00038E72E46284605E70646E3E61846F8E690
:1052E0004B45A9D2B9EB020864EB0C0E0138A3E7D9
:1052F0004646EAE7204694E74046D1E7D0467BE7BA
:10530000023B614432E7304609E76444023842E731
:10531000704700BF02E000F000F8FEE772B63748C1
:1053200080F30888364880F3098836483649086093
:1053300040F20000CCF200004EF63471CEF20001D3
:105340000860BFF34F8FBFF36F8F40F20000C0F2D1
:10535000F0004EF68851CEF200010860BFF34F8F87
:10536000BFF36F8F4FF00000E1EE100A4EF63C7174
:10537000CEF200010860062080F31488BFF36F8F1F
:105380003CF11AFF3BF1CCFF4FF055301F491B4A4F
:1053900091423CBF41F8040BFAE71D49184A91427B
:1053A0003CBF41F8040BFAE71A491B4A1B4B9A42CF
:1053B0003EBF51F8040B42F8040BF8E700201849EF
:1053C000184A91423CBF41F8040BFAE73CF1F8FE61
:1053D0003BF1FAFF144C154DAC4203DA54F8041BB0
:1053E0008847F9E703F03AF9114C124DAC4203DA61
:1053F00054F8041B8847F9E73CF1E0BE00060020A2
:10540000002200200040000808ED00E0000000201D
:105410000006002020751808002200209C31002082
:10542000A031002094AB0120E04100087842000840
:1054300078420008784200082DE9F04F2DED108ADF
:10544000C1F80CD0C3689D46BDEC108ABDE8F08F52
:10545000002383F311882846A04700203BF1E6FC97
:10546000FEE73BF153FB00DFFEE7000001F0FF0128
:10547000102A2BDB10F0070F08D010F8013B013A7F
:105480008B422DD010F0070F42B3F6D1F0B441EAB1
:10549000012141EA014122F007047FF000070023C7
:1054A000F0E80256083C85EA010586EA010685FA1D
:1054B00047F5A3FA87F586FA47F6A5FA87F68EB977
:1054C000EED1F0BC01F0FF0102F0070232B110F89A
:1054D000013B013A83EA010313B1F8D10020704780
:1054E00001387047002D06BF35460338073815F0E0
:1054F000010F07D1013015F4807F02BF013015F490
:10550000C03F0130F0BC0138704700BFEC46A0E856
:10551000F05F4FF000007047B0E8F05FE54608002C
:1055200008BF0120704700BF10F8012B11F8013BA4
:10553000012A28BF9A42F7D0D01A7047034613F8C1
:10554000012B002AFBD1181A0138704738B5002208
:10555000002304460D46FFF7DFFA28B92046294606
:10556000BDE8384000F00AB8204605F1004100F0DF
:1055700005F8404261EB410138BD00BFD0B50C4B8E
:10558000002206460F46FFF755F8FFF72BFB0446AF
:10559000FEF7D6FF074B0022FFF74CF802460B46FA
:1055A00030463946FEF78EFEFFF71CFB2146D0BD84
:1055B0000000F03D0000F04110B5044620461CB14B
:1055C00054F80C3B013300D110BD0822012100F03A
:1055D00067FB54F80C0C54F8082C14F8041C121A2D
:1055E000B2FBF1F200F05CFBE8E700002DE9F041CE
:1055F000D0E90031C26A5C4C12F0040FA6B018BFAB
:105600000B46CDE90003D0064CBF03F1200203F1A5
:1056100068020392DA699B6900210291D209039919
:105620001B8802F004020A4303924FF0E02203F4C5
:105630007F43D2F8882D02F4A002B2F5A00F08BF74
:105640000122A3F53E4108BF02924B424B41049315
:1056500004260127454D03A82C6000F01FFA44489A
:105660000422012100F01CFB0422012102A800F009
:1056700017FB01981022012100F012FB0098202254
:1056800001210C3000F00CFB0198042201211030A4
:1056900000F006FB0422012103A800F001FB0198A1
:1056A0000C220121143000F0FBFA0C220098012199
:1056B00000F0F6FA029BDA071ED5009BDB6ADB06D8
:1056C0004DD415A8FEF7F6FDDDF804C00DF1140E5B
:1056D0000CF120030CF1600818685968724603C287
:1056E000083343459646F7D1DCF860302593842291
:1056F000012105A800F0D4FA00F0B8F8FFF75CFF2C
:105700004FF0E023D3F8003D03F47023B3F5402FAE
:105710000ED0184B05931433069305A84FF0FF33B2
:10572000CDE908338DF81C608DF82870FFF744FF31
:105730002B68A34206D0104B05930422012105A833
:1057400000F0AEFA00F020FA002883D0049B1BB1D1
:10575000019A93690233936126B0BDE8F08105A8F0
:10576000FEF7A2FDC3E700BFED55CEACA03100208F
:10577000A4B2140828ED00E0ACCE55ED08B5272002
:1057800039F154FC104B1A6A42F480221A621A6AE8
:1057900022F480221A621A6A1A6C42F480221A6475
:1057A0001A6E42F480221A661B6E084B2E229A60F3
:1057B00000221A601A685A6842F20C02DA60044B3E
:1057C00001221A7008BD00BF0038024000480040A6
:1057D000CC33002037B50E4D2A78202A15D10D4C38
:1057E0000D4823680D49019218443CF123F82368C1
:1057F000019A0A48203300212360297040F106FEF7
:1058000003B0BDE830403CF1A1BC03B030BD00BFE7
:1058100094330020BC330020C08418089633002045
:10582000014B1868704700BFFCFF1F08014B02487E
:10583000C01A7047C084180800002008004870474C
:10584000C08418080749084B00225B1A9A4201D30A
:105850000120704751F8040B013001D10432F5E703
:1058600000207047C0841808000020082DE9F74F79
:105870005C4BDFF89C911A685B4B5C4F5C4CDFF82B
:1058800094A102F56A581A7808F1180890443BF17F
:1058900061F802250646A9EB070B0EB14E2D4AD939
:1058A000A9EB0702B2EB080700F18F804E2D00F242
:1058B0008C80DFF864C14F4EACEB06006B1C0C21F2
:1058C000B842DBB205FB01F16FDD601866504FF0A6
:1058D000010C3E4480F808C046609046B2EB0802D6
:1058E00013D44F2B11D0444E44481946AB1C351AE3
:1058F00095424FF00C05DBB205FB01F15FDD651849
:105900000126024460502E726A600C225343E21852
:10591000012111724FF0FF31E1505160384B1B787B
:105920002BB1384B1B682360374B1B6863603048D2
:1059300003B0BDE8F08F336AF06953450ABF334BBB
:10594000F31AA3EB0A0380B101933CF1EDF8019B3C
:1059500058B12A460C214A43A01801210172F1696D
:10596000A15001350D31EDB241600C2000FB05FC6A
:1059700004EB0C02012144F80C6006F13C0C11729E
:10598000C2F804C06A18D2B24243A0189844017207
:10599000316AA15002351944D845EDB2416014D2A4
:1059A00030463AF1E7FF064677E767184FF0010EF9
:1059B000665087F808E0C7F804C080448EE7621894
:1059C00001256050157256609FE74F2D01D82B4678
:1059D0009BE7012384F8BC334FF0FF33C4E9ED3378
:1059E0009CE700BFBC33002094330020C08418081B
:1059F00004220020A03100200000032098AB0120E9
:105A000000220020C0330020B833002000220020F4
:105A1000000020080006002094AB01200C4B1B78EE
:105A200010B50BB9FFF7AAFE0A490B4800230A6814
:105A30009206FCD54A681C5CD2B2944205D101336F
:105A4000DBB20E2BF3D1002010BD0023EFE700BF27
:105A5000CC33002000480040A8B2140838B5084BE9
:105A60001B7804460BB9FFF789FE064DE4B26C6063
:105A70002B685B0600D538BD3CF168FBF8E700BF3A
:105A8000CC3300200048004010B5441E14F8010F2C
:105A900000B910BDFFF7E2FFF8E7000070B502683B
:105AA0000446EFF30581D9205369C9B2DCF0BAFF8F
:105AB000294B1B78A3B194E80300284B83E803002B
:105AC0002748FFF7E1FF6368B3B12648FFF7DCFF23
:105AD0002548FFF7D9FFFFF7A1FF2448FFF7D4FFC0
:105AE000234D2B783BB124681CB120463CF11CF8B7
:105AF00020B900232B7070BD1E48E7E720463CF11B
:105B00002BF800F2145084421B4E1FD220463CF169
:105B100023F8306020463CF139F804F5E053834225
:105B2000164E17D920463CF131F83060144A002354
:105B30001360144A1370FFF785FE0028D9D03CF19A
:105B400005FBBDE8704001203BF1E8BEA4F2145310
:105B50003360DFE73360E9E795330020C43300208A
:105B6000B8B21408BDB21408CEB21408BAB2140800
:105B700000220020C8B21408C0330020B83300202F
:105B8000BC33002094330020284B1A7870B542B102
:105B90002748FFF779FF274B5868003818BF0120C6
:105BA00070BD254A107800283CD0244E244C336820
:105BB0002448254D21781A1D2D1A0A44AA4205D3DE
:105BC000224A4FF0FF31D161202222702278D2B1D7
:105BD00003F120018D4205D81F2A9FBF1B4AD361C4
:105BE000202222701949202218443BF123FE3268FA
:105BF000237816481344002120223360217040F19D
:105C000005FC3CF1A3FA33689D4207D90F491048BF
:105C1000CB6120223BF10EFE3CF198FA00203BF1D3
:105C20007DFEB8E701221A70BAE700BF9533002065
:105C300014B31408C433002000220020BC33002019
:105C400094330020C08418080000200896330020F8
:105C5000E0FF1F082DE9F843DFF83C90DFF83C80B7
:105C600007460E460024B44201D1BDE8F88324B1B2
:105C7000230702D14846FFF707FF3D5D2B0905F0DA
:105C80000F0518F80300FFF7E9FE18F80500FFF705
:105C9000E5FE0134E7E700BFBAB2140824B31408E4
:105CA000474B1B782DE9F74F07460E4690465BB1F0
:105CB000022925D0042938D0012902D11146FFF745
:105CC000C9FF4048FFF7E0FE3F4B1B78002B4ED04A
:105CD0003E4A3F4B0025A2EB030938E037F8143069
:105CE000ADF8043024B1620702D12846FFF7CCFE9C
:105CF000022101A8FFF7AEFF0134A045EED1E0E795
:105D0000304D0024F9E757F82430019324B1A3075C
:105D100002D12846FFF7B8FE04210DEB0100FFF782
:105D200099FF0134A045EED1CBE7264D0024F9E7D9
:105D3000FFF750FD022E1DD0042E2CD0012E06D1CF
:105D40002378795D5A1C2270224AD1540135A84526
:105D50000DD0214B214C1B682278043313444B4552
:105D6000E6D31C4B4FF0FF32DA612023237003B0DF
:105D7000BDE8F08F2378DFF85CA05A1C22703A78D7
:105D80000AF80320FFF726FD23785A1C2270002210
:105D90000AF80320DAE7DFF83CB04FF0000A227877
:105DA0003B78511C23FA0AF30AF1080A0BF8023077
:105DB0002170FFF70FFDBAF1200FF0D1C6E700BF49
:105DC00095330020BAB214080022002000002008F9
:105DD000C084180896330020BC3300209433002080
:105DE000036800221B6818477FB5039140210546D0
:105DF000C2F0B6FB039A18B90124204604B070BD66
:105E0000134E039296F98E32002BF5D082F0E0FE0D
:105E1000437A039A53B982F0DBFE847A039A2CB951
:105E20000C4B40212846C2F0A3FBE6E70A4BB6F92B
:105E30009012D3F8C43FB3F906309942DCDD074B2A
:105E400000934021064B2846C2F092FB0024D4E781
:105E5000D073002038B31408D083002057B314083F
:105E600045B31408F0B50D469DB020210446C2F09C
:105E700077FB002800F0A780544E96F98E32BBB114
:105E800006F58052B6F99032D2F8C42FB2F90A1052
:105E900003F10A02914203DD40F28D32934207DCA6
:105EA0004B4B2A4620212046C2F062FB002088E0AE
:105EB00096F97D32022B05D1464B2A4620212046F9
:105EC000C2F056FBB6F85032A3F57A739BB241F696
:105ED000583293420DD8404F96EDAF7AD7F88C3FA9
:105EE000D3ED097AB4EEE77AF1EE10FA03DD3B4B1D
:105EF000D7E73B4BD5E796EDB07AD3ED0B7AB4EE0E
:105F0000E77AF1EE10FAF2DCB6F98A32002B01DC06
:105F1000344BC6E796F8742D0D2A06D8012393401A
:105F200013F4215F01D0304BBBE7304812F006FB81
:105F3000012806D1D7F8980FCFF004FA48B101280C
:105F400010D02B4B93F8551411F010011FD0294B92
:105F5000A7E7294B0093294B2A4620212046C2F06F
:105F600007FBA3E7264B93F8D83F73B125481921C7
:105F70006AF006FA48B12348D6F8686219216AF037
:105F800031FA8642DDDD204BE4E7204BE2E7602278
:105F900004A8039140F13AFA1D49D7F8940F6423FD
:105FA00003AACDF095FA18B903AB0093194BD3E7C8
:105FB0001949D7F88C0F642303AAC9F0A5FE00285D
:105FC000F2D01DB0F0BD0120FBE700BFD073002070
:105FD00060B3140873B31408D0A30020ABB3140843
:105FE0009BB31408C5B31408DAB314087CC70020A7
:105FF000D093002054B414081FB41408FAB3140842
:10600000D0830020684B00203EB414082FB414083D
:1060100069B414086DB414087FB4140870B59AB04C
:10602000602205460E4602A80021019140F1EEF9DA
:106030000A48642201A9A2F019F9044640B99DF961
:10604000043043B9064B074A31462846C2F01CFDCE
:1060500020461AB070BD01ABF5E700BFFC900020F0
:1060600084B414088DF0170807B50448D0F0C4FFB5
:1060700000F0010003B05DF804FB00BF40B3002056
:106080002DE9F043DFF848910446D9F83C04036851
:10609000A5B01B690D46984780461AF04DFD0021BA
:1060A000074660220CA80B9140F1B0F964230BAABB
:1060B0004146384619F058FF064648B93A4A0BABF4
:1060C00029462046C2F0E0FC304625B0BDE8F0830A
:1060D0003648A0F0C3F8B8F1000F03D194F91E3090
:1060E000012B0AD1324816F071FC80B9314A294699
:1060F0002046C2F0C9FC0026E6E710F0060FE3D008
:10610000A9F5C04016F062FC08B92B4AEFE703A9D5
:10611000384619F087FB28B19DF80D305B0601D594
:10612000264AE4E7DFF8AC80D8EDAB7AF5EEC07A2A
:10613000F1EE10FA4FF00003C6DD089309930A93BD
:106140000DF1200907AB019305AA06AB04A9CDF810
:10615000009038461AF04EF9484642F0B7FED8EDA6
:10616000AB7AB4EEE70AF1EE10FA01DB144ABEE7AF
:106170009DED057AF4EEC77AF1EE10FA01D8114AD6
:10618000B5E79DED047AF4EEC77AF1EE10FA01D886
:106190000D4AACE79DED067AF4EEC77AF1EE10FAFF
:1061A00092D80A4AA3E700BF3B5317089C7100200E
:1061B000D03300209CB41408B3B41408D9B4140824
:1061C000E7B41408FCB4140812B5140828B5140870
:1061D000D0930020D073002008B5064B93F85534B7
:1061E0009B0704D5044AC2F04FFC002008BD0120E3
:1061F000FCE700BFD09300203CB5140870B50E46F4
:106200009AB020210546C2F0ABF918B90124204606
:106210001AB070BDD6F0F4FB04460028F6D0002179
:10622000602202A8019140F1F1F82046642201A900
:10623000D6F0A8FB04460028E8D1034A01AB31465A
:106240002846C2F021FCE2E78DF0170870B50C4C2F
:106250000546D4F83C0403685B690E46984710B1C4
:106260000124204670BDA4F5C04016F0C1FB0446D1
:106270000028F5D1034A31462846C2F005FCF0E774
:10628000D09300204CB514082DE9704E4B4ED6F833
:10629000603493F8D5509BB082468B4665B9484B25
:1062A0001B68986A03685B6B9847044640B9454A87
:1062B00059465046C2F0E8FB28461BB0BDE8708E38
:1062C00082F086FC202183F0EBFE58B182F080FC46
:1062D0001F2183F0E5FE88B33B4A59465046C2F081
:1062E000D3FB002496F8323403F01403142B05D1A9
:1062F000364A59465046C2F0C7FB0024594650461C
:10630000C3F04CFD002188424FF0600202A808BF94
:106310000C46019140F17AF8D6F86004036801AAAE
:106320001B6864219847054680B9294A01AB594644
:106330005046C2F0A9FB2C462546BDE782F048FC3A
:10634000A52183F0ADFE0028C6D1CBE7002CF3D009
:10635000DAF808303BB9DAF8003059469B6B504602
:1063600098470446E8E759465046FFF77BFD5946F3
:1063700081465046FFF752FE09EA0000C4B2594672
:106380005046FFF729FF594604405046FFF736FFB5
:10639000594604405046FFF727FD594604405046F1
:1063A000FFF754FF594604405046C2F0B3FC59462B
:1063B00004405046C3F00AFD0440BDE7D0930020DE
:1063C00010CC002060B5140877B5140891B51408F6
:1063D000A9B5140808B5FFF757FF054A92F830141D
:1063E00060F3041182F83014024A907108BD00BFB6
:1063F000D0930020EDCE0020F7B505460F46C2F041
:10640000EBF8044678B102212846C2F0A9F8064606
:1064100048B11548D0F0F0FDC205C0F30723C0F322
:10642000002403D53446204603B0F0BD9B07F9D5C0
:106430000D48D0F0EFFD0D4B03F63C73D3ED007A21
:10644000F8EEE77A30EE670ADFED097AB0EEC00ABF
:10645000B4EEE70AF1EE10FAE4DD064B3A4602210B
:106460002846C2F085F8DEE740B30020D0A3002024
:106470000000C842B4B51408F8B504460F46C2F08F
:10648000FFFC102105462046C2F06AF858B12046AC
:10649000FFF7EAFD064630B9044B3A461021204684
:1064A000C2F066F835462846F8BD00BFC8B51408E6
:1064B00070B505460E46C2F065FA044678B18021F3
:1064C0002846C2F04DF850B1074B93F8213A43B13A
:1064D000064B324680212846C2F04AF80024204666
:1064E00070BD0446FBE700BFD0930020DCB5140864
:1064F00038B50D4D0446D5F8980FCEF023FF01288E
:1065000010D0D5F8980FCEF01DFF022804D02046F9
:10651000BDE83840C1F0AABF044812F00FF80128C6
:10652000F5D138BD0020FCE7D0A300207CC70020B7
:10653000F0B5134C04F5A04385B0D3F8BC2F0092FE
:10654000D3F8C02F0192D3F8C42F0292D3F8C83FDA
:1065500003936A4606460F46C3F0AEFB394605462E
:106560003046C2F05FF804F5C044284094F8303457
:1065700060F3C303C3F3C00084F8303405B0F0BD4A
:10658000D03300202DE9F84306462748DFF8A890CD
:10659000DFF8A8800F469FF061FE0446D9F83C045E
:1065A00003681B699847054630B914F0060F03D1FC
:1065B000D9F87034022B09D139463046C2F004F9BB
:1065C000054618B9002488F807400AE039463046E5
:1065D000FFF756FD04460028F4D02DB9012388F8B2
:1065E00007302046BDE8F88308213046C1F0B8FFE7
:1065F0000028F3D00D482CF0C1FA0028EED00C4B47
:1066000093F86426B02101FB023203F58043B2F80F
:106610006E24B3F97E329A42E0DD064B3A460821F9
:106620003046C1F0A5FFCDE79C710020283700203F
:10663000D0330020F0B51408D0930020EDCE002018
:1066400070B588B005460E46C2F046FA044698B3C7
:1066500020212846C1F084FF70B31B4B93F8D4204F
:1066600052B393F8B0309B0726D5184807AA06A95D
:106670009BF008FA00B3DDED077A9FED157AF4EE92
:10668000C77AF1EE10FA17D80DA3D3E9002317EE5D
:10669000900ACDE90423FDF775FFDDED067A0D4B79
:1066A000FDEEE77ACDE90201CDED007A32462021F8
:1066B0002846C1F05DFF0024204608B070BD00BF31
:1066C000000000403333E33FD0B300209C7700202C
:1066D0009A99193F00B614082DE9F3410E46054674
:1066E0001AF02AFA804619F04FF8044640B95E4A7B
:1066F00001212846C2F0C8F9204602B0BDE8F08169
:10670000404619F015FF48B923F0D6F990F8461322
:1067100023F0A6F8044608B9544AE9E7544FD7F8DD
:106720003C04036831469B699847044658B9D7F83A
:106730003C0403681B6C98474E4A034601212846D7
:10674000C2F0A2F9D8E7AB68002BD5D010212846BB
:10675000C1F006FF20B3D8ED937A98ED920A20EEAF
:10676000270A3DF10BFBDFED447AA7F5005320EE3D
:10677000270AB3F95032DFED417A20EE270A07EEFF
:10678000903AF8EEE77AB4EEE70AF1EE10FA07DD98
:106790003B4B012210212846C1F0EAFE0024ABE762
:1067A00020212846C1F0DCFE38B197F85534DB06CD
:1067B00003D5344B01222021EDE740212846C1F0CA
:1067C000CFFE38B3012E1ED0232E1CD0042E1AD09B
:1067D0002D4CD4F8C43FB3F9083000EE103AA4F5BC
:1067E000A040B8EEC00A00F0D7FBB5EEC00AF1EE4B
:1067F00010FA1DDD254B00930122254B4021284630
:10680000C1F0B6FECAE7D7F83C040368DB6B9847D3
:106810000028DDD01F4B1B68D86A0368DB699847E6
:106820000128014619D11C4A2846C2F02DF9B5E7C6
:10683000D7F83C0403685B69984730B1D4F8C43F8B
:10684000B3F90830002BE5DDD4E7D7F83C04036842
:106850001B6898470B28DDD1F0E73146284602B087
:10686000BDE8F041C2F004BE2CB614083DB61408D1
:10687000D093002051B61408E02E65420000C842B3
:1068800065B6140854B41408D083002057B3140814
:106890006DB6140810CC002079B6140870B5054602
:1068A0000E46FFF7EDFB084B0446D87131462846EB
:1068B000FFF7CCFC31460028284608BF0024C3F06F
:1068C000A9F9204070BD00BFEDCE00202DE9F041B8
:1068D000524F3B78002B40F09F80514CD4F86054CD
:1068E00095F8D55001263E701DB13B702846BDE895
:1068F000F081C3F041FB054630B94A4A387013783D
:1069000043F001031370F1E774F0DCFD314673F0DE
:10691000ADFDA4F5C04007F0C1FF434B1E710B262F
:1069200061F07EFE013E61F099FD16F0FF06F7D1A1
:106930003E4801F079FA1AF0FFF8D0F80022C4F8C6
:10694000882490F87C32DA0754D419F0A3FB74F051
:10695000B9FD3C2174F048FB04F5896300221A60FC
:1069600000213248324E01F0F1FA304816F02EF88C
:1069700001463048D5F03AFD2F4B1B68D86A0368B2
:1069800001211B68984796F81031D4F860046FF322
:10699000410386F8103103689B6A98470121D4F8B7
:1069A0006004D1F091FE74F08DFD8046D4F83C0473
:1069B00003681B689847A6F58043014693F8642056
:1069C000404673F02FFFA6F5004007F059FF70F026
:1069D0006DF86FF0A9FB00233B70DCF093F8B4F87E
:1069E000323446F85C0C23F4087343F02003A4F817
:1069F00032347BE79B07B3D431460C4805F0B0FF37
:106A00000E48D0F007FBDFED0E7A20EE270A04F5E2
:106A1000896383ED000AA3E7002567E7CD330020F3
:106A2000D09300200CCF0020EDCE0020D0330020EA
:106A3000D0B300208C8F002010CC002040B3002069
:106A40000AD7233C2DE9F043374DD5F8603493F84D
:106A5000D53087B0002B64D062B1012901D0232941
:106A600008D195F93034002B04DB0024204607B010
:106A7000BDE8F083C3F038FB04460028F5D01AF0D7
:106A80005BF8074623F018F88046384618F08AFC71
:106A9000D8B198F92830022B17D100264FF0000901
:106AA000F1B203AA38460191CDF80C90CDF81090C0
:106AB000CDF8149019F0F0F8019918B103AA4046E6
:106AC00022F092FC0136032EEAD11848012108F089
:106AD00053F91648012108F083F80021D5F8600425
:106AE000D1F0F2FD124844F0F9FC74F0EBFC002107
:106AF00073F0BCFC0F4B1B68D86A036800211B684D
:106B0000984795F83234D5F83C140B486FF3451389
:106B100085F832340B1A594259413C30D9F02CFADD
:106B2000A4E70124A2E700BFD0930020D0330020C7
:106B30004CC1002010CC002000C3002010B5064C32
:106B4000D4F83C0403685B6A984718B1D4F8603401
:106B500093F8D50010BD00BFD093002030B52DEDC7
:106B6000028B89B00C46B0EE408AFFF7E7FF05467E
:106B7000002838D0B4EE488AF1EE10FA7CBFDFED81
:106B80001C8ADFED1C7A226863689FED1A0A68BFD1
:106B9000DFED198A029278BF68EE288A02A878BFD2
:106BA00068EEA78AD4ED027A0393F1EE677ACDED11
:106BB000047A41F06BFDB4EE488A00220123F1EE25
:106BC00010FACDE900238DED050ACDED060A9FED03
:106BD0000A0A0A488DED071AF0EE680A68BF1346E4
:106BE00005A90FF0C7F9284609B0BDEC028B30BDEE
:106BF000E02E65420000C842000000001CC60020D4
:106C000007B50191FFF79AFF30B10199044803B02D
:106C10005DF804EB00F094BB03B05DF804FB00BF2B
:106C2000D033002001489FF0A5BC00BF9C7100201C
:106C300008B500F5C04090F83034C3F340128A42E2
:106C40000BD061F3451380F8303431B174F03AFC65
:106C5000BDE808400F2174F0C7B908BD70B500F554
:106C6000C0460546D6F870348B420C4612D0012936
:106C700011D0022916D059B974F024FC1B2174F0EC
:106C8000B3F90D4A05F5C3400621483078F066F89F
:106C9000C6F8704470BD74F015FC1A2174F0A4F9A4
:106CA000064AEFE7012101F051F974F00BFC1D21B8
:106CB00074F09AF9024AE5E7E8B61408FDB614083C
:106CC000F8B6140810B500F5C0420C4692F85534D9
:106CD00003F00101A14209D064F3000382F85534A6
:106CE000DB0704D407F0A2F9024B9C7210BD07F039
:106CF00089FBF9E7EDCE002000F5C04090F855344F
:106D000061F3410380F85534014B1973704700BF9C
:106D1000EDCE002010B5044681F05AFF202183F00B
:106D2000BFF904F5C043003893F8322418BF01209E
:106D300060F3820283F8322410BD000010B50446CF
:106D40006FF0B4FE04F5C042436FD2F8602404F53E
:106D5000E044D360D4F88C2F9366D4F8942FC2F813
:106D60000833D4F88C0F03685B6D9847D4F88C0F08
:106D70000368BDE810409B6D18470000F8B52DED85
:106D8000028B00F5C0450446D5F8603493F8D53041
:106D9000002B7FD095F93034002B7BDB00F50043CE
:106DA00093F8A03C002B75D1D5F83C0403685B69CF
:106DB000984700286ED1394BD3F83C0403681B6810
:106DC00098470B2866D004F5E0479FED357AD7F851
:106DD000943FD3EDE47AF0EEE77AF4EEC77AF1EE81
:106DE00010FA57D5D5F86004443077F023F90346FC
:106DF000DFED2C0A93ED000A9F20B7EE001A3CF05D
:106E000041F8B5EEC00AF1EE10FA43DD04F5FE409C
:106E10007030D0F00BF9DFED247AB0EEC00AB4EE9A
:106E2000E70AF1EE10FA35D504F50056D7F88C0FC5
:106E3000D6F8283607EE903A0368D3F89830B8EEC3
:106E4000E78A984738EE400ADFED187AB0EEC00ABC
:106E5000B4EEE70AF1EE10FA1CD5D6F82C3640F263
:106E6000E63203F2F313934214D8D5F860049FED91
:106E7000100AD3F08FF8BDEC028BD5F860349FED8B
:106E80000C0AD3ED0C0A04F5E3501030BDE8F840CD
:106E9000B1F0AABEBDEC028BF8BD00BFD0930020BC
:106EA0000000003400000000000070420000FA43BF
:106EB0000AD7233C08B500F5C040D0F86004036849
:106EC0001B699847F6EE007A20EE270AB5EEC00A55
:106ED000F1EE10FA48BF9FED010A08BD0000000066
:106EE00038B52DED028B00F5E0450446D5F88C3F12
:106EF000DFED110A93ED370A04F5C0447120B7EEB7
:106F0000001A3BF0BFFFD4F86004D5F8945F036823
:106F10001B69B0EE408A984738EE400ABDEC028B00
:106F2000DFED067A05F50575284620EE270ABDE84F
:106F30003840AEF009B800BF0000000000007A44FD
:106F400000F51050D0EDA05AD2ED007AD0EDA36A32
:106F500091ED006A26EEE77A67EEA57AA6EE257A2D
:106F6000E6EE267A81ED007AC2ED007A70470000E5
:106F700000F5A043B3F9883C43B900F58040B0F96F
:106F80008A020028B8BF404280B2704783EAE370AB
:106F9000A0EBE370F8E7000070B52DED028B00F573
:106FA000C04382B093F8551411F00106044605D091
:106FB0009FED2E0A02B0BDEC028B70BD8DED010A73
:106FC00081F006FE037F002BF2D0DFED298ADFED92
:106FD000270A9DED010AB0EE681A4E203BF052FFE1
:106FE00004F580454FF4C8723146B5F99202B0EE0F
:106FF000408A3BF085FFA5F89202204615F01EFA64
:10700000B5F9923207EE900AB8EEE77A07EE903AB9
:10701000F8EEE77A77EE676AB4EEE68AF1EE10FAF8
:107020000DD52046FFF7A4FF07EE900A38EE668ADA
:10703000B8EEE70A20EE088A88EE260ABAE777EE6D
:10704000877AB4EEE78AF1EE10FAB1DDB5F98A324B
:1070500000EE103A38EE678AB8EEC00A78EEE77AAA
:1070600020EE088A88EE270AA4E700BF000000008F
:1070700000007A447047000070470000002070470D
:1070800000207047002070470020704700207047A4
:107090000020704700207047002070470020704794
:1070A0007047000000F58540203070470048704769
:1070B0008CEF140800F5C040D0F83C0403681B684E
:1070C00018470000034808603921117008221A602F
:1070D000704700BF4CBD140800F5E0409FED0A7AF0
:1070E000D0F8A03FD3ED0E7AF4EEC77AF1EE10FAA5
:1070F000B8BFD3ED047A9FED057A67EE877A012059
:10710000C1ED007A704700BF000000340AD7233C6D
:1071100000F5C040DFED047AD0F83C04036820EEAF
:10712000270A5B6E184700BF0000C84200F5004305
:1071300093F8F93E002B14BF1B2003200B1A584272
:107140005841704700F5C04090F85504C0F38000E6
:107150007047000000F5C040D0F83C0403685B6D48
:107160001847000000F5C040D0F83C040368DB6C11
:107170001847000000F5C040D0F83C0403689B6C41
:107180001847000000F5C04300F50D40D3F83C342B
:1071900040301B1A584258417047000010B500F5A6
:1071A000C0400C46D0F83C040368DB6D984707EEFE
:1071B000900A9FED057AF8EE677A012067EE877AEC
:1071C000C4ED007A10BD00BF0AD7233C10B500F50E
:1071D000C0400C46D0F83C0403689B6D984707EE0E
:1071E000900A9FED057AF8EEE77A012067EE877A3C
:1071F000C4ED007A10BD00BF0AD7233C10B500F5DE
:10720000C0400C46D0F83C0403681B6E9847DFED85
:10721000047A20EE270A012084ED000A10BD00BF89
:107220000AD7233C90F022BFD5F0C8BB16F05ABB5A
:1072300004F0EABF96F0C0BF84F056B96FF080BB8F
:1072400038F026BD73F094BA1EF066BA84F0A4BE7E
:1072500081F0ECB87EF0F8BD14F056BD15F00ABA16
:1072600007F0C6BF16F0D2BA06F036BF06F07EBCF5
:1072700006F0A4BB14F0E0BE92F0FABD9EF0F6BD9D
:1072800012F010B8FFF77ABD14F080BEC0F052B90A
:107290009AF016BC15F024B903F0CABF14F0FEBD75
:1072A00014F07ABD81F0D2BB64F0BEB82DF0D0B935
:1072B00007F060BB03F0ACBA84F07EBE15F052B9A3
:1072C00007F04EBF05F038BB08F0BCB806F008BCAC
:1072D00007F000BC14F0A4BCFFF730BD39F0B2BA1F
:1072E00008B500F5E040D0F8A00FCDF023FC012058
:1072F00008BD000010B400F50D4400F5C040403456
:10730000D0F83C04A04203D15DF8044B09F096BFCD
:1073100000205DF8044B704700F50D4300F5C040B8
:107320004033D0F83C04984201D109F0A5BF704722
:1073300007F0EAB80CF006B80BF040BE0BF0D4BD75
:107340001FB500F5C0430446D3F83C04039103681D
:107350005B6A984760B1DFED070A0399002304F5E3
:1073600012400093B0EE600A1A464C300EF0FCFE5C
:1073700004B010BD0000000010B52DED028B00F52B
:10738000C0430446D3F83C0403685B6AB0EE408A0D
:10739000984720B90024BDEC028B204610BD9FED1C
:1073A000080A04F5124028EE000A4C300EF0F8F8F6
:1073B00004460028EED003480121FFF739FCEAE734
:1073C0000000C842D03300207FB5044668460D4611
:1073D000164620F041FF04F5C0436946D3F83C044B
:1073E00003685B6D98476946284621F05FF810B93D
:1073F000002004B070BD6946284621F063F80028DB
:10740000F6D0284620F058FF0546304620F054FFBD
:107410008542EDD1236831461B6A20469847E8E74C
:1074200030B52DED028B0C4600F5C0410546D1F874
:107430003C0489B001680392496A0293B0EE408A25
:10744000F0EE608A884728B39FED140A94ED006A35
:10745000D4ED016A94ED027A9DF83C10019126EE7C
:10746000006A66EE806A27EE407A9DF83810009137
:1074700005F5124068EE800A029B039A8DED056ABD
:1074800028EE000A05A94C30CDED066A8DED077A8D
:107490000EF084FD09B0BDEC028B30BD0000C84287
:1074A00070B500F5C0430646D3F83C0403688EB0BF
:1074B0005B6A0D4614469847D8B3DFED1F7A95ED09
:1074C000006AD5ED016A95ED027ADFED1C0A26EE21
:1074D000276A66EEA76A27EE677A8DED056ACDED1D
:1074E000066A94ED006AD4ED016A8DED077A94ED99
:1074F000027ACDED0B0A002326EE276A66EEA76A14
:1075000006F5124067EE677ACDE901330093B0EEDD
:10751000600A0BAB08AA05A94C308DED086ACDEDC9
:10752000096ACDED0A7ACDED0C0ACDED0D0A0EF00B
:1075300021FF0EB070BD00BF0000C8420000000077
:10754000F0B52DED028B1C4600F5C0430746D3F87D
:107550003C0403688FB05B6A0E461546B0EE408A65
:10756000F0EE608A984700284CD09FED280A96EDEF
:10757000006AD6ED016A96ED027A9DF860300293BA
:1075800026EE006A66EE806A27EE407A8DED056A87
:10759000CDED066A95ED006AD5ED016A8DED077AAD
:1075A00095ED027A9DF85C30019326EE006A66EE56
:1075B000806A27EE407A8DED086ACDED096A94ED78
:1075C000006AD4ED016A8DED0A7A94ED027A9DF895
:1075D0005830009326EE006A66EE806A27EE407A05
:1075E00007F5124068EE800A0BAB28EE000A08AAE5
:1075F00005A94C308DED0B6ACDED0C6A8DED0D7A41
:107600000EF0B8FE0FB0BDEC028BF0BD0000C8421A
:1076100070B500F5C0430646D3F83C04036886B055
:107620005B6A0C469847054610B39FED136AD4ED8C
:10763000006A94ED017AD4ED027ADFED100A00239E
:10764000012266EE866A27EE067A67EEC67A06F5AE
:107650001240CDE90032B0EE600A1A4603A94C3060
:10766000CDED036A8DED047ACDED057A0EF082FC46
:10767000284606B070BD00BF0000C84200000000F0
:10768000F0B52DED028B144600F5C0420746D2F846
:107690003C048DB002680593526A0D46B0EE408AF4
:1076A000F0EE608A90470646C8B39FED1F0A95ED3D
:1076B000006AD5ED016A95ED027A059B26EE006A17
:1076C00066EE806A27EE407A01228DED066ACDEDE6
:1076D000076A94ED006AD4ED016A8DED087A94EDA5
:1076E000027A02929DF85420019226EE006A66EE1C
:1076F000806A27EE407A9DF85020009207F51240EC
:1077000068EE800A09AA28EE000A06A94C308DED21
:10771000096ACDED0A6A8DED0B7A0EF0C1FB304699
:107720000DB0BDEC028BF0BD0000C84270B52DED70
:10773000048B00F5C0430646D3F83C04036888B0C8
:107740005B6AF0EE408AB0EE609AF0EE419AB0EEDD
:10775000618A9847054600B39FED120A00244FF056
:107760007E5329EE801A69EE000A04A828EE800AEA
:1077700004930794069405943FF01EFE9FED0A0AB9
:10778000019406F5124028EE000A002301AA04A97C
:107790004C30029403940EF017FA284608B0BDEC62
:1077A000048B70BD35FA8E3C0000C84230B52DED1B
:1077B000048B00F5C0430546D3F83C04036889B048
:1077C0005B6AF0EE409AB0EE609AF0EE418AB0EE5D
:1077D000618A98470446F0B14FF07E53049304A8A1
:1077E000002307930693059340F04AF89FED0C0A97
:1077F000CDED019A01A88DED029ACDED038A40F0FE
:1078000099FF05F512400123B0EE480A01AA04A928
:107810004C300EF0D9F9204609B0BDEC048B30BDD8
:1078200035FA8E3C0A4A92F93024002A0B4605DAD2
:1078300000228A604A600A600120704700F5E0403B
:10784000D0F88C2F783207CA83E80700F4E700BF2E
:10785000D09300206E4B70B5044640F8043B90F086
:1078600025FD04F110001DF0F1FA04F1B000C2F0A2
:107870008FFC04F528706EF0F1FD04F556702BF0C6
:1078800061F804F5F4601BF059FA04F63C1021F09D
:1078900021FA04F6884037F053FF04F5B65008305B
:1078A00090F0B2FA04F5BC50183068F08FFC04F583
:1078B000D250083072F02AFD04F5DA501C309DF0E9
:1078C000C5FD04F5DB50183084F0ECF904F5DD500B
:1078D00014301FF00DFE04F5E3501030B2F008F83C
:1078E00004F50C50BEF052FA04F50C501C306FF049
:1078F00077F904F50E500C3091F0B8FE04F5005302
:107900000025444A83F8D05304F50F5004F50F5373
:1079100010332030136060F085FB04F510502946C9
:10792000303017F005FA04F52C50283096F054FC4E
:1079300004F52D501830AFF0BDF904F55550243042
:10794000B7F06AF804F559503C30B5F05FFE04F525
:107950005A502430B9F082FA04F55C503030BDF052
:107960006FFB04F55E501430BDF0A4FF04F55F50CA
:107970002C30ADF027FD04F56250143016F086F976
:1079800004F56850AFF050FF04F569501830BFF0AF
:10799000A9FB04F5765020492C3066F0DBFF04F596
:1079A00077500430C4F09EFA04F577500C309EF006
:1079B000F9FA04F57A500830BFF068FA04F57B5004
:1079C0002030DBF0BFF804F5804304F5834683F8EC
:1079D00064501D467435743628460C3576F026FB07
:1079E000AE42F9D104F58440BFF0D0FA0B4D04F556
:1079F0008440243075F02CFE2B6813B10848DBF06E
:107A00004FF82046074966F0A5FF2C60204670BD60
:107A10009C001608FCDA00201417170800D000207C
:107A20000CB7140804FF150810B514F07BFC81F0A6
:107A3000CFF80368BDE810405B681847FFF7F4BF54
:107A400010B5044607F0E4F8204614F0E9FF20469C
:107A500004F0BCFD2046BDE8104004F023BF000048
:107A6000FFF7EEBF70B500F5C9450C350446284652
:107A70001CF012FE22F020F890F9253093B390F814
:107A800044337BB304F5C04304F63C16D3F86004DA
:107A9000443076F0CFFA0346DFED130A93ED000A87
:107AA0009F20B7EE001A3BF0EDF994F97439012BE1
:107AB000284608BF86ED0F0A00211CF047FBDFEDCA
:107AC0000B7A04F6983494ED287A20EE270ADFED3D
:107AD000087AA7EE270A304684ED280ABDE87040F0
:107AE00021F0E0BE70BD00BF00000000CDCCCC3D59
:107AF0006666663FFFF7B6BF10B50121044614F075
:107B0000CBFF60B1114BD3F83C0403689B6A9847E4
:107B100028B9204602F082FD204602F08FFD4FF486
:107B20000011204614F0B8FF18B13AF015F837F0FC
:107B3000ABFC4FF48021204614F0AEFF28B13AF0A0
:107B40000BF8BDE8104037F0A3BB10BDD093002068
:107B5000FFF7D2BF7FB500F5E0460446D6F88C0F9C
:107B60009FED650A6C3040F091FD04F5105001A9BD
:107B700030308DED010ACDED020A8DED031A16F0BD
:107B80006BFF0221204614F087FF70B101212046CF
:107B900014F082FF48B9594BD3F83C0403689B6A40
:107BA000984710B9204602F039FD0121204614F013
:107BB00073FF48B9514BD3F83C0403689B6A98475C
:107BC00010B9204602F03AFD0121204614F064FF6E
:107BD00010B9204602F08CFD4FF40031204614F01D
:107BE0005BFF30B104F5C043D3F8600403685B6CFD
:107BF00098474021204614F04FFF68B104F5D25554
:107C00000835284671F030FE04F5805393F9783B2F
:107C100013B1284671F0ECFF4FF48061204614F058
:107C20003BFF20B104F5D250083071F0B7FE20219F
:107C3000204614F031FF58B104F5C045D5F83C0496
:107C400003681B699847C8B3D6F8940FCAF094FA32
:107C50008021204614F020FF00283CD039F07CFF22
:107C600037F03AFB1021204614F016FF68B1D6F821
:107C70008C0FC6F00BFE04F587404C309AF056F896
:107C800004F586401030BFF0C7FC4FF6FF71204668
:107C900014F002FF20B104F5B8406C30D4F09CFE23
:107CA0004FF40041204614F0F7FE18B304F50040ED
:107CB0002C3004B0BDE8704084F000BB20460FF0CB
:107CC00085F90028C0D1D5F83C0403685B69984762
:107CD0000028B9D0BCE74FF48021204614F0DCFE28
:107CE0000028BBD14FF40021204614F0D5FE002817
:107CF000B4D1B7E704B070BDE02E6542D093002048
:107D0000FFF728BF10B50121044614F0C5FE10B1DD
:107D1000204602F0EDFC8021204614F0BDFE48B163
:107D20004FF48021204614F0B7FE18B939F014FF43
:107D300037F0AEFA4FF40011204614F0ADFE30B12A
:107D400004F5E3501030BDE81040B0F0E5BF10BDC1
:107D5000FFF7D8BF10B5044606F0A8FC204606F091
:107D6000EFFA204606F0E8FC204615F0DFFD20463D
:107D7000BDE8104004F026BAFFF7ECBF70B54FF62F
:107D8000FF71044614F088FE04F5C04528B1D5F80B
:107D900030240721204602F0DDFCD5F8603493F84A
:107DA000D5308BB92046FEF7B5FFD5F8600404F551
:107DB0008043026893F8741D166A93F8A622B047B0
:107DC000D5F86004D2F0B2F883F084F882F090FC29
:107DD000204615F09DFD95F8303404F50042DB4354
:107DE000C3F3C01304F5E04482F8BD3B0C4AD4F859
:107DF0008C5F53712B681E6F6EF058FE6EF0C0FAE8
:107E00002846B047D4F8944F6EF050FE04F5057440
:107E10006EF0B6FA2046BDE87040ACF067BE00BF19
:107E2000EDCE0020FFF7AABF2DE9F04100F5005686
:107E300000F5C04506F5866305F27448D3F8502274
:107E4000C8F8002005F58F67D3F85C323B60044624
:107E5000D6F8300600F58C4050303AF0E7FF04F5D4
:107E6000C943C5F87C04D8F800201A6005F284459F
:107E70003B682B604FF6FF71204614F00DFE38B1C1
:107E8000D6F8302620460921BDE8F04102F038BC82
:107E9000BDE8F08130B500F5C043D3F87044002C44
:107EA00053D093F83124D1074FD56FF3000283F8F4
:107EB000312400F5A042012CD2F8BC1FD2F8C05FDB
:107EC000B1F9084007EE104AB5F9084006EE904AAD
:107ED00012BF03F2844303F2744403F58F63D3EDBE
:107EE000005A07BFD4ED007AF8EEE66AF8EEE66ACB
:107EF00000F5C94418BFD4ED007AB8EEC77A25EE74
:107F0000E66A00F51050A7EE276A67EEA67AD0ED74
:107F1000A06AE7EE257A90EDA37A27EE877AA6EE9F
:107F2000267ABDEEC77A17EE103A0B8190EDA07A53
:107F3000D2F8C03F67EE877A90EDA37AE6EE477AF3
:107F4000FDEEE77A17EE902A1A8130BD38B5044667
:107F50002DED028B00F5C04571B1204614F038F8C4
:107F6000D5F87C341B1A03F2F31340F2E632934245
:107F70000CD8BDEC028B38BDD5F87034022BF8D18B
:107F800014F008F8B0F57A7FE7D2F2E700F58C43F9
:107F9000C5F87C045033642093FBF0F308EE103AEC
:107FA000DFED0B7AB8EEC88A04F5C94428EE278ABB
:107FB00005F28445B0EE480A3BF1CCFC84ED000AA2
:107FC000B0EE480A3BF176FE85ED000AD1E700BF2E
:107FD00035FA8E3C00F510500121303018F012BDFA
:107FE000FFF7F8BF10B5044614F02EFA1021204612
:107FF00014F052FD98B1204602F05AFA4FF40011E5
:10800000204614F049FD50B939F0A6FD37F03CFA8E
:1080100004F5E3501030BDE81040B0F07DBE10BD57
:10802000FFF7E0BFF8B50446254607F01FF9224BDD
:1080300045F83C3B214BA465C4E91734204BC4E907
:108040001934204BE36604F1800020F005F904F1B7
:108050009C0020F001F904F1B80020F0FDF84FF683
:10806000FF76194BC4F8CC30A4F8D06004F1D400EA
:1080700020F0F2F84FF0FF37144B1549C4F8307177
:1080800028461D6066F066FCA4F87870A4F8946039
:1080900004F5A27020F0E0F804F5B07020F0DCF8F0
:1080A00004F5BE7020F0D8F8002384F89031C4F8AD
:1080B000B4312046F8BD00BFA01F15083573000875
:1080C000397300083D7300080000FFFFBCCE00209C
:1080D0004CB6150810B5044607F0C8F80A4B2360E3
:1080E0000123A38704F1400020F0B6F804F150000A
:1080F00020F0B2F804F1600020F0AEF804F1700056
:1081000020F0AAF8204610BD082B15082DE9F043F1
:1081100004468BB0FFF79EFBB54B236004F585400A
:10812000483002F0E5FC04F5A04204F58543143321
:10813000C2F8D03F04F5BF45062382F8D43F4FF084
:108140007C5707A905F16000079776F085F805F1DF
:10815000780004F5C045D9F013FE04F5FE4600236F
:1081600070362B74192306A92B77AE6105F1280010
:10817000069776F071F805F14000D9F001FE4FF056
:1081800001081823284604F5C14785F86430603794
:1081900085F858802E66783082F0A0FF3846C0F00F
:1081A0006FF908AE934BC5F8E0303146381D8DF8B5
:1081B000208067F0A5FB04F5C240403063F0D8F89A
:1081C00004F5C340BEF0A4FF8B4B8C4FC5F8803143
:1081D00004F5C34031461830089776F03DF804F5B1
:1081E000C34031462430089776F036F804F5C34092
:1081F0003146303004F5C348089708F1480876F056
:108200002BF87F4BC5F8C83108F10C00D9F0B8FD48
:1082100004F5C34704F5C549783709F1180938460C
:1082200014377BF049FAB945F9D10723C5F8C833AB
:108230000023A5F8CC334FF4CB7020F0E9FCC5F84F
:10824000C40304F5C7405030D9F09AFD04F5C84086
:108250001430D9F095FD6B4B1A680AB9C3F8008049
:1082600004F51448684BC5F8C83108F1380804F51E
:10827000C840C5F83C844030C1F070FF05F2744539
:1082800004F5C9434FF07E572F601F605F4B099381
:108290005F4B0894009304F5C94096E80C004FF436
:1082A00000710C301BF0E6FC04F5D4402430A4F03F
:1082B0000FFD04F5FE4005A94030059775F0F6FF67
:1082C00004F5FE4005A95430059775F0C5FF04F587
:1082D000FE4060301FF0C0FF04F5E04303F5776215
:1082E000002616605660966003F67C7204F5FF4027
:1082F00016605660966004F510523032C3F8882F2D
:10830000002283F8A92F4FF400412C301CF0E6FE28
:1083100004F500402C3083F029FE04F50040B03015
:10832000A0F070FA04F5004004F50045EC3067F069
:108330001DFC384BC5F8EC3004F501409DF038FDCC
:10834000354B364904F501401C3004F501491860ED
:1083500009F13C0966F0FEFAFF2385F84C3185F8F7
:1083600054312F49484666F0F5FA2E4B1F6817B175
:108370002D48DAF095FB04F501405C30C3F800901D
:108380006FF058FD04F50A400430CBF0BDFB04F556
:108390000A40F830CBF074FA04F50B41084603911B
:1083A000ABF01CFD04F50C4003993030D2F0B4FD65
:1083B0001E4BC5F8303C062385F8843C1C4BDFF887
:1083C00084C0C3F800C004F50C423B469032142729
:1083D00098B207FB00C10133097C0029F8D1154B85
:1083E0001880154B1880154B1F686FB31448C0E7F1
:1083F000D0C1140890B61408D4B614080000A040E8
:108400003825160874D40020B4C21408317300084B
:10841000C0C11408E4B6140808DB00201C5016087C
:1084200054151708C8DB002020B71408B416150827
:10843000BCCF0020B8CF002090CF002064CF002018
:1084400041B71408700C150804F50C401A6005A912
:108450006E4B0593A43075F0FFFE04F50C40C4305C
:1084600006F004FF6A4BC5F8C43C04F50D40043027
:1084700006F0FCFE04F50F49664BC5F8043D04F513
:108480000D4009F130094030FFF7CCFD484606F0B9
:10849000EDFE614BC5F8303F09F13C00D6F0F4F930
:1084A0005E4BC5F86C3F04F5104004F51045F03004
:1084B00006F0DCFE5A4BC5F8F03004F511403430BC
:1084C00006F0D4FE574BC5F8343104F5114085F859
:1084D0007071743006F0CAFE534BC5F8743104F560
:1084E0001140B03006F0C2FE504BC5F8B03104F573
:1084F0001240C5F8EC61C5F8F061C5F8F4610430CC
:1085000006F0B4FE4A4BC5F8407204F51240C5F8B7
:1085100004324C3006F0AAFE464BC5F84C3204F546
:108520001240C5F88872903006F0A0FE424BC5F8A4
:10853000903204F51240D83006F098FE3F4BC5F853
:10854000D83204F51340183006F090FE3C4BC5F8C5
:10855000183304F51340C5F89063C5F89463AC3044
:10856000FFF7B8FD404606F081FE364BC5F83834BB
:1085700004F51440743010F065FF04F515403030F8
:1085800006F074FE304BC5F86C7504F51540C5F85F
:108590003035743006F06AFE2C4BC5F8743504F59E
:1085A0001540A5F8B075C43006F060FE284BC5F83C
:1085B000007604F51640C5F8C4350830FFF78AFD8B
:1085C000244BC5F80836012385F8913605F5D363A9
:1085D00004F516401E605E609E60A4300CF08AF8C0
:1085E00004F51740783012F0C1FA04F51740F03066
:1085F00006F03CFE184BC5F8F03705F5036520463C
:108600002E606E600BB0BDE8F08300BFCDCC4C3D5A
:10861000901B1508381C150848201508DC20150883
:1086200040221508E422150888231508242415087B
:10863000682615080C2715084C281508E828150881
:108640008C2915086C2C15089C21150890301508EC
:10865000B8271508C42B15085831150838B5054B2F
:108660001C6823680A461D68034B01462046A8473C
:10867000002038BD10CC0020D033002038B503795D
:1086800004463BB905682DB1284635F073FF2846EE
:1086900020F0C0FA204638BD3A4B70B5036004465E
:1086A00000F575500C301FF05FFD04F5405393F852
:1086B000882742B9D3F884572DB1284635F05AFFA0
:1086C000284620F0A7FA04F50C50BDF073FB04F522
:1086D000F4500430FFF7D2FF04F5F3501C30FFF7DD
:1086E000CDFF04F5F3501430FFF7C8FF04F5DB505D
:1086F000183083F0EFFA04F5BA5504F5B7560C3587
:108700000C36B54204D0183D284635F07DFBF8E71D
:108710001D4BC4F8883C04F58D5504F58B56103577
:108720000836B54204D0083D2846FFF7A7FFF8E712
:1087300004F64C6075F05AF904F5626075F056F96C
:1087400004F6F45075F052F904F6485075F04EF9FD
:1087500004F61C5075F04AF904F54F6075F046F9BF
:108760000A4BC4F8FC3094F8103243B9D4F80C52D8
:108770002DB1284635F0FEFE284620F04BFA204663
:1087800070BD00BF9C0016081CA51508747517085D
:1087900038B5104B036000F50043044693F8242CD1
:1087A00042B9D3F8205C2DB1284635F0E3FE2846C7
:1087B00020F030FA04F5C043074AD3F8C403C3F8E5
:1087C000C82108B120F02AFA2046FFF765FF2046AD
:1087D00038BD00BFD0C114083825160810B5D9F02F
:1087E00095FD064C064B18602046FFF78FFC20468F
:1087F000044A0549BDE810403AF120BFD0330020BB
:1088000010CC0020003A0120918700080120704719
:1088100090F8D0308B4286BF00EB8100D0F8D400B6
:108820000020704790F8D0308B4286BF00EB81006B
:10883000D0F8D40000207047FA207047014B93F81D
:1088400056027047D0730020034BD3F87004431EC8
:1088500058425841704700BFD0930020034BD3F8D3
:108860007004831E58425841704700BFD0930020C7
:10887000034BD3F8600408B1D0F02EB8014870471C
:10888000D0930020A0C2140838B5436A4E4D43F47B
:10889000E0524262826A42F4E0528262C26A42F468
:1088A000E052C262D5F8942F0446E2B143F4F84393
:1088B0004362D5F8940FC8F0B7FE38B1A36A43F409
:1088C0008043A362E36A43F48043E362D5F8940FE4
:1088D000C8F0D8FF38B1A36A43F40053A362E36A37
:1088E00043F40053E362394899F028F918B1636AF8
:1088F00043F080636362354899F0CAF818B1A36AFF
:1089000043F08063A362314899F04AF918B9E36AE9
:1089100043F08063E3622E4B1D6845B11921284660
:1089200067F02EFD18B1636A43F480736362294BCC
:1089300093F8D83F6BB1A36A43F48073A36245B147
:108940001921284667F06AFD18B1E36A43F4807381
:10895000E362214B93F9042A8AB1D4E9091242F067
:10896000800241F080016162A26293F9042A32B16F
:1089700093F8EC2A1AB1E26A42F08002E26293F8BC
:10898000003A013B012B0BD8D4E9092343F48003BF
:10899000A362E36A42F4800243F480036262E3620A
:1089A000636A43F080436362A36A43F08043A36237
:1089B0000A4BD3F8603493F8C1301BB9E36A43F033
:1089C0008043E36238BD00BFD0A300209C77002025
:1089D000C8CF0020D0830020D0B30020D093002047
:1089E00013B54FF44470CDE9002120F00BF9044693
:1089F00028B1DDE900217EF0E9FC024B236020462E
:108A000002B010BDFCC4140800207047704700007D
:108A10000320704708207047014B93F858027047B5
:108A2000D0730020034B93F9680D003818BF012064
:108A3000704700BFD0730020014B93F95A02704772
:108A4000D07300207047000008B50C4BD3F8940F8A
:108A500070B910230A4AD2F8602443F0400022B1D2
:108A600092F8D5200AB143F0C00040F0010008BDE3
:108A7000C8F0DAFD0028ECD01823EBE7D0A30020E3
:108A8000D093002038B5C5780B46352D044628BF55
:108A900035253522002118463DF1B8FC2A4604F15F
:108AA0000C01BDE838403DF167BC000000B589B05D
:108AB000002302930393049305930693079318F0FE
:108AC0003BF802A917F004FEA0B118F035F800F544
:108AD0005A7007C805AB83E80700184640F0F6F95E
:108AE000F1EE047A20EE270AFCEEC07ACDED017A91
:108AF0009DF8040009B05DF804FB00001FB5184C98
:108B000094F8EA1904F6940015F0E8FA78B194F8AC
:108B1000EA1904F6940015F063FD40B194F8EA19DF
:108B200004F6940004B0BDE8104015F09DBD00238C
:108B300001930293039317F0FFFF01A917F0C8FDFB
:108B400020B101A840F0C2F904B010BD2BF0BEFD69
:108B500090F80C33B02202FB030090ED410AF3E7DA
:108B6000D063002008B50D4BD3F86004A8B14430A1
:108B700075F060FA034693ED000ADFED090A9F20C5
:108B8000B7EE001A3AF07EF9DFED067A20EE270AFA
:108B9000BDEEC00A10EE103A18B208BDD093002006
:108BA000000000000000C8422DE9F04FDFF8D88037
:108BB000344F8DB00446042508F5405617F8019B44
:108BC000B8F9B03209F1FF3A43FA0AF3D90742D5AE
:108BD000207C77F0F1F88346207C78F007F800F1EC
:108BE00021039B4505D2207C0DB0BDE8F04F76F007
:108BF00005BBBAF1030F2ED8DFE80AF00234393E84
:108C0000D6F88C0F03689B68984700F1A0035A6957
:108C1000D3F800A0D3F804E0D8681969D3F818C0D5
:108C200008925A6A1B6ACDF82520CDF829306222B5
:108C30002123CDE9003206900791207CCDF80CA0CD
:108C4000192303AAC221CDF810E0CDF814C08DF885
:108C5000249077F02FF9013D15F0FF05AED10DB04E
:108C6000BDE8F08FD6F88C0F0368DB68CCE7D6F848
:108C70008C0F03681B69C7E7D6F8943F03F52D7383
:108C8000C5E700BFECC51408D073002007B50190FC
:108C9000D3F0B6FE28B1019903B05DF804EBD3F030
:108CA0006BBE03B05DF804FB13B5044607480191A1
:108CB0000AF070F830B90199204602B0BDE81040C2
:108CC00078F010BA042002B010BD00BF10C100201F
:108CD000014809F0F7BD00BF10C1002070B50B4B73
:108CE000D3F86C3DDB0705460E46144603D508480D
:108CF0001146D2F0C9FC21460648D4F037FD224681
:108D000031462846BDE870407CF036BFD073002065
:108D100000C000206090002010B588B0044679F0B3
:108D200001FD0C4BD3F8600438B90B4A06212046EC
:108D300008B0BDE8104079F0DDBC69461E22CFF0D6
:108D4000D3FD064A6B460621204679F0D3FC08B0D5
:108D500010BD00BFD0930020ECC214088DF017089E
:108D6000034A92F8B83F013382F8B83F78F090BCDC
:108D7000D08300200148CBF0E7B800BFD4BD00206D
:108D800007B5084601911FF0C5FB38B104480199A9
:108D900003F042F8002003B05DF804FB0420FAE77A
:108DA0001CCC0020F7B58B8BCD2B06460C46174606
:108DB0001DD1D1ED067AFCEEE77ACDED017A9DF872
:108DC0000430022B13D10E4D95F8A51005F12C009F
:108DD00083F002F958B195F8A51005F12C0083F045
:108DE00003F920B994ED020A064802F0F5FF3A466D
:108DF0002146304603B0BDE8F04078F0DBBC00BF50
:108E0000D0B300201CCC0020162A10B40C4605D08C
:108E1000542A03D05DF8044B78F080B90323237003
:108E200001205DF8044B704710B5074B93F95C21A6
:108E300040F6CD3440F6CD13002A08BF1C4678F02A
:108E4000DDFB204310BD00BFD0B300201FB517F0DD
:108E500073FE044668461FF0FFF96946204617F086
:108E600085FB0E4B93F8310410F0200014D003F56D
:108E70008053DDED017AD3F8943FF8EEE77A93ED75
:108E80000F7A77EE877A9FED067A67EE877AFDEEA6
:108E9000E77A17EE903A18B204B010BDD0930020D4
:108EA0000AD7233C10B504461FF0B4FE204610BD7F
:108EB00010B50C4C94F93034002B0FDBD4F83C0483
:108EC0000368DB6C984758B9D4F83C0403689B6C82
:108ED000984700280CBF0220032010BD0120FCE7AA
:108EE0000420FAE7D093002008B5134B93F831041F
:108EF00010F020001ED0D3F83C040368DB6D9847C7
:108F000007EE900AB8EE677ADFED0C7A27EE277A43
:108F1000DFED0B7AB4EEE77AF1EE10FA58BFB0EE5F
:108F2000677AF2EE046AC7EE267AFCEEE77A17EE6D
:108F3000903A98B208BD00BFD09300200AD7233CD6
:108F400000FF7F4710B44C69012C05D101465DF844
:108F5000044B034803F04EBD5DF8044B78F0B2BB00
:108F6000D03300202DE9F341B1F90430002B06463F
:108F70000C46154635DB4FF00008CDE900281A4FA6
:108F8000B1F902209FED190AD7F8BC1F4FF47A738C
:108F90007DF044F90123CDE900539FED140AB4F9A3
:108FA0000020D7F8C01F4FF47A7330467DF036F9B1
:108FB0009FED0F0AB4F90420D7F8C41F434630468A
:108FC000CDE900587DF02AF9CDE900589FED070A58
:108FD000B4F90620D7F8C81F4FF47A7330467DF0F5
:108FE0001DF902B0BDE8F081D08300200000FA44F2
:108FF00000007A4408B5094B93F8310410F02000C2
:109000000AD0D3F83C0403689B6D984739F00EFFF3
:10901000C82390FBF3F0C0B208BD00BFD09300207E
:10902000044B187820B9044B93F83204C0F3801035
:10903000704700BFA8CD0020D09300207FB500234B
:1090400003930493059317F077FD03A917F040FBF2
:10905000D8B117F071FDD0EDDA0A90EDDB0AF1EE30
:10906000600AB1EE400A3AF1F1FEDFED097A20EE36
:10907000270A39F051FEF6EE007A20EE270AFCEEC0
:10908000C07ACDED017A9DF8040007B05DF804FBCD
:10909000E02E654207B5124B93F8310410F0200022
:1090A0001AD003F58053D3F8940F00F565703FF0A4
:1090B0000DFFDFED0C7A20EE270ADFED0B7AB4EE20
:1090C000E70AF1EE10FA58BFB0EE670AFCEEC07A7C
:1090D000CDED017A9DF8040003B05DF804FB00BFFC
:1090E000D0930020CDCC4C3D00007F430B4B93F838
:1090F000212A7AB993F8552492060BD193F930249A
:10910000002A09DB93F8313413F0200F14BF042038
:10911000012070470520704703207047D09300203E
:1091200008B5074B93F9A432032B03D0BDE80840E0
:1091300079F070BB034A022179F0DCFA042008BD03
:10914000D073002004C31408094BD3F86C2D920788
:1091500001D477F0D7BF03F5405303F6647393ED62
:10916000000ADFED047AB8EEC00A20EE270A704745
:10917000D07300200AD7233C10B594B0044603A84E
:109180001FF06AF81C4BD3F83C04036803A95B6D1D
:10919000984778B3002103A81FF028F950B3247C26
:1091A000D9F0B0FC059BDDED047A0893069B09938A
:1091B0000023F8EEE77A9FED117A0B930C930D9351
:1091C0000E930F931093119312934FF6F853ADF83B
:1091D0004C300023962267EE877A8DF84E30332389
:1091E000CDE90032079007AA57212046CDED0A7A33
:1091F00076F060FE14B010BDD09300200AD7233C57
:10920000F0B52DED0A8B834C0546D4F83C04036879
:1092100099B05B6A9847002867D004F54054D4F8A9
:109220008832062B00F2E180DFE803F004040463D7
:10923000A0C35F0078489FED798A0DF0A7F9044636
:10924000D0E90201FBF7EEFC0746D4E90401FBF785
:10925000E9FC0646D4E90001FBF7E4FC9FED700A47
:109260000B900BA80C970D963FF010FAF0EE489A71
:10927000B0EE40CAF0EE60BAB0EE419AB0EE48AA45
:10928000F0EE488AF0EE48AAB0EE48BA40F6F8543C
:109290002D7CD9F037FC00231593169301238C22E3
:1092A0008DF85E303323CDE900320B90B1EE499A50
:1092B000F1EE688AB1EE488A0BAA552128468DED59
:1092C0000CCACDED0DBA8DED0E9A8DED0FBACDED28
:1092D00010AACDED118A8DED12AACDED139A8DED68
:1092E000148AADF85C4076F0E5FD19B0BDEC0A8B50
:1092F000F0BD49480DF04AF90446D0E90201FBF7F8
:1093000091FC0746D4E90401FBF78CFC0646D4E93E
:109310000001FBF787FC9FED420A0B900BA80C970E
:109320000D963FF0B3F93C48F0EE60BAB0EE419ACA
:10933000B0EE40CA0DF02EF99FED390A3FF0A6F9C4
:109340003548B0EE40BAF0EE60AAF0EE418A0DF07A
:1093500025F99FED330A3FF099F94FF44064B0EEE0
:1093600040AAF0EE609AB0EE418A91E72A489FED5C
:109370002B9A0DF00FF99FED2A0A3FF087F9264846
:10938000B0EE40BAF0EE60AAF0EE418A0DF006F9B8
:109390009FED230A3FF07AF9F0EE49BAB0EE40AA09
:1093A000F0EE609AB0EE418AB0EE49CA40F607444A
:1093B0006EE71948DFED198A0DF0F0F89FED180AF5
:1093C0003FF064F9F0EE68AAB0EE40AAF0EE609AC1
:1093D000B0EE418AB0EE68BAB0EE689AF0EE68BAC4
:1093E000B0EE68CA40F63F4452E79FED0C8A002475
:1093F000F0EE489AB0EE48AAF0EE488AF0EE48AA9D
:10940000B0EE48BAB0EE489AF0EE48BAB0EE48CAAC
:109410003EE700BFD09300201CC6002000000000E3
:109420000AD7233C2DE9F0412DED068B3B4D95F8F5
:10943000313499068CB004466AD505F580579FED06
:10944000380AD7F88C0FDFED378A6C303FF01EF901
:109450008DED041A21EE281AD5F83C648DED020A30
:10946000BDEEC11ACDED030A11EE103A1DB23368FC
:1094700094F810809B6D304660EE289A20EEA89AF2
:10948000984707EE900AF8EEE77A304667EEA87A3A
:10949000FDEEE77A17EE903A1CB23368DB6D984721
:1094A00007EE900AB8EE678AD7F8943FDFED1E7A90
:1094B00093ED0FAA336828EE288A1B6EB4EEE78A74
:1094C000F1EE10FA58BFB0EE678A30469847BCEE0E
:1094D000C88A0023089318EE103AB7222AEE28AA69
:1094E00020EE280AADF82C301A23CDE900323E21B7
:1094F00005AA4046CDED059A8DED069A8DED07AA99
:109500008DED090AADF82850ADF82A4076F0D2FC6E
:109510000CB0BDEC068BBDE8F08100BFD0930020FD
:109520009F0CB3450AD7233C00FF7F472DE9F04F3E
:109530002DED028B1A4B047CD3F88C3F8DB0D3F801
:109540008480D3F88870D3F88C60D3F8905093ED72
:10955000258AD3F898B0D3F89CA0D3F8DC90D9F042
:10956000D1FA00238DF82C3016222523CDE90032C4
:10957000029002AA532120468DED078ACDF820B033
:10958000CDF824A0CDF82890CDF80C80049705964E
:10959000069576F08FFC0DB0BDEC028BBDE8F08F28
:1095A000D0A3002070B58A7A4B7A43EA0223CA7AA4
:1095B00043EA02439D2B06460C4621D1134D95F8F4
:1095C000A51005F12C0082F007FDC8B195F8A51093
:1095D00005F12C0082F014FD022811D195F8A51098
:1095E00005F12C0082F000FD50B9D4ED057A9FED15
:1095F000080A0848F8EEE77A27EE800A02F0ECFB4A
:1096000021463046BDE8704077F042BFD0B300201D
:109610000AD7233C1CCC0020054BD3F860342BB177
:1096200093F8CA00002808BF022070470220704744
:10963000D093002008B5034BD3F83C0403681B68A3
:10964000984708BDD0930020024B93F83104C0F333
:1096500040107047D093002070B52C4E2DED028B3A
:109660000546D6F83C0491ED018A036886B05B6A32
:109670000C46984750B9BDEEC88A18EE103ADB0781
:1096800004D4022006B0BDEC028B70BDD4E9040105
:109690003AF040FF0028F4D002A81EF0DDFD02AA37
:1096A000214628467CF0C8FC0028EAD0184902A8C8
:1096B0001EF03CFF03460028E3D1DFED160A0090C0
:1096C0000246B0EE600A144802A90CF04DFDD8B174
:1096D000D6F83C0403685B6A9847044608B100204A
:1096E000D0E70E480222042106F00CFA60B1DFED4B
:1096F000090A094800942346B0EE600A224602A9EE
:109700000CF032FD0028EAD10420BBE7D093002002
:1097100030B30020000000001CC60020D033002021
:1097200008B591F82030032B1CD1D1ED027A9FEDC2
:109730000E7A91ED060A0D4BF0EEE77AF4EEC77A59
:10974000DFED0B7AD3F83C04F1EE10FA4CBF0121A7
:10975000002120EE270A13F0F1FC002814BF00209E
:10976000042008BD0220FCE700000034D093002054
:109770000000C84210B52DED028BD1ED007AF5EE58
:10978000C07AF1EE10FA82B00C4604DA042002B07E
:10979000BDEC028B10BD9FED197AF4EEC77AF1EEA5
:1097A00010FAF3D891ED030A9FED158AF0EEC07A16
:1097B000F4EEC87AF1EE10FA19D5D4ED037A114817
:1097C000D4ED010A94ED000AF4EEC87AD4ED027AE1
:1097D000FDEEE77AF1EE10FACDED017A9DF9041075
:1097E000ACBF0122002202F059FA0020CFE7F7EEC9
:1097F000000A39F023FA0028C8D0DEE70000B4439D
:10980000000000341CCC002091ED010AB5EEC00A26
:10981000F1EE10FA08B501DC042008BD9FED107AC6
:10982000104BD1ED007AD3F83C0420EE070A9FEDEF
:109830000E7A0368F4EEC77AF1EE10FA05DDDB6EFE
:1098400098470028E8D00020E7E79FED087AF4EE7B
:10985000C77AF1EE10FACCBF9B6E5B6EF0E700BFEB
:109860000000C842D09300209A9939403333F33F27
:1098700008B5D1ED007A9FED157AF0EEE77AF4EEB7
:10988000C77AF1EE10FA1DD5D1ED017AF0EEE77A44
:10989000F4EEC77AF1EE10FA14D50D480222032136
:1098A00006F030F980B10A480121FDF7C1F90948F5
:1098B00090F8803D012B03D000F67C5042F0BCFDB7
:1098C000002000E0022008BD0420FCE70000003476
:1098D000D0330020D0B3002010B5D1ED007AFCEEDB
:1098E000E77A17EE903A9CB2012C02D0022C06D0F7
:1098F0004CB90648214692F093FA002010BD044866
:1099000003F044FEF9E70420F8E700BFECB40020C0
:10991000D03300201FB5D1ED017A0B7CFCEEE77A45
:10992000CDED027AD1ED007A0093FCEEE77AD1ED2D
:10993000030ACDED037A91ED020A9DF808309DF8F7
:109940000C200146024812F0D1F805B05DF804FB86
:10995000D033002013B513480C46D2F061FFF0B1AC
:10996000D4ED017AFCEEE77ACDED017A9DF80400A2
:10997000012807D002280CD088B90B4B83F87A0C49
:1099800002B010BD94ED020A0648D2F05BFF002041
:10999000F6E794ED030A0348D2F098FFF7E70420B6
:1099A000EEE700BF3C900020D083002010B50A4CA9
:1099B00094F85534DB070CD402220521A4F5C040ED
:1099C00006F0A0F828B902221146A4F5C04006F01E
:1099D00099F8002010BD00BFD093002010B5D1ED44
:1099E000007AFCEEE77A044617EE903A13F0FF0394
:1099F0000FD10F4BD3F83C0403689B6F984708B115
:109A0000002010BD0B4A2046062178F073FE04208A
:109A1000F7E7012B09D1064BD3F83C040368DB6F51
:109A200098470028ECD1044AEDE70220E9E700BF9F
:109A3000D093002028C3140838C314089FED0B7A74
:109A400001F10C03F1EC017AF4EE677AF1EE10FA11
:109A50000AD6F0EEE77AF4EEC77AF1EE10FA03DCFC
:109A60009942EFD1012070470020704700007A44EE
:109A700030B52DED028B8DB0002305460393049382
:109A8000059317F059F803A916F022FE58B317F002
:109A900053F800F55A7393E8070006AC84E8070012
:109AA000DDED060A9DED070A2D7CF1EE600AB1EEB0
:109AB000400A3AF1CBF92046B0EE408A3FF006FA70
:109AC000DFED0B7A089B0B93012228EE278A0C23EB
:109AD000CDE90032A82109AA28468DED098A8DED2D
:109AE0000A0A76F0E7F90DB0BDEC028B30BD00BF7D
:109AF000E02E65422829F7B505460E4623D00CD83E
:109B000024292BD0272910D01B290CD031462846D8
:109B100003B0BDE8F0407CF027BE402928D0A1F179
:109B20004203012BF2D8012405E0122175F078FBE5
:109B3000044618B90024204603B0F0BD297C204813
:109B40006DF0AEFBF7E7162175F06AFB04460028BE
:109B5000F0D0297C1A486DF07DFCECE70C2175F003
:109B60005FFB04460028E5D02846FFF781FFE2E7C7
:109B7000262175F055FB04460028DBD0297C1148CE
:109B8000AAF082FA104B1F68002FD4D02621284655
:109B900075F046FB04460028CDD000230DF10602E7
:109BA00031462846ADF806307DF038FD0028C2D099
:109BB000BDF80620297C3846A2F0BEF8BBE700BFFE
:109BC0002CB50020D0BE0020C4DB002038B5194CD5
:109BD00094F85534DB070D460AD4D4F8603493F872
:109BE000D5303BB90122114604F1E000FCF76EFECE
:109BF000002038BD94F93034002B4FF0020212DA05
:109C00000521A4F5C04005F07DFF0028F0D095EDBA
:109C1000000ADFED097AD4F83C0420EE270A01217E
:109C200013F08CFAE4E70921A4F5C04005F06AFFBF
:109C3000DEE700BFD09300200000C84210B5214CE1
:109C400094F85534DB070ED4D4F8603493F8D5304B
:109C50004BB194F93034002B07DA0122082104F1CA
:109C6000E000FCF7EFFE002010BDD1ED007A9FED83
:109C7000167AF0EEE77AF4EEC77AF1EE10FA0BD529
:109C800012480222112105F03DFFA0B9022211461F
:109C90000E4805F037FFE6E7D4F83C0403681B687C
:109CA00098470428DFD0D4F83C0403681B68984721
:109CB0001428E5D1D7E7064840F6C41109F0C4FEE0
:109CC000D1E700BFD093002000000034D033002043
:109CD000C0C4002073B58B8BC12B05460C4644D8FD
:109CE000BB2B0DD8202B67D02ED8113B99B205295C
:109CF00018D92146284602B0BDE870407EF018B859
:109D0000BC3B052BF5D801A151F823F05D9E00085E
:109D1000679E0008F39C0008F39C0008EB9D000878
:109D2000F79D0008052BE4D801A151F823F000BFEE
:109D3000439E0008F39C0008F39C0008579E00080F
:109D4000579D00080D9E0008732B30D006D8542B69
:109D50005CD0552BCDD10222092174E0B22BC8D1A1
:109D600002B0BDE87040FFF74FBD4AF21146B34262
:109D700058D00BD8D12B44D0B3F5967F57D0D02BE9
:109D8000B7D102B0BDE87040FFF7A6BD4AF2134656
:109D9000B34242D04AF26866B3424DD04AF212460C
:109DA000B342A6D102B0BDE87040FFF70FBF02B0CA
:109DB000BDE87040FFF7DEBCD1ED007AF5EEC07A69
:109DC000F1EE10FA54DD9FED2B7AF4EEC77AF1EE46
:109DD00010FA4DD8FCEEE77A274ACDED017A9DF8CE
:109DE0000430A2F8923C002033E0214602B0BDE8E6
:109DF0007040FFF731BC214602B0BDE87040FFF76C
:109E0000EDBD02B0BDE87040FFF784BD2146284695
:109E100002B0BDE87040FFF783BC02B0BDE87040FF
:109E2000FFF70CBF02B0BDE87040FFF7BFBD02B046
:109E3000BDE87040FFF71CBD02B0BDE87040FFF701
:109E400089BD022205210D4805F05CFE0028CAD11B
:109E5000042002B070BD02220621F4E70221084866
:109E600007F07AF9F2E70221054807F03FF9EDE73C
:109E70000220EEE700007F43D0830020D033002093
:109E800010C1002008B591ED007AF6EE007AB4EE2C
:109E9000E77AF1EE10FA06DD044801220521FCF70D
:109EA000D1FD002008BD0420FCE700BFB0940020D5
:109EB00030B52DED028BCD7893B0272D28BF272507
:109EC0000C462722002108A83CF1A0FA2A4604F1FA
:109ED0000C0108A83CF150FA424BD3F83C0403684B
:109EE0005B6A9847002841D09DF8465068063DD4EB
:109EF00000244FF07E53290604930794069405949A
:109F000027D504A83DF0BCFCEA0701940294039411
:109F100005F006032ED4002B2ED10D9B01930E9B32
:109F200002930F9B039330480BF046FE9DED100A01
:109F3000044630B340F2ED40B7EE001AFFEE000ADF
:109F400038F0A0FF2848234601AA04A90BF03CFEE4
:109F50000CE0099B04930A9B05930B9B069304A8B2
:109F60000C9B07933DF092FC0028CDD113B0BDECC3
:109F7000028B30BD062BD6D001211B480BF0B8FD5B
:109F8000F4E7DFED1A0A4FF49E60B7EE001A38F0DE
:109F900079FFF6EE000AB0EE408A38F04FFEE8B9DD
:109FA000B6EE000A124BB4EEC08AF1EE10FAD3F806
:109FB000983F08DD38EE400A30EE008A93ED070A3C
:109FC00028EE000ABEE730EE480AD3ED087A30EEFC
:109FD000000AF0EEE77A27EEC00AB3E79FED030A26
:109FE000B0E700BFD09300201CC600200000000096
:109FF000D0A300202DE9F0439DB0814608460EA96C
:10A00000FEF740FD844BD3F83C0403685B6A984735
:10A0100050B19DF86C30012B09D0DA1F022A06D905
:10A020007E4801210BF064FD1DB0BDE8F083BDF852
:10A030006840A20504F0070604F0380704F4E07550
:10A0400001D5002DF0D04FF00008CDF81480CDF8E8
:10A050001880CDF81C803EBB9FED716A9DED107A93
:10A06000DDED117ADDED0F6A27EE067A67EEC67A2E
:10A0700066EE866A083B012BCDED056A8DED067A0A
:10A08000CDED077A04D8674806AA05A9FCF758FF62
:10A090009DF86C30073B022B06D86348CCF0B6FF26
:10A0A000014605A83EF012FBCDF82080CDF82480B3
:10A0B000CDF82880F7B9DDED147A129B0893F1EE04
:10A0C000677A139B099308A94846CDED0A7AFFF7F2
:10A0D000B5FC0028A4D09FED520A08A83EF02AFB48
:10A0E0009DF86C30083B012B04D84E4809AA08A9FA
:10A0F000FCF726FFCDF82C80CDF83080CDF83480E9
:10A10000EDB99FED476A9DED167ADDED177ADDED2D
:10A11000156A9DF86C3027EE067A67EEC67A66EE11
:10A12000866A083B012BCDED0B6A8DED0C7ACDEDE7
:10A130000D7A04D83B480CAA0BA9FCF701FF14F4D4
:10A14000806233D1DFED397A9DED180A9DF86C10ED
:10A1500020EE270ADFED327A0839012920EE270A9E
:10A160008CBF0021012114F4006305BFDFED2F7ABD
:10A17000DDED190ADFED2E0A60EEA70A04BFDFED60
:10A18000287A60EEA70AAEB9002F35D1B3FA83F36F
:10A19000B2FA82F25B0952090291019300920BAB71
:10A1A00008AA05A91D480CF0E5F83DE79FED200A37
:10A1B0000021D8E77FB9B3FA83F35B09012000934C
:10A1C000B2FA82F3CDE901105B0914480BAA08A981
:10A1D0000BF066FE28E7002D7FF422AF0120B3FAD2
:10A1E00083F3B2FA82F2CDE900105B090B48520901
:10A1F0000BA90BF0EBFD17E7002D3FF411AFB3FAFD
:10A2000083F3B2FA82F2CDE900165B09520905A97F
:10A2100002480BF0C3FE07E7D09300201CC60020C5
:10A220000000C842D033002040B30020E02E654239
:10A23000000000002DE9F047A2B08046084614A9AE
:10A24000FEF720FC7E4BD3F83C0403685B6A98471A
:10A25000C0B1BDF88040A30504F0070904F4E0771D
:10A2600000D57FB10CAE30461DF0F6FFB9F1000FFE
:10A2700029D1DDE915013AF04DF930B971480121D4
:10A280000BF036FC22B0BDE8F0879DF8841009AAD7
:10A2900040467BF0BBFE0028F0D0DDED177A9FED45
:10A2A0006A7A099B009367EE877A10ADFDEEE77A34
:10A2B000DDE9151217EE903A28461DF0EDFF95E8FE
:10A2C0000F0086E80F00002514F0380A0695079560
:10A2D000089514D1DDED1A7A189B0693F1EE677A92
:10A2E000199B079306A94046CDED087AFFF7A6FB18
:10A2F0000028C3D09FED540A06A83EF01BFA09952A
:10A300000A950B959FB99FED506A9DED1C7ADDED86
:10A310001D7ADDED1B6A27EE067A67EEC67A66EED9
:10A32000866A8DED0A7ACDED096ACDED0B7A14F4CB
:10A33000806805BFDFED457A9DED1E0A9FED440A5A
:10A3400020EE270A04BFDFED407A20EE270A14F43E
:10A35000006405BFDFED3D7ADDED1F0ADFED3C0A4D
:10A3600060EEA70A04BFDFED387A60EEA70AB9F104
:10A37000000F31D1BAF1000F52D13046CDED050AB0
:10A380008DED040A1DF098FF03289DED040ADDED14
:10A39000050A3FF473AF10A93046CDED050A8DEDE7
:10A3A000040A1095119512951EF06EF900283FF4DD
:10A3B00065AFB4FA84F46409B8FA88F3DDED050AF0
:10A3C0009DED040ACDF804A000945B0906AA10A92B
:10A3D0001C480CF049F855E7BAF1000F0FD10123E2
:10A3E000B4FA84F4CDE901A36409B8FA88F31548F6
:10A3F00000945B0909AA06A90BF052FD42E7002F61
:10A400007FF43CAF0123CDE90073B8FA88F2B4FAC7
:10A4100084F30C485B09520909A90BF0D7FC31E71A
:10A42000002F3FF42BAFB4FA84F3B8FA88F2CDF8DA
:10A4300000905B095209314602480BF095FE21E776
:10A44000D09300201CC600200000C842E02E6542C8
:10A450000000000030B48D7A4B7A43EA0523CD7AB0
:10A4600043EA0543562B04460A461BD008D8522B14
:10A4700012D0542B13D02046114630BC7CF0C4BC03
:10A4800003F18073863B23F07F43012BF3D8017CDB
:10A49000064830BC6DF0A6B830BCFFF709BD30BC33
:10A4A000FFF7A8BD30BCFFF7C5BE00BF2CB500202C
:10A4B0002DE9F0412DED028B044690B000F50140EE
:10A4C0000023012269465C3000936DF039FE08B923
:10A4D0004F4B009304F5C046DFED4E8AD6F83C049E
:10A4E00003685B69984704F5E048002840F08C80D9
:10A4F000D8F8945FD5E9E001FAF794FB07EE900AEB
:10A5000027EEA88AD5EDE77AFDEEE77A17EE903AC6
:10A510001DB204F5C047683701A9384612F03EF96C
:10A5200018B970F0CFFF3A4B01933722002102A8EF
:10A530003BF16CFFA3238DF8083095238DF809308B
:10A54000D8F0E8FAD8F88C3FCDF80B00D6F86004C4
:10A55000D3F8DC20D3F8E030CDF80F104430CDF83C
:10A560001320CDF8173073F065FD0346DFED2A0A9E
:10A5700093ED000AB7EE001A9F2038F083FC10EE2E
:10A58000103AD6F86004CDF81B3003681B69984771
:10A5900010EE103A04F5FE46CDF81F30703618EE76
:10A5A000103A3046CDF82330CCF034FD20EE280AA6
:10A5B000384610EE103ACDF82730D8F83C3FCDF8A9
:10A5C0002B30019BCDF82F3012F014F910EE103A19
:10A5D0003046CDF83330009BCDF83730ADF83B50E6
:10A5E000CCF024FDBDEEC00A04F5D25010EE103AB6
:10A5F000372202A90830ADF83D306FF053FF10B09C
:10A60000BDEC028BBDE8F0819FED038A002580E759
:10A610002292CA7F0AD7233C0000000010B500F543
:10A62000E044D4F88C0FC3F007F9D4F8941FD4F8A1
:10A630008C0FBDE81040C3F065B9000070B54FF451
:10A640008051054612F028FA00284FD005F5E04663
:10A6500005F5D254D6F88C0F03689B6898470834E8
:10A6600000F1A002692120466FF05AFDD6F88C0F48
:10A670000368DB6898476A2100F1A00220466FF06A
:10A680004FFDD6F88C0F03681B6998476B2100F1CA
:10A69000A00220466FF044FDD6F8942F6C2120468E
:10A6A00002F52D726FF03CFD2021284612F0F4F9DE
:10A6B000E0B105F5C043D3F83C0403681B69984733
:10A6C00078B1D6F8942F204690326E216FF028FD95
:10A6D000D6F8942F2046BC32BDE870406F216FF051
:10A6E0001FBD28460CF072FC0028EAD170BD0000A6
:10A6F00008B516F021FABDE8084015F00DBF0000BE
:10A700007FB50E464FF6FF710446154612F0C4F9A8
:10A71000E8B11022002168463BF178FEA3238DF8B2
:10A72000003095238DF8013003238DF80230D8F0E6
:10A73000F1F9CDF8030004F5D250CDF8071010223E
:10A74000694608308DF80B6003956FF02BFF04B05D
:10A7500070BD00007FB50E464FF6FF7104461546EA
:10A7600012F09AF9E8B11022002168463BF14EFE42
:10A77000A3238DF8003095238DF8013004238DF844
:10A780000230D8F0C7F9CDF8030004F5D250CDF867
:10A7900007101022694608308DF80B6003956FF0A2
:10A7A00001FF04B070BD000030B52DED048B87B003
:10A7B00004460D46182200216846B0EE409AF0EE9D
:10A7C000608AB0EE418A3BF121FEA3238DF8003070
:10A7D00095238DF8013006238DF80230D8F09AF9D0
:10A7E000CDF8030004F5D250CDF8071018226946C1
:10A7F00008308DF80B508DED039ACDED048A8DED68
:10A80000058A6FF04FFE07B0BDEC048B30BD000031
:10A8100010B54FF48011044612F03EF930B104F542
:10A8200010503030BDE8104014F0F0B910BD0000F9
:10A830002DE9F04F2DED028B8DB080462F220021A7
:10A84000684611EE10BA11EE90AA12EE109A12EEAE
:10A85000907A13EE106A13EE905A14EE104AF0EE4E
:10A86000408AB0EE608A3BF1D1FDA3238DF8003021
:10A8700095238DF8013009238DF80230D8F04AF97C
:10A8800018EE903ACDF80300CDF80B3008F5D25011
:10A8900018EE103ACDF807102F2269460830CDF88F
:10A8A0000F30CDF813B0CDF817A0CDF81B90CDF830
:10A8B0001F70CDF82360CDF82750CDF82B406FF0F6
:10A8C000F1FD0DB0BDEC028BBDE8F08F30B52DED84
:10A8D000088B8BB004460D46282200216846B0EE56
:10A8E00040BAF0EE60AAB0EE41AAF0EE619AB0EE86
:10A8F000429AF0EE628AB0EE438A3BF187FDA323D1
:10A900008DF8003095238DF801300A238DF8023040
:10A91000D8F000F9CDF8030004F5D250CDF80710B7
:10A920002822694608308DF80B508DED03BACDED25
:10A9300004AA8DED05AACDED069A8DED079ACDED11
:10A94000088A8DED098A6FF0ADFD0BB0BDEC088B68
:10A9500030BD00002DE9F0438FB01446054689460E
:10A960003122002101A8DDE9167698463BF14EFD23
:10A97000A3238DF8043095238DF8053008238DF836
:10A980000630D8F0C7F82368049363680593A3687A
:10A9900006933B68CDF81D307B68CDF82130BB684D
:10A9A000CDF825303368CDF80700CDF8293005F50E
:10A9B000D2507368CDF80B10CDF82D303122B3682A
:10A9C0008DF80F9001A908308DF81C80CDF831303A
:10A9D0006FF068FD0FB0BDE8F083000070B52DED9D
:10A9E000068B8CB0144605460E462C22002101A889
:10A9F000B0EE409AF0EE608AB0EE418AB0EE61AA05
:10AA0000F0EE429A3BF102FDA3238DF8043095232A
:10AA10008DF805300B238DF80630D8F07BF8DFED8C
:10AA20001A7A94ED007ACDF8070027EE277A29EEFE
:10AA3000279A8DED077A94ED017ACDF80B1027EE69
:10AA4000277A68EEA78A8DED087A94ED027A8DF860
:10AA50000F6028EE278A05F5D25067EE277A2C2260
:10AA600001A908308DED049ACDED058A8DED068A99
:10AA7000CDED097A8DED0AAACDED0B9A6FF012FD9E
:10AA80000CB0BDEC068B70BDE02E6542B020704767
:10AA900030B5154B044689B004F5D255D3F860049F
:10AAA000694608351E22CDF01FFF6A460F49284629
:10AAB0006FF094FE04F5C043D3F83C0403681B68B0
:10AAC000984704F58043014693F8642028466FF0C8
:10AAD000A9FE04F51050303016F098FA04F55670BF
:10AAE00028F01AFD09B030BDD09300208DF0170872
:10AAF000F8B5424B4360002343618361C361C36384
:10AB00003F4A404B426303644FF080423E4B4364F4
:10AB1000044682634830BCF005FB04F5827096F071
:10AB2000D1FD04F52B607DF0B9FE384F384BC4F8E9
:10AB3000B03A40F6683540F6686660197EF016F95E
:10AB400067513035B542F8D104F668607FF0DCFF1C
:10AB500004F5C75000211430D1F07CF904F5CD5034
:10AB600004F580560430D1F04BFE2A4DC6F8C45986
:10AB700004F5CE500830D2F0D1FBA5F5E76304F51B
:10AB8000D350C6F8583A04309DF03CFBA5F50C7341
:10AB900004F5E150D435C6F81C3C9FED1F1ADFEDDB
:10ABA0001F0A9FED1F0AC6F8285C0C30C3F00AFE8E
:10ABB0009FED191A9FED1B0A04F5E250F0EE410AD1
:10ABC0000430C3F0FFFD9FED141A9FED160A04F543
:10ABD000E250F0EE410A1C30C3F0F4FD04F5E550FC
:10ABE0000C30C8F0C5FC20460F4963F0B3FE204688
:10ABF0000E4963F0AFFE2046F8BD00BF984A002022
:10AC00000000C8410AD7233C0000E0407C1615082C
:10AC10009016150874CA0020000000009A99993E09
:10AC20000000B44300804A43F0081508E00B150803
:10AC300070B54C4D4C49ADF50E7DD02206465AA854
:10AC40003BF19AFB0FCD0EAC0FC40FCD0FC40FCD4F
:10AC50000FC495E80F0084E80F0000245AAB1819C0
:10AC60000021B7EE000A103463F036FBD02CF5D18A
:10AC70003E4B0FCB02AC84E80F0001A9204663F0E5
:10AC8000DFFA90B19DF90430DFED396AE06807EE34
:10AC9000103AB8EEC77AF0EE007AE7EE267AB7EE11
:10ACA000000A80EE270A64F0E3F900240EAB1819BD
:10ACB00000211034B7EE000A63F00EFB402CF5D1F2
:10ACC0002C49902236A83BF157FB0022092136A8D7
:10ACD00063F0AEFB96F9D46DD6B9274D0FCD1EACFF
:10ACE0000FC40FCD0FC40FCD0FC495E80F0084E83B
:10ACF0000F00324604211EA863F09AFB9FED1F0A45
:10AD00001F4864F0B5F91F48B7EE000A64F0B0F9C7
:10AD10001D4C9FED1E0A0FCC06AD0FC594E80F0029
:10AD200085E80F00002106A863F0D6FA9FED170A08
:10AD30000021284663F0D0FA04F1100160221EA819
:10AD40003BF11AFB00241EAB18190021B7EE000AD4
:10AD5000103463F0C1FA602CF5D17FF02FFC0DF5B3
:10AD60000E7D70BDECA814081CA814082CA91408AA
:10AD7000CDCCCC3D3CA91408CCA91408000000009F
:10AD8000D8071508E70715080CAA14080000344274
:10AD900010B5B4B00849D02268463BF1EDFA002462
:10ADA0000DEB04000021B7EE000A103463F094FAB2
:10ADB000D02CF5D134B010BD8CAA14082DE9F04781
:10ADC00090B00DF106011D207FF0ECFC002800F092
:10ADD0009E809DF80630614A0133DBB211210BA839
:10ADE0008DF80630D7F084F800220DF107010BA88A
:10ADF00062F072FF9DF80630594A112105460BA8F2
:10AE0000D7F076F800220DF107010BA862F064FF7D
:10AE10009DF80630534A112106460BA8D7F068F872
:10AE200000220DF107010BA862F056FF9DF80630D5
:10AE30004D4A03F03F03112107460BA8D7F058F8FD
:10AE400000220DF107010BA862F046FF8046002D9D
:10AE50005DD0002E5BD0002F59D0002857D0284657
:10AE600063F036F9002852D1304663F031F90028FA
:10AE70004DD1384663F02CF9002848D1404663F0A4
:10AE800027F9002843D1394C94E80F000DF10C0C40
:10AE900010348CE80F0094E80F000DF11C0989E8CC
:10AEA0000F0002A9604663F0CBF998B3BDF80840E3
:10AEB00002A9484663F0C4F900284AD0BDF808301A
:10AEC00054BB23B340F2E2449C420FFA84FA0FFAD7
:10AED00083F927D80DF10A013046ADF80A9064F0E5
:10AEE0008FFD0DF10A012846ADF80AA064F088FD37
:10AEF0000DF10A013846ADF80AA064F081FD002387
:10AF00000DF10A014046ADF80A3064F093FD10B02F
:10AF1000BDE8F0870024CBE740F2D662002B08BFE3
:10AF20001346D1E70DF10A013046ADF80AA064F0EE
:10AF300067FD0DF10A012846ADF80A9064F060FD46
:10AF40000DF10A013846ADF80A9064F059FD01236D
:10AF5000D6E7002CDBD040F2D663B5E7F80715083A
:10AF600004081508100815081D0815085CAB14081E
:10AF700037B500F584417822543104466DF0C4FAA7
:10AF800000220C21284863F053FA2046FFF716FFF1
:10AF900004F584400022B7EE000A0221683063F015
:10AFA000CFFA012504F5775100230C3145201F4AC3
:10AFB000009563F041FA1E490B68D8070CD41D4B6D
:10AFC0000D6004F568521A6004F57B522032DA6095
:10AFD00004F5DA521C329A6104F5854015490322C2
:10AFE000483063F07BFA012504F5D251124A0095EE
:10AFF00000230831FD2063F01FFA104B1A68D207B6
:10B0000005D40F4A1D6004F50C541C3414600C4820
:10B01000012163F07FFA63F091FE0A4A138843F03E
:10B020000103138003B030BD30081508900D1708D8
:10B0300014CC0020C42500201808160818CC0020C5
:10B04000E82500209CCF00200F299DBF302303FB63
:10B050000100B83000207047014B93F99B02704704
:10B06000D0730020024B93F8550400F001007047A4
:10B07000D0930020044BB3F86032DB075ABF00695D
:10B08000C0F3401000207047D0730020014BD3F86C
:10B09000C80F7047D083002008B503689B689847A5
:10B0A00030B9044B93F95404B0FA80F0400908BD5C
:10B0B0000020FCE7D093002038B50C1E2EDB184D85
:10B0C00095F8D42FE3B29A4228D3D5F8D03F012285
:10B0D000195DA5F5A04004F015FDF8B17DF078FDEF
:10B0E00003217EF0DDFFC8B97DF072FD0D217EF0F9
:10B0F000D7FF98B9A5F58052A5F5A04092F9803206
:10B10000E340DB075ABF92F99A12E1400221BDE801
:10B11000384058BF01F00101FBF7A0BD38BD00BFAA
:10B12000D0830020022910B5044606D10146BDE8AF
:10B1300010400948352204F0E5BC084BD3F83C0424
:10B1400003681B689847844205D17DF041FDBDE846
:10B1500010407DF0B7BC10BDD0330020D09300204C
:10B1600029B1022907D1044BC3F834147047024BAC
:10B170000122C3F834247047D093002031B1022952
:10B1800007D1044B012283F838247047014B83F820
:10B1900038147047D093002010B500F5A043DFEDC0
:10B1A000186AD3F8C02FD3F8BC3FB2F90820B3F91E
:10B1B00008309FED147A07EE902AF8EEE77A0446FD
:10B1C000C7EEA60A00F510500121303007EE903A84
:10B1D000F8EEE77A60EE870A87EEA60A20EE070A05
:10B1E00015F04CFD70F06EF926216FF0FDFE04F5B0
:10B1F000C340054ABDE810400621483073F0AEBD9B
:10B200000000C84235FA8E3C5414150800F5E0429F
:10B21000002382F8A83F044A00F5C34013720621B8
:10B22000024A483073F09ABDEDCE00206014150834
:10B2300070B500F5E045044695F8A81F002957D0E1
:10B240002C4B2D4AD3F83C04904204D1D3F86034FF
:10B2500093F8D53023B92046BDE87040FFF7D6BF3C
:10B26000264E95F8A90F04F5C043012293F9303416
:10B270003272D0BB002B3BDB85F8A92F0139C9B254
:10B2800004F5A04385F8A81FD3F8C02FD3F8BC3F1E
:10B29000B2F90820DFED1A6AB3F908309FED197A88
:10B2A00007EE902AF8EEE77AB1FA81F1C7EEA60A26
:10B2B00004F510504909303007EE903AF8EEE77A7D
:10B2C00060EE870A87EEA60A20EE070A15F0D6FC84
:10B2D00095F8A83F63B904F5C34033720A4ABDE844
:10B2E00070400621483073F039BD002BC6DAB2E752
:10B2F00070BD00BFD093002008C80020EDCE002014
:10B3000000007A4535FA8E3C741415086D2900F357
:10B31000E380012901DC7EF0A3BC8B1E6B2BFAD8E5
:10B320000FF2040C5CF823F037B5000831B50008C3
:10B3300037B5000837B5000817B3000837B500085F
:10B3400017B3000817B3000831B5000817B3000899
:10B3500037B5000831B5000831B5000817B300084B
:10B3600037B5000837B5000837B5000817B300082F
:10B3700017B3000831B5000837B5000831B500082B
:10B3800017B3000831B5000831B5000817B300083D
:10B3900017B3000817B3000817B3000817B3000865
:10B3A00031B5000837B5000817B3000817B3000817
:10B3B00017B3000837B5000817B3000831B5000807
:10B3C00017B3000817B3000837B5000831B50008F7
:10B3D00031B5000837B5000817B3000837B50008C5
:10B3E00037B5000837B5000817B3000817B30008D1
:10B3F00037B5000817B3000817B3000837B50008C1
:10B4000037B5000837B5000817B3000817B30008B0
:10B4100037B5000837B5000817B3000817B30008A0
:10B4200017B3000817B3000817B3000817B30008D4
:10B4300037B5000837B5000837B5000837B500083C
:10B4400037B5000837B5000817B3000831B5000854
:10B4500031B5000817B3000817B3000817B3000888
:10B4600017B3000817B3000817B3000837B5000872
:10B4700031B5000817B3000817B3000817B3000868
:10B4800017B3000817B3000817B3000817B3000874
:10B4900017B3000817B3000817B3000817B3000864
:10B4A00017B3000817B3000817B3000837B5000832
:10B4B00017B3000817B3000817B3000817B3000844
:10B4C00017B3000817B3000817B3000817B3000834
:10B4D00017B3000831B50008A12921DC96297FF7B0
:10B4E0001AAFA1F197030A2B3FF615AF0FF2040C28
:10B4F0005CF823F037B5000837B5000817B300082B
:10B5000037B5000817B3000817B3000817B30008D1
:10B5100017B3000831B5000831B5000837B5000889
:10B52000B42908D0DB2903D0B2297FF4F4AE7047E8
:10B5300000237EF05DBB704770B563298AB0144666
:10B5400000F3D280012905DC22460AB0BDE8704034
:10B550007EF058B88B1E612BF6D801A252F823F06A
:10B5600063B7000877B7000897B70008A1B70008CD
:10B5700049B50008D1B7000849B5000849B5000829
:10B5800087B8000849B5000849B5000885B7000824
:10B59000ABB8000849B5000881B80008E7B8000852
:10B5A000F7B8000849B5000849B500080FB9000808
:10B5B0001DB900082BB9000849B5000851B90008A9
:10B5C00063B9000849B5000849B5000849B5000845
:10B5D00049B5000849B5000875B900088FB90008D9
:10B5E00049B5000849B5000849B5000895B90008F3
:10B5F00049B500089BB9000849B5000849B50008DD
:10B60000B5B9000849B50008BBB9000867B700081C
:10B6100049B5000849B5000849B5000849B5000812
:10B6200049B5000849B500085FBA000849B50008E7
:10B6300049B50008FDB8000803B9000809B90008B9
:10B6400049B5000849B50008DBB9000815BA00087B
:10B6500049B5000849B5000849B5000849B50008D2
:10B6600049B5000849B500084DBA000853BA0008AA
:10B6700059BA000865BA00086BBA000871BA000828
:10B6800049B50008B5BA000877BA000849B50008FE
:10B6900049B5000849B5000849B5000849B5000892
:10B6A00049B50008E9BA000807BB000849B5000819
:10B6B00049B5000849B5000849B5000849B5000872
:10B6C00049B5000849B5000849B5000849B5000862
:10B6D00049B5000849B5000849B5000849B5000852
:10B6E00049B500081DBB0008A0291FDC96297FF77B
:10B6F0002BAFA1F19703092B3FF626AF01A252F819
:10B7000023F000BF23BB000829BB000849B500088F
:10B710003DBB000849B5000849B5000849B5000817
:10B7200049B5000815BB000861BB0008B42900F04A
:10B73000DD80DB2917D0B2297FF406AF002A00F0A4
:10B74000CC81022A0FD1A64BD3F83C0403689B6F2F
:10B75000984740B97AF0BEFEA24A042173F0FEFA7F
:10B7600001E0022C01D001242FE035220E219E4859
:10B7700004F0C8F9F7E7211E18BF01219A48FBF72A
:10B780006DFAF0E7012C04D0022C14BF0021022135
:10B79000F4E72146F2E721460620FFF7C3FCE2E783
:10B7A000022CE0D18E4DD5F83C040368DB6A984743
:10B7B00004460028D7D055F83C3CB3F90830002B9C
:10B7C000D1D1A5F5C040FFF7E7FC20460AB070BD17
:10B7D000022CC8D1824ED6F83C1406F5355291425F
:10B7E000C1D0D6F8602492F8D520002ABBD006F547
:10B7F0000054A6F58056B4F9B02D2AB9D6F8C43F46
:10B80000B3F90830002BAED01C22002103A805ADEF
:10B810003AF1FCFD28461CF01FFDB4F9B03D734C15
:10B8200093B91623ADF80E30D4F8643F7048642BFA
:10B83000B8BF642303A906933EF0B2F820B16FF0BD
:10B8400041FE27216FF0D0FB04F576630FCB85E82E
:10B850000F00D6F8C43F6648B3F90830002BCCBFC0
:10B860001023152303A9ADF80E303EF099F80028F7
:10B870003FF479AF6FF026FE27216FF0B5FB72E73A
:10B880002146032089E7022C5A4D03D0002385F876
:10B89000D83F68E75848192164F072FD0446002833
:10B8A000F4D0012385F8D83F8FE7012C0BD0022C70
:10B8B00012D0002C7FF457AF504B83F8C4426FF086
:10B8C00001FE2B21D9E74D4B83F8C4426FF0FAFDFE
:10B8D0002C216FF089FB78E7484B83F8C4426FF066
:10B8E000F1FD2D21C9E721460F2056E744481146B6
:10B8F000D4F00AFD37E7214609204EE7214604200F
:10B900004BE72146052048E72146172045E7A01EC2
:10B91000414241413B4890F083FA24E7022C7FF4F6
:10B9200022AF314801F032FE1DE7012C06D0022C77
:10B9300009D0002C7FF417AF2146EBE731482146B0
:10B9400090F06EFA41E72F48012190F069FAE8E79C
:10B95000264BA21ED3F88C3F5442544183F820401A
:10B9600001E7A31E59425941204BD3F88C0FC4F074
:10B9700035F8F8E61A4B013C93F83224012C8CBFC1
:10B980000024012464F3041283F83224EBE62146F8
:10B99000112002E721461220FFE6012234B1022CD9
:10B9A0007FF4E1AE184B83F81423DCE6164B83F8E2
:10B9B0001443D8E621461520EFE6012C08D9022CC5
:10B9C0007FF4D1AE9FED110A1148D0F07FFFCAE697
:10B9D000084B002283F87A2CC5E621461820DCE6C5
:10B9E000D0930020AF141508D0330020D0A300203E
:10B9F0004CC10020D0830020684B0020D073002071
:10BA00003CC30020ECB40020D0C3002000000000A4
:10BA10003C900020594BD3F83C04594B98427FF49A
:10BA2000A2AE01900FF02CFC012C019808D0022C42
:10BA30000AD0002C7FF497AE21460FF0D1FC92E69D
:10BA400000210FF035FCC0E60121F6E72146002079
:10BA5000A3E621461020A0E6214602209DE62146CD
:10BA600001209AE62146162097E62146072094E613
:10BA700021460B2091E6022C424B0ED1012483F883
:10BA8000A04C6FF01FFD4A216FF0AEFA7AF022FD54
:10BA90003D4A062173F062F997E6002283F8A02C54
:10BAA0006FF010FD4B216FF09FFA7AF013FD374ACB
:10BAB000062153E6012C09D0022C0CD0002C7FF477
:10BAC00052AE0121324810F0ADFE4CE63048002164
:10BAD00010F0A8FE79E62146F4E7284BD3F83C04A1
:10BAE0000368DB6F98473EE6244BD3F83C04244BB5
:10BAF00098427FF438AE022C02D10FF07BFD32E683
:10BB00000FF062FC2FE62146FFF72AFB214804F0E4
:10BB100047FD28E62146FFF731FB24E621461B209E
:10BB20003BE621461C2038E6022C7FF41CAE1A4866
:10BB3000FCF77AF97AF0CEFC184AB9E721467DF095
:10BB4000C1FB1748BCF000FD044600283FF40BAED3
:10BB50000A4A92F8333443F0020382F8333434E66D
:10BB6000012234B1022C7FF4FEAD0E4B83F8A02FDE
:10BB7000F9E50C4B83F8A04FF5E500BFD09300200A
:10BB800048CB0020D0B300208C1415089D14150854
:10BB90003894002094C00020D0330020C814150829
:10BBA000B0940020D083002010B504460448CBF0A8
:10BBB0002FFA04F10801BDE8104038F029BC00BF9D
:10BBC00040B3002038B504462DED028B1148CBF070
:10BBD00025FA05463CF014F90F48B0EE408A10F003
:10BBE000F5FE90B1DFED0D7AB4EEE78AF1EE10FAD2
:10BBF0000BDDD5ED000A95ED010A38F127F9DFEDEF
:10BC0000087A20EE270A84ED080ABDEC028B94ED39
:10BC1000080A38BD40B30020D033002000401C4645
:10BC2000E02E6542074B93F98102022805D00328D4
:10BC300006D0003818BF0120704781F0010070471E
:10BC400004207047D073002003688B4216D004296B
:10BC5000C0E9001302D007290ED07047084B9FEDB2
:10BC6000097A03F5C663D3ED007AF8EEE77A67EE5A
:10BC7000877AC0ED087A704700238362704700BF5F
:10BC8000D05300200AD7233C08B50246FFF7CAFF6D
:10BC9000BDE8084001461046FFF7D6BF70B52DED50
:10BCA000048B0446F0EE408AB0EE608A0D461646DC
:10BCB000D6F028FF9FED329ADFED329AE06176B33D
:10BCC000236843B9304B03F5C663D3ED007AF8EE31
:10BCD000E77AC4ED097A68EE898A002DB7EE000A8A
:10BCE000FFEE007AB8BFB0EE670A68EE808AC4ED56
:10BCF000058A264BB4EEE98AF1EE10FAD3F88C0FE0
:10BD000030DAC2F049FE20EE090A84ED060ABDECE5
:10BD1000048B20460321BDE87040FFF795BF94EDEA
:10BD2000090A98EE890A37F04BF8002D84ED050AD0
:10BD30000BDAB4EEE90AF1EE10FADADBDFED147A91
:10BD400030EE670A84ED050AD3E7D2D0DFED117A31
:10BD5000B4EEE70AF1EE10FACBD8DFED0D7A30EE53
:10BD6000270AEFE7C2F018FEB4EE480AF1EE10FA27
:10BD700048BFB0EE408A28EE098A84ED068AC6E7FD
:10BD80000000C84200000034D0530020D0A300209F
:10BD900000A00C47000000B410B52DED028B044646
:10BDA000B0EE608AF0EE408AD6F0ACFEDFED090A14
:10BDB000E06168EEA08A68EE200AC4ED098ABDEC55
:10BDC000028BC4ED0A0A20460621BDE81040FFF7A9
:10BDD0003BBF00BF0000C84210B52DED028B0446EA
:10BDE000B0EE408AD6F08EFE94ED090ADFED097AB6
:10BDF000E061A8EE270A36F0CDFFBDEC028B0023F0
:10BE000084ED090AA36220460621BDE81040FFF731
:10BE10001BBF00BF0000C84270B54B68154D0646F9
:10BE20000C4673B98B6863B9C96851B91248FFF7FA
:10BE30002BFF95F8A51005F12C00BDE8704080F0AF
:10BE400083BA95F8A5100D4880F0CEF848B906F1F0
:10BE5000080120461CF018FC18B107480221FFF722
:10BE6000F3FE95F8A51005482246BDE8704080F025
:10BE70005FBA00BFD0B300201CCC0020FCB3002070
:10BE800008B50721FFF7E0FE80ED0A0A08BD0000B3
:10BE900008B50368032B23D1D0ED057A9FED127A04
:10BEA000F0EEE77AF4EEC77AF1EE10FA1AD50F4BFE
:10BEB00090ED090A03F5C663D3ED007AF8EEE77A50
:10BEC00037EEC00A36F07CFFDFED097AB0EEC00A2B
:10BED000B4EEE70AF1EE10FA94BF0120002008BD8D
:10BEE0000120FCE70020FAE700000034D0530020D6
:10BEF0000000484330B50368023B85B00446082B78
:10BF00006FD8DFE803F0050D30374D634163630000
:10BF1000FFF74AFE84ED090A94ED090A05B030BD29
:10BF2000D6F0F0FDE369DFED320AE061C31A07EEF7
:10BF3000903AF8EE677A94ED050A67EEA07AD4EDB0
:10BF4000060AF12020EEA71A67EEE00A36F09AFF03
:10BF5000D4ED057A77EEC07AC4ED057AD4ED097A8E
:10BF600037EE800AD6E7FFF72DFEDFED227A20EECE
:10BF7000270ACFE7204B03F59163D3ED007AF8EE63
:10BF8000E77AC0ED097AC7E71C4DD5F8A00FC8F0D5
:10BF9000F1FD0028C0D0D5F8A03F1B6C6362BBE761
:10BFA000D6F0B0FDE3699FED127AD4ED0A6AE06144
:10BFB000C31A07EE903AF8EE677A67EE877A94ED47
:10BFC000097AA6EEA77A84ED097AA5E70B4B9FEDD7
:10BFD0000C0AD3F88C0F6C303CF058FB84ED091A36
:10BFE0009AE7064BD3F8943FD3F85033D6E700BF17
:10BFF0006F12833A0000C842D0930020D0A30020E3
:10C000009F0CB3450368092B08D8DFE803F0050A45
:10C0100005050505070705100023836290ED0A0A50
:10C020007047044BD3F8943FD3F85433F5E7C36A11
:10C03000F3E700BFD0A30020F0B5304D2DED028B0B
:10C040000446D5F83C04036889B0D3F880300E4626
:10C05000984700283FD0D5F83C0403F0AFFB05F526
:10C06000805708EE100AD7F8943FD7F88C0FD3ED1D
:10C07000D28A0368D3F898309847D7F8943FD5F818
:10C080003C0493EDD31A03688DED041A78EEC00AD0
:10C090009B6CCDED050A98470390D5F83C040268E7
:10C0A000D26C9047B8EEC88A9FED150A0090039BAA
:10C0B0009DED041ADDED050A28EE000A324607A9B7
:10C0C000A5F18C00C7F06CFA48B10A212046FFF7B1
:10C0D000BBFD079BA36209B0BDEC028BF0BD2368DA
:10C0E0000A2BF8D161680023A362204611B9FFF73B
:10C0F000CBFDF0E7FFF7A8FDEDE700BFD0930020F0
:10C100000AD7233CF8B50023264FCB6297F8553465
:10C11000254E13F0010F04460D4637D1D7F83C04E5
:10C1200003685B6F984788B3D7F83C0403F0B2FE0E
:10C13000DFED1E7A85ED0B0AB0EEC00AB4EEE70A19
:10C14000F1EE10FA03D409213046FFF77DFDD5ED5D
:10C150000B7AFDEEE77A284617EE903A19B2FFF710
:10C160006BFF1148FFF7C6FE0F4884ED000AFFF78A
:10C1700049FF336884ED010A0A2B0FD8DFE803F08A
:10C180000C1010101010100C100C0C003368092B40
:10C19000DDD105480021D8E70223A3602046F8BD81
:10C1A0000123FAE7D09300201CCC002000000034CB
:10C1B000034B01221A6000229A60DA601A6170470C
:10C1C0001CCC002013B501A9044610F04DFA04F56B
:10C1D000004320B9012283F8D52002B010BDDDED67
:10C1E000017ADFED086AB8EEE77AD3ED327A67EECE
:10C1F000A67AB4EEE77AF1EE10FA54BF01220022DB
:10C20000E9E700BF0000C84210B5044600F50B4046
:10C21000A8F03CF904F50C403030BDE81040CFF0F8
:10C2200009BA000008B509480F2203F06BFC60B999
:10C2300006480F22062103F065FC30B9BDE808402E
:10C2400002480F22092103F05DBC08BDD033002055
:10C2500070B5154E96F85534DA0604460D4622D5CB
:10C260006FF3041386F85534A6F500566FF02AF9DB
:10C27000002214216EF0D8FE96F864300E2B12D1F5
:10C28000022D0AD0032D0AD0012D0CD194F85410A0
:10C290002046BDE87040FFF7C5BF0621F8E794F8D7
:10C2A00054100329F4D070BDD093002010B50E4C6B
:10C2B00049B9D4F83C0403681B689847A0F11303FC
:10C2C0005842584110BDD4F83C0403681B68984795
:10C2D0001328EED00E221321A4F5C04003F012FC67
:10C2E0000028E6D1EEE700BFD093002030B50D4620
:10C2F00089B01146FFF7DAFF0446F0B104A81BF03D
:10C30000ABFF14F019FC04A914F030F928B1286926
:10C31000059B8342D4BF002001209FED137A134B6D
:10C320008DED017AD3F8982F8DED027A40B1D36963
:10C3300003930F4801A907F093FA204609B030BDD6
:10C34000A3F54051D2ED087AD3F8642FD1F86832C2
:10C35000F0EEE77AF1EE677A9A42B8BFF0EE477AEC
:10C36000CDED037AE5E700BF00000000D0A3002078
:10C3700000C90020F0B50F4685B011460646FFF70C
:10C3800095FF044658B1002501AA3946304601956B
:10C3900002950395CFF05AFA044618B900242046B6
:10C3A00005B0F0BDDDED017A9FED177A0395F0EE53
:10C3B000E77AF4EEC77AF1EE10FA08D5DDED027AED
:10C3C000F0EEE77AF4EEC77AF1EE10FAE6D401A8BF
:10C3D0003CF07CFD01A83CF0C1F90C4B9DED017ACD
:10C3E000D3F8983FDDED027AD3ED066A084827EED0
:10C3F000267A67EEA67A01A98DED017ACDED027A53
:10C4000007F02EFACBE700BF00000034D0A30020D5
:10C4100000C9002070B52DED028B0E4684B0114688
:10C420000546FFF743FF044680B39FED238A01AA28
:10C43000314628468DED018A8DED028A8DED038A05
:10C44000CFF004FA044608B31C4B9DED017AD3F8F3
:10C45000982FDDED027AD2ED066A27EE267A67EE96
:10C46000A67A8DED017A9DED037ACDED027AB4EED8
:10C47000C87AF1EE10FA0EDDD2ED077A67EE877A10
:10C480000F48CDED037A01A907F0EAF9204604B080
:10C49000BDEC028B70BDD2ED087AD3F8642FA3F502
:10C4A0004051F0EEE77AD1F8683267EE877A9A4227
:10C4B000B8BFF0EE487AE3E700000000D0A3002008
:10C4C00000C900202DE9F0413D4F97F8553414463E
:10C4D000DA060646884616D4D7F83C0443F0100323
:10C4E00087F8553403681B689847012586F854007F
:10C4F000D7F83C0403681B689847092805D1002435
:10C500002046BDE8F0810025F2E7D7F83C04036837
:10C510001B6898471228F2D0D7F83C0403681B68C0
:10C5200098470E28EBD0012C12D8062C38D801A33E
:10C5300053F824F001C50008A1C5000893C5000800
:10C54000A7C50008B3C5000869C5000889C500086B
:10C550001C4801F08DFE0028E7D01B4801220A216B
:10C56000FAF770FA00241BE0002DC9D00E22062134
:10C57000144803F0C7FA00B900246EF0A3FF224666
:10C5800014216EF051FDBBE7002DB9D00E2205211C
:10C59000EEE72A4641463046FFF7A8FE0028E1D0E4
:10C5A000002DADD0E9E72A4641463046FFF7E2FECE
:10C5B000F4E72A4641463046FFF72CFFEEE700BF7E
:10C5C000D0930020D0330020B09400202DE9F04F0C
:10C5D0002DED068B00F5804300F5105993F9D2320A
:10C5E0008DB0054600F5004409F1300933B100F57E
:10C5F000C048D8F8603493F8D5707FB90021A4F80A
:10C60000941C484614F034FD94F8951C48460DB02F
:10C61000BDEC068BBDE8F04F14F034BDD6F072FAD5
:10C6200005F5E04B0190DBF8940F9FED968A90EDB5
:10C63000E4AAC4F0F9FF09AE002800F0CE80DBF8D0
:10C64000943F03F5657393E8070086E807003046DA
:10C650008DED0B8A3CF03AFCB0EE409A284610F083
:10C66000B5F905F5FE4A0AF1700A002800F0B88015
:10C670005046CAF0D3FC07C886E8070030468DED67
:10C680000B8A3CF023FCF0EE409AD8F83C04036897
:10C690001B689847122840F0AC80002384F8943C33
:10C6A000D8F83C0403685B69984738B105F5A043A6
:10C6B000D3F8C43FB3F90830002B0DDC98F93034BF
:10C6C000002B09DA019BC4F8983C5046CAF0A2FC42
:10C6D00004F69C4383ED000A94F8943C5BB1019B03
:10C6E000D4F8980C181A41F28833984240F28F809F
:10C6F000002384F8943CDBF88C0F9FED630A6C30C8
:10C700003BF0C4FF8DED090ACDED0A0A8DED0B1A41
:10C7100096E8070006AB03AE9FED5C0A83E80700CE
:10C7200086E8070030463BF0B1FF2846B0EE408A6D
:10C73000F0EE608A8DED060ACDED070A8DED081A40
:10C7400010F044F9002874D0DFED517AF4EEE79A46
:10C75000F1EE10FA94BF01250025DBF8940FC4F028
:10C7600063FF30B1DFED4A7AB4EEE79AF1EE10FAEA
:10C7700009D9002D64D1D8F83C0403681B68984798
:10C78000022864D00027DBF8940FC5F07BF805463B
:10C79000002873D0B5EEC0AAF1EE10FA6DD5DFED2A
:10C7A0003D7AB4EEE7AAF1EE10FAACBF01260026FE
:10C7B0005046CAF03BFC5EB9DFED377AB0EEC00AF6
:10C7C000B4EEE70AF1EE10FA5AD8002D08BF0027A0
:10C7D00094F8941C84F8957C13E7B0EE489A3DE7F2
:10C7E000284610F0BBF800287FF442AFDFED259A11
:10C7F0004BE7D8F8603493F8D530002B3FF450AFB6
:10C8000098F93034002BBFF64BAF012346E7504672
:10C81000CAF000FC04F69C43D3ED007A30EE670AC0
:10C82000DFED1E7AB4EEE70AF1EE10FA3FF760AFE3
:10C8300061E7284610F092F80546002884D18CE77D
:10C84000DBF8940FC4F0F0FE002894D19BE7B0EE23
:10C85000680A37F17FF8F0EE408AB0EE480A37F107
:10C8600079F8DFED0F7A20EE280AB4EEE70AF1EE50
:10C8700010FACCBF0127002785E700252E4697E751
:10C880003746A5E7000000009F0CB345D3023739B7
:10C890000000FA420000C8C2000070420000484296
:10C8A00055CF7D3F38B5044610F090F804F510558B
:10C8B000303548B9204610F051F8014620B92846D5
:10C8C000BDE8384013F066BD04F5C044D4F83C041C
:10C8D00003689B6C984720B9D4F83C040368DB6C70
:10C8E00098470146EBE7000030B5044689B068463A
:10C8F00004F510551BF0B0FC303504A81BF0ACFC5F
:10C900006946284613F032FEA0B104A9284613F068
:10C91000F7FE78B1059B019323680022D3F8B0306D
:10C9200069462046984728B104F5B74001213C30BC
:10C93000CFF05CFD09B030BD00F5005292F8AC2696
:10C94000D2070CD400F5C042D2F8602492F8D5107A
:10C9500009B1FFF7C9BF0368D3F8AC301847704777
:10C9600030B587B0044602A801911BF075FC04F5B0
:10C97000105002A9303013F0F9FD019A18B90025C2
:10C98000284607B030BD236802A9D3F8B03020464E
:10C99000984705460028F2D004F5B74001213C3005
:10C9A000CFF024FDECE70000F0B5044685B004F5B7
:10C9B0001056684630360F4615461BF04DFC69464A
:10C9C000304613F09DFE10B9002005B0F0BD394689
:10C9D000304613F051FC0028F6D0002DF5D004F5B8
:10C9E0000054284694F8AC3643F0020384F8AC3681
:10C9F000EBE700002DE9F04F2DED0A8BBDB00446AA
:10CA000024220D4618A8002139F100FD242200211E
:10CA100021A839F1FBFC242200212AA839F1F6FCD7
:10CA200004F5C0462422002133A839F1EFFC00238D
:10CA3000CDE90D330F9396F8313413F008082FD158
:10CA400004F5A04943F0080399F8B82F079286F837
:10CA500031341DF031F890F9253023B390F8443388
:10CA60000BB304F63C1738461CF01CFFC34694F881
:10CA700062395FFA8BF18B421FD938461CF0F0FE09
:10CA80000BF1010B82460028F1D1CE4A0221284643
:10CA900075F030FE96F831346AF3C30386F831340A
:10CAA0004FF0010852E3C84A0221284675F022FEE1
:10CAB00096F831346FF3C303F0E704F5C1436033F4
:10CAC000012118460BEE903AF9F732FD824608B97B
:10CAD000BE4ADBE720460FF025FCD9F8C43FB3F986
:10CAE0000890B9F1000F01D0B94ADDE796F930346A
:10CAF000002B09DBB74A0221284675F0FBFD96F8AA
:10CB0000313469F3C303C9E7204601F0C7FE04F5D9
:10CB1000C9430C3318464A460CA90CEE103A17F0DC
:10CB200065FB002814BF022301230393F123CDE901
:10CB300013398F210A23CDE9003113AA287CADF8DF
:10CB4000549003234D2173F0B5F9A34B9FEDA38AB5
:10CB500001225A720621A24A284675F0CBFD039B9A
:10CB6000022B0CBF9F4AA04A0621284675F0C2FD41
:10CB700004F580434FF0000983F88E924946384609
:10CB80001CF0DAFD94F862395FFA89F18B420CD916
:10CB900013AA38468DED138A8DED148A8DED158A12
:10CBA00009F101091CF04CFCECE738461CF07AFE58
:10CBB0004FF0000A4FF07C0B94F862295FFA8AF973
:10CBC0004A4519D9494638461CF018FAC0B20BFB41
:10CBD00000403CAA0C2300F51D6003FB092C07C88C
:10CBE000ACF1900C8CE807003CAA02EB890909ED36
:10CBF0002F8A0AF1010ADFE741F288310AA831F0F1
:10CC00004FFAD6F860049FED759A03689FED77AAF6
:10CC10009B6ADFED77AA9847D6F860040121CBF034
:10CC200053FD744B1B680293D86A036801211B688B
:10CC30009847D5F067FF0590D5F064FFF0EE499A6C
:10CC40000690002604F5A049079A99F8B83F934248
:10CC500040F0D88094F8821C38461CF001FE002871
:10CC600000F0D08004F5C04BDBF8603493F8D53089
:10CC70000493002B00F0C68041F288310BA831F0FC
:10CC80000FFAD5F03FFF059BC01A132840F2D98058
:10CC9000D5F038FF059020460FF044FB7EF01AF9DE
:10CCA00082467EF07BF8D9F8C43FDBF86004B3F924
:10CCB000083000EE103AB8EEC00A20EE0A0ACDF0B5
:10CCC0005DFB50467EF072F838461CF0EBFD1CEE22
:10CCD000100A17F0E1FCD9F8C43FDFED400AB3F9C0
:10CCE000083000EE103AB8EEC00AA22020EE0A0A80
:10CCF000B7EE001A36F0C6F8B4EEE90AF1EE10FA13
:10CD00001CEE100A4FF000020CA958BFF0EE409A3A
:10CD1000F0EE408A17F06AFA08B900230C939DEDF3
:10CD20000C8ADFED357AB4EE498AF1EE10FAF4EEB2
:10CD3000E78A48BFB0EE498AF1EE10FA80F28F80A0
:10CD40009FED2E9ADFED2E8A4FF0000A94F862399B
:10CD50005FFA8AFB5B4540F296814FF00C0918ABF5
:10CD600009FB0BF903EB0900B0EE490A3BF08EFC1E
:10CD700059463846CDED110A8DED121A8DED100A87
:10CD80001CF03CF97C23C0B203FB0040B0EE680A03
:10CD900000F51D603BF07AFC3CAB13A910A8994448
:10CDA0008DED130ACDED140A8DED151A3BF042FC02
:10CDB0000AF1010A09ED240A49ED230A09ED221AB4
:10CDC000C4E700BFCD161508BC161508E3331508D7
:10CDD000DB161508ED161508EDCE0020000000004A
:10CDE000F81615080D17150857B314086F12833A73
:10CDF0000000C84210CC002000000034A4707D3F29
:10CE00000AD7233C04F5C049D9F8600403689B6A3B
:10CE10009847D9F860040021CBF056FC029BD86AF1
:10CE2000036800211B689847002E40F05F81284668
:10CE3000C94A052175F05EFC314638461CF07CFC81
:10CE400070E1029B986A036805215B6898470BA80C
:10CE500031F032F9B0EE498AB0EE489AF2E64FF07E
:10CE600000094FF00C0B04F67C1A94F862295FFA63
:10CE700089F39A4222D91946384608931CF0BEF825
:10CE8000089B0BFB03F13CAB5A18A2F16C034FF06B
:10CE90007C0CC0B2CDE908320CFB00A018AB1944E1
:10CEA00054303BF0DDFB089B099A09F1010902EDC2
:10CEB0001B0AC3ED010A83ED021AD6E7039B012B7F
:10CEC0004FF0000A46D19FEDA5BA9FEDA59A4FF00D
:10CED0000C0B94F862395FFA8AF6B34240F286800E
:10CEE0000BFB06F63CAB03EB0609A9F148030893DC
:10CEF00021ABB0EE680A98193BF0D8FB089B09ED0E
:10CF0000120AC3ED010A83ED021A33ABB0EE4B0AED
:10CF100098193BF0BBFB2AAB98198DED100AB0EEC7
:10CF2000490ACDED110A8DED121A3BF0AFFB13A9A2
:10CF300010A88DED130ACDED140A8DED151A3BF0F6
:10CF40008FFB0AF1010A09ED090A49ED080A09ED0A
:10CF5000071ABEE79FED819A9FED81BAF0EE088A2D
:10CF600094F862395FFA8AF94B4564D99DED0C0A51
:10CF7000B4EEE80AF1EE10FA35DB0C2303FB09F9F5
:10CF80003CAB03EB090621AB03EB09003BF08EFB46
:10CF900033AB46ED110A06ED101A06ED120A03EB4B
:10CFA0000900B0EE490A3BF071FB2AAB03EB090024
:10CFB0008DED100AB0EE4B0ACDED110A8DED121A6F
:10CFC0003BF064FB13A910A88DED130ACDED140AF4
:10CFD0008DED151A3BF044FB06ED090A46ED080AF3
:10CFE00006ED071A049E0AF1010AB9E74FF000099D
:10CFF0004FF00C0A94F862395FFA89F6B34241D9CE
:10D0000033AB0AFB06303BF061FF1BEE900AF0EEFB
:10D01000408ABBF095FA07EE900AB8EE677A3CAB0F
:10D02000C8EE877A03EB860609F1010967EEAA7A52
:10D0300046ED2F7ADEE74FF0000A4FF00C0B94F824
:10D0400062395FFA8AF94B451DD933AB0BFB0930C6
:10D050003BF03CFFC8EE297A0AF1010A1BEE900A68
:10D0600067EE808ABBF06CFA07EE900AB8EE677A3A
:10D070003CABC8EE877A03EB890967EEAA7A49EDE3
:10D080002F7ADCE7049ED5F03DFD069BC01AB0F573
:10D09000FA7F27D9D5F036FD04F5A043DDED0D7AF2
:10D0A000D3F8C43F0C9A1B891392FCEEE77A339AAB
:10D0B0001492ADF85C30349A159217EE903A359A86
:10D0C0001692ADF85E30F0221423CDE90032B12182
:10D0D000069013AA287C72F0EDFEAAF069FB297C69
:10D0E000AAF01CFA0BA830F0E7FFB5E60399384622
:10D0F0001CF022FB00264FF00C0A94F86239F1B2C2
:10D100008B4207D933AB0AFB013238461CF098F941
:10D110000136F2E738461CF0A5F9124A06212846E6
:10D1200075F0E8FA104B002520465D7201F0A8FB6F
:10D1300004F585400E3061F0DBFC99F8313465F37D
:10D14000C30389F831340AA830F0B6FF40463DB039
:10D15000BDEC0A8BBDE8F08FC1A41708A4707D3F19
:10D160000AD7233C15171508EDCE0020F0B5544F13
:10D17000D7F8503FDA0785B0044600F19F8000F5EC
:10D18000C045D5F8603493F8C120002A40F096805D
:10D1900093F8D530002B00F08E8095F93034002BB9
:10D1A000C0F2898000F5004393F8A03C002B40F0CA
:10D1B000858000F5E0469FED430AD6F88C0F6C3071
:10D1C0003BF064FACDED020A60EEA00ADFED3E7A94
:10D1D0008DED010AE0EE000A8DED031AF4EEE70A88
:10D1E000F1EE10FA67DCD6F88C3F9FED387AD3ED7C
:10D1F000377AF4EEC77AF1EE10FA04D5D5F8603438
:10D200001B7A002B57D0B5EE007AF4EEC77AF1EE18
:10D2100010FA50D404F5FE407030C9F007FFDFED7E
:10D220002C7AB4EEE70AF1EE10FA44D8D6F88C3F27
:10D230009FED287AD3ED367A67EE877AB3EE0E7AD1
:10D24000F4EEC77AF1EE10FA35DA234AB4F9DC12BB
:10D25000138801339BB2138019B9B4F8DA12A4F819
:10D26000DC12B4F8DC12994228D8002616806EF041
:10D2700029F9012219216DF0D7FED5F86004036861
:10D280005B699847431C04F5C340144A3146483053
:10D2900071F064FDD5F86034012283F8C120D7F81D
:10D2A000503F5B070AD504F5DA501C3005B0BDE8E5
:10D2B000F04098F00FB9084B00221A8005B0F0BD7D
:10D2C000D08300209F0CB3454054094A6666663FF0
:10D2D000000000B4E02E654256CC00202C17150843
:10D2E000F0B52DED028B4B4BD3F8503F9B0785B02B
:10D2F00004461FD400F5E046DFED478AD6F88C0FD0
:10D3000003681B699847D0ED017AF4EEE87AF1EEF4
:10D3100010FA0FDB04F5C04304F50C45D3F8602484
:10D3200092F8C110A43549B1002303A928460393FC
:10D3300070F082FE05B0BDEC028BF0BD92F8D520F6
:10D34000002AF1D093F93034002BEDDB04F50047CF
:10D3500097F8A03C002BE7D1D6F88C0F03681B6927
:10D360009847D0F8B030D6F88C0F039303681B6948
:10D37000984704F5547200F1B001284670F07EFF22
:10D38000DDED037AB0EEC08AF0EEE77AF4EEC87A0B
:10D39000F1EE10FA03D503A9284670F04DFED6F839
:10D3A0008C0F03681B699847D0ED040AF4EEE80A75
:10D3B000F1EE10FABEDBF6EE087A60EEA77AF4EE34
:10D3C000C87AF1EE10FA1DD5D5F09CFBD7F8B03C29
:10D3D00042F21072C31A9342ACD9DFED107AC7F84B
:10D3E000B00C68EE277A04F5C34417EE900AF7F7FD
:10D3F000C9F84834CDE90001094A0021204671F0FE
:10D40000ADFC97E79DED030A35F018FC0028DBD151
:10D4100090E700BFD0830020000000340000C84225
:10D420004817150810B5044600F501401C308EF071
:10D4300009FD04F501400121BDE810403C309EF09B
:10D4400053BE00002DE9F04100F50046044696F970
:10D450001C314BB300F5C04596F8302195F83034B7
:10D46000DB43C3F3C01363F3C30200F5014700F5C8
:10D47000FE4086F830217030C9F0D8FDDFED3F7AEC
:10D480001C3720EE670A38468EF05CFD96F8A03C0B
:10D4900053B938468EF002FDD5F8603493F8D53094
:10D4A00023B9374B00221A80BDE8F08196F830315D
:10D4B000DB07F9D4D5F83C0403689B6B9847002838
:10D4C000EFD095F93034002BEBDB2D4D2B8804F594
:10D4D000E0484BB9B6F9223133B1642213FB02F3B1
:10D4E000D8F8642F9A42DFDB38468EF047FDD8F833
:10D4F0008C3F9FED247AD3ED367A67EE877AB3EED0
:10D500000E7AF4EEC77AF1EE10FA05D82B88002BCC
:10D51000CAD0013B2B80C7E7B4F9DC321BB9B4F8A1
:10D52000DA32A4F8DC322B88B4F8DC22B4F9DC025D
:10D53000154993423CBF01332B802B88D8F83C2FF0
:10D54000012B01D10A60AFE709689142A9DD18B942
:10D55000B4F8DA22A4F8DC22B4F8DC229A42A3D888
:10D5600000232B806DF0AEFF02220C216DF05CFDDC
:10D570002046BDE8F041FFF755BF00BF0AD7233C66
:10D5800054CC0020E02E654250CC002008B500F5B8
:10D59000004393F91C217AB300F5C04292F930247C
:10D5A000002A0EDA00F5C340144A0621483071F013
:10D5B000D5FB6DF087FF0322BDE808400F216DF019
:10D5C00033BDB3F922319BB100F5E0426421D2F8BA
:10D5D000642F13FB01F39A420ADA00F5C340084AAC
:10D5E0000121483071F0BAFB6DF06CFF0222E3E7D5
:10D5F000BDE80840FFF716BF08BD00BF601715085B
:10D600007217150870B52DED028B00F5C0455B4E05
:10D61000D5F8603493F8D5308CB0044643B195F911
:10D620003034002B04DB00F5804393F9AA322BB988
:10D63000002333800CB0BDEC028B70BD00F50043BD
:10D6400093F8A03C002BF3D101F090FB00287BD194
:10D65000D5F83C0403689B6B98470028E8D004F594
:10D66000FE40403070F03EFD3BF030FCF0EE087ABA
:10D67000B4EEE70AF1EE10FAF0EE408AD8DA04F5DB
:10D680001053D3ED9F7A93ED9E0A20EE270A36F1D0
:10D6900075FBDFED3B7A20EE270AB2EE0E7AB4EE90
:10D6A000C70AF1EE10FAC3D904F5E043D3F88C3F72
:10D6B00093ED368A28EE278AF3EE0E7AB4EEE78AE7
:10D6C000F1EE10FAB4D904F51050002309A9303056
:10D6D00009930A930B9313F01FF800283DD1338868
:10D6E000B4F9DC2201339BB23380002A40D0B4F875
:10D6F000DC22B3EB420F9DDB6DF0E4FE01220C2136
:10D700006DF092FC1F4B002218EE900ACDE9062323
:10D71000F6F738FF1C4BCDE90401002218EE100A81
:10D72000CDE90223F6F72EFF04F5C3444834CDE9D2
:10D730000001164A2046002171F010FB01220C2145
:10D740001348F9F77FF975E7D5F83C040368DB6CFB
:10D75000984700287FF47CAF6AE709A83BF0B6FB46
:10D76000F2EE047AB4EEE70AF1EE10FAB7DB5FE707
:10D77000B4F8DA22A4F8DC22B9E700BF4CCC0020D0
:10D78000E02E65420000084000003E408817150862
:10D79000B0940020F0B52DED028B8BB000230793E1
:10D7A0000893099305AB0446019300F5105007ABAD
:10D7B000009302AA04AB03A9303012F01BFE04F55B
:10D7C000C046054686F8BC0128B9002528460BB09E
:10D7D000BDEC028BF0BDD5F089F9D6F8C0319FEDD4
:10D7E000337AC31A07EE903AF8EE677A074667EE87
:10D7F000877A04F5C34006AA02A91830CDED067A4F
:10D8000070F03CFD04F5C34006AA03A924308DED59
:10D81000020A70F033FD04F5C34006AA04A93030B3
:10D820008DED030A04F5804470F028FDC6F8C07140
:10D8300094EDAB8AB5EEC08AF1EE10FAC5D9DDEDF4
:10D84000080A9DED070A36F10BF9DDED090A36F1FC
:10D8500007F9D6F84021DDED037AB4EEC08AF1EE87
:10D8600010FA94BF012300231AB196F84421D2077D
:10D8700012D438EE087AB4EEE77AF1EE10FA0BD84B
:10D880000233DBB2DDED027AB4EEE78AF1EE10FA94
:10D8900009D8002B99D099E7B4EEE78AF1EE10FA97
:10D8A000F0D80133EDE7012B90D88EE7BD378635F0
:10D8B00070B500F5C045044695F8553443F00403AF
:10D8C00085F855346DF0FEFD012211216DF0ACFBA1
:10D8D000D5F8603493F8D530002B43D0D5F83C040C
:10D8E00003681B68984709280AD1204609F06EFB97
:10D8F00030B104F512409030BDE8704009F04EBBE5
:10D90000194BD3F83C0403681B69984704F580431E
:10D9100040B993F9A932032B24D10621204609F0FE
:10D9200041FB0DE093F9A9120229F6D195F855347F
:10D93000DB07F2D40622204602F0E4F80028ECD0FF
:10D940000A4BD5F83C0401225A7303681B6C9847B4
:10D95000034604F5C340064ABDE870400221483042
:10D9600071F0FCB970BD00BFD0930020EDCE002057
:10D97000BC17150808B500F5C04292F85534590790
:10D9800017D56FF3820382F855340A4B5A7B42B1A4
:10D99000002200F5C3405A730221074A483071F053
:10D9A000DDF96DF08FFDBDE80840002211216DF01A
:10D9B0003BBB08BDEDCE0020E0171508F0B50546CD
:10D9C00085B005F51057684630371AF045FC6946B2
:10D9D000384612F095FE80B105F58043D3EDAB7A61
:10D9E000374CF5EEC07AF1EE10FA08D8354A00232C
:10D9F00028462380D373FFF7BDFF05B0F0BD28464E
:10DA0000FFF7C8FE064628460EF0A8FF10B92846C4
:10DA10000EF07EFFA378002E18BF00200343DBB278
:10DA2000A370002BE9D06378A8BB83BB23780133B4
:10DA3000DBB2082B237003D14EB3384612F060FDE1
:10DA40002378092B02D1384612F052FD2378092B96
:10DA50001DD94FF4857323806DF034FD022210210F
:10DA60006DF0E2FAD5F04EF86368C01A47F2305311
:10DA7000984209D905F5C340134A0221483071F094
:10DA80006DF9D5F03FF860602846FFF711FF0D4BA8
:10DA90006278DA73B1E72678002EF8D0013EF6B24C
:10DAA0002670002BF3D0002EF1D166706DF00AFDC8
:10DAB000324610216DF0B8FA2846FFF75BFFE6E723
:10DAC00058CC0020EDCE0020F817150800F5C04313
:10DAD00093F855345B0701D5FFF7EABE70470000A5
:10DAE00073B5044600F5105001A9303004F5C04567
:10DAF00012F0B8FAD5F88431834206460CD004F50A
:10DB0000E043D3F88C0FC2F025FBC5F884616DF0BB
:10DB1000D9FC3E216DF068FA04F5005695F988119C
:10DB200096F9402796F8403791421BD0FF2B19D029
:10DB300004F5E043D3F88C0FC2F00CFB96F84037A5
:10DB400085F888316DF0BEFC95F8882118216DF0BC
:10DB50006BFA04F5C34095F98831034A0421483033
:10DB600071F0FCF802B070BD081815082DE9F043FB
:10DB70008FB00546D4F0C6FF0023059306930793A4
:10DB8000089309930A930B930C930D9305F5105882
:10DB900004AB019308F1300803AB009306460BABCE
:10DBA00008AA05A9404612F003FCDFED487A9DED76
:10DBB000077AB4EEE77AF1EE10FA074632DB9DED14
:10DBC0000A7AB4EEE77AF1EE10FAACBF0124002431
:10DBD00005F5C049404699F8BC31002B08BF002725
:10DBE00012F0FAFB8046FFB9444605F5A04393F9CD
:10DBF000E83E012B29D164B1D9F8603493F8D540BF
:10DC00003CB1D9F83C0403685B69984780F0010097
:10DC1000C4B299F88C31CBBBCCB9C9F890610FB0C4
:10DC2000BDE8F0830024D3E7002CDDD005F5C34028
:10DC3000243070F0FFF990ED007AF7EE007AB4EE40
:10DC4000E77AF1EE10FAD0DCCEE70024E1E7D9F86C
:10DC50009001301AB0F57A7FE1D9C9F894310124E6
:10DC600005F5E04389F88C41D3F8943F83F84844A4
:10DC70006DF028FC22461D216DF0D6F9144A05F5F9
:10DC8000C3400221483071F069F8C8E714B1C9F8FF
:10DC90009461C4E7D9F8940143F69823361A9E425A
:10DCA000BDD905F5E043C9F8904189F88C41D3F816
:10DCB000943F83F84844C9F894416DF003FC224630
:10DCC0001D216DF0B1F9034AD9E700BF000000340F
:10DCD000201815083A1815080B4B10B501220446F8
:10DCE0005A72D4F00FFF04F50042D2F88C3CC31AEC
:10DCF000142B08D9C2F88C0C04F50F502030BDE865
:10DD000010405AF0ABBB10BDEDCE00202DE9F7431B
:10DD1000044604F5C04600F58540002324300DF18B
:10DD200007018DF8073061F019FED6F8600490F90C
:10DD3000C030026883B3083BDBB2012B95692BD955
:10DD40003221A84704F1100017F010F9204B04F518
:10DD5000C3481F684FF0000908F14808F86A0368D3
:10DD6000DB69984701281ED1D4F0CCFE41F28733FD
:10DD7000A0EB09029A42054605D9164A06214046FB
:10DD800070F0ECFFA9462046FFF7A6FFB86A0368CB
:10DD900003215B689847E1E704F580439269B3F893
:10DDA000B8129047CEE70121D6F86004CAF08CFC87
:10DDB000D6F860040368DB6A98477CF069FBF86A70
:10DDC00003681B68012103B0BDE8F043184700BF9A
:10DDD00010CC00205818150870B5044600F5C34053
:10DDE0002DED028B184A194E9FED198A06214830F5
:10DDF00070F0B4FF2046FFF789FF2046FFF76CFF65
:10DE000020460EF08FFA3368986A036803215B6836
:10DE100098477DF05FF805467CF0C0FF04F5A0430D
:10DE2000D3F8C43FB3F9083000EE103A04F5C0430C
:10DE3000B8EEC00AD3F8600420EE080ACCF09EFACF
:10DE400028467CF0B3FFD8E77C18150810CC0020DA
:10DE50006F12833A2DE9F047044600F5C3402DEDDB
:10DE6000028B2A4ADFF8AC900621483070F076FF2A
:10DE70002046FFF74BFF7DF02DF804F5C046054620
:10DE80007CF08CFFB7EE000AD6F86004CCF076FA8E
:10DE900028467CF08BFFD4F035FE41F2873A0746E6
:10DEA000D4F030FEC01B5045D9F8008017D99FED43
:10DEB000188A28467CF072FFB0EE480AD6F8600453
:10DEC000CCF05CFA28467CF071FF2046FFF704FF97
:10DED000D8F82800036803215B689847E9E72846DB
:10DEE0007CF05CFFB7EE000AD6F86004CCF046FA8E
:10DEF00028467CF05BFF2046FFF7EEFED8F82800AE
:10DF0000036803215B689847CAE700BFAC1815088F
:10DF10000000000010CC0020F7B500F5C043044617
:10DF2000D3F8603493F9C030032B2BD0374E6525DE
:10DF300000F50047013D15F0FF050CD0D7F8883CEF
:10DF40004BB93368986A036814215B689847204688
:10DF50000EF0E8F9EEE704F5C14001216030F8F772
:10DF6000E7FA04F5804393F9A43268B953B1092B59
:10DF700008D08DF8070004F585400DF10701243025
:10DF800061F0ECFC03B0F0BD032B38D8DFE803F000
:10DF90000227313404F5A043D3F8C43FB3F9082075
:10DFA00040F2B5339A422CDD04F5854001250DF190
:10DFB000070124308DF8075061F0D0FC04F5C34010
:10DFC000134A0221483070F0C9FE124B5D720F4BAC
:10DFD0001C68A06A036805215B689847F9E704F5A7
:10DFE000A043D3F8C43FB3F9082040F2B5339A42B6
:10DFF00007DD2046FFF7F0FE2046FFF72BFF092B39
:10E00000C0D000238DF80730B5E700BF10CC00204A
:10E01000D0181508EDCE002000F5C3400B46024A8B
:10E020000421483070F09ABEF018150810B5044667
:10E030006DF048FA002205216CF0F6FF04F5C340AC
:10E04000034ABDE810400421483070F087BE00BF8D
:10E05000FC18150813B50B464AB100F5C3400092F1
:10E060000421054A483070F079FE02B010BD02B0BC
:10E07000BDE81040FFF7D0BF1419150808B500F52A
:10E08000C340064A0421483070F068FE6DF01AFA69
:10E09000BDE80840002208216CF0C6BF2819150809
:10E0A00038B504460D46D4F02DFD04F5C0433DB906
:10E0B000D3F84C24C3F850040AB9C3F84C0438BD53
:10E0C000D3F85024801A642882BF0022C3F8502459
:10E0D000C3F84C24F3E7000037B5044600F5FE40D2
:10E0E0007030C8F089FF04F5C042C0F3803592F863
:10E0F0003234C3F34001A9421DD065F3410304F556
:10E10000C34482F8323448346DB16DF0DBF9022239
:10E110000B216CF089FF094A0221204603B0BDE8BB
:10E12000304070F01BBE6DF0CDF92A460B216CF02B
:10E130007BFF034AF0E703B030BD00BF401915086C
:10E140005C19150838B50A460C460621054601F04B
:10E15000D9FC28B1054A137843F00803137038BD81
:10E1600021462846BDE8384008F01CBF0CCF0020EF
:10E1700038B50A460D461521044601F0C3FC28B106
:10E18000094A137843F00803137038BD04F5C340FF
:10E1900004214830054A70F0E1FD29462046BDE8DB
:10E1A000384008F0FFBE00BF0CCF00206C191508E6
:10E1B00038B50A460D461521044601F0A3FC28B1E6
:10E1C000094A137843F00803137038BD04F5C340BF
:10E1D00004214830054A70F0C1FD29462046BDE8BB
:10E1E0003840FFF7AFBF00BF0CCF002094191508CF
:10E1F00038B50A460D461B21044601F083FC28B1C0
:10E20000094A137843F00803137038BD04F5C3407E
:10E2100004214830054A70F0A1FD29462046BDE89A
:10E220003840FFF78FBF00BF0CCF0020AA19150898
:10E2300038B50A460D461121044601F063FC28B1A9
:10E24000094A137843F00803137038BD04F5C3403E
:10E2500004214830054A70F081FD29462046BDE87A
:10E26000384008F09FBE00BF0CCF0020BC19150835
:10E2700010B500F5C04494F832349A0623D4D4F88B
:10E280003C0403681B689847032808D005D8022877
:10E290000ED194F83004C00914E01B28F9D194F889
:10E2A000300400F0A000A0F180035842584109E07A
:10E2B000B4F8300420F4FE4020F07F0080B2003833
:10E2C00018BF012010BD0120FCE7000038B500F5A3
:10E2D000C045044695F85534184A43F0080300F544
:10E2E000C34085F855340221483070F037FD6DF099
:10E2F000E9F8012217216CF097FE2046FFF7B8FFDE
:10E3000040B104F5C1400122BDE83840152160301C
:10E31000F8F798BBD5F83C0403681B6898470628B3
:10E3200006D104F51340AC30BDE838400AF0ECB833
:10E3300020460B21BDE83840FFF704BFD01915086F
:10E3400070B500F5C0450646D5F84C24D5F85034D4
:10E350009B1A41F28832934211D9D5F83C040368E4
:10E360001B6D9847044695F85534C3F3C003A34288
:10E3700013D034B13046BDE87040FFF7A7BF00248A
:10E38000F1E76DF09FF8224617216CF04DFE95F8ED
:10E39000553464F3C30385F8553470BD0B4610B58E
:10E3A00011460446072B07D8DFE803F02A041316AA
:10E3B000191C242708F0F6FD04F5A043D3F8EC3E21
:10E3C0009B061DD504F5DA501C30BDE8104097F0CF
:10E3D00081B8FFF7B7FEEFE7FFF7EAFEECE7FFF7DC
:10E3E000C7FEE9E700F5C140012214216030F8F7CB
:10E3F00029FBE1E7FFF7FCFEDEE7FFF719FFDBE7AC
:10E4000010BD000070B504466DF05CF801220521D6
:10E410006CF00AFE04F58043204693F88E32072BF9
:10E4200096BF324A0125D55CFFF722FF68B1304A1A
:10E4300030492046FFF70EFE04F5C14001221021AD
:10E440006030F8F7FFFA002514E004F5C046D6F86E
:10E450003C040368DB6C984798B196F8213A83B185
:10E4600096F9203A012B0CDC234A24492046FFF779
:10E47000F1FD0125294620460322BDE87040FFF743
:10E480008DBFD6F83C040368DB6C984728B104F5CF
:10E49000A043D3F8EC3E190717D4D6F83C04036820
:10E4A0001B689847032805D104F5A043D3F8EC3E38
:10E4B000DA070DD4D6F83C0403685B6A984768B95C
:10E4C0000C492046FFF7A8FDD4E70B4A0949CDE7E0
:10E4D0000B4A08492046FFF7BDFDB4E704F5A04309
:10E4E000D3F8EC3E5B07EBD5064AF2E79C1A150819
:10E4F000F0191508FA501608FA1915080D1A15081A
:10E500001D1A15082D1A150838B5044615466CF065
:10E51000D9FF012206216CF087FD2046FFF7A8FEF7
:10E5200098B104F5C140012207216030F8F78AFA5A
:10E53000144A15492046FFF78DFD0025294620463F
:10E540000422BDE83840FFF729BF04F5C043EDB20F
:10E55000D3F83C040368DB6C984768B104F5A0432A
:10E56000D3F8EC3E1B0707D535B1084A06492046CB
:10E57000FFF770FD0125E1E703492046FFF74CFD59
:10E58000DCE700BFF01915084A1A1508FA19150832
:10E59000F8B504466CF096FF012208216CF044FDAA
:10E5A0007AF006FA04F5804304F5C04693F87D320C
:10E5B000072B9CBF364AD55CD6F8603493F8D570EB
:10E5C00088BF02255FB933492046FFF725FD0025A6
:10E5D000294620460522BDE8F840FFF7DFBE204669
:10E5E000FFF746FE60B104F5C14001221221603000
:10E5F000F8F728FA284A27492046FFF72BFDE6E7D7
:10E60000D6F83C040368DB6C984768B196F8213A69
:10E6100053B196F9203A012B06DC204A20492046C6
:10E62000FFF718FD0125D3E7D6F83C040368DB6C3F
:10E63000984704F5A04718B1D7F8EC3E190713D452
:10E64000D6F83C0403681B689847032803D1D7F821
:10E65000EC3E9A070BD4D7F8EC3EDB0609D40D4903
:10E660002046FFF7D9FCB3E70C4A0A49D7E70D4A21
:10E67000C1E7D6F83C040368DB69984706460028E2
:10E68000EDD1094A03492046FFF7E4FC35469FE7F0
:10E69000A41A1508B2041508F0191508FA19150876
:10E6A000441A1508521A1508671A150870B500F5AE
:10E6B0008043044693F97D32BBB300F5C045D5F8DD
:10E6C000C06396B3D4F01EFA04F5BE4393ED120A6C
:10E6D000DFED167A9FED161ADFED160A861B20EE87
:10E6E000270A8D2034F0CEFBBCEEC00A10EE103AA3
:10E6F0009E420CD295F855349A0716D52046002133
:10E70000F8F7FAFA2046BDE87040FFF7B7BC0CD91D
:10E7100095F855349B0708D420460121F8F7ECFA08
:10E720002046BDE87040FFF733BF70BD00007A445B
:10E730000000804F000000002DE9F341074600F57E
:10E74000FE407030C8F058FC07F5C044C0F3804864
:10E750000190D4F0D7F994F858344345454606461D
:10E760000DD007F5C34084F858844830002D41D0BF
:10E770003B4B3C4AC4F85C64022170F0EFFA94F819
:10E78000583407F5A04843B394F859342BBBB8F973
:10E790005E3F9FED350A9FED351ADFED350A07EE36
:10E7A000903AF8EEE77A40F2571027EE800A34F0FC
:10E7B00069FBBCEEC00AD4F85C0410EE103A361ABD
:10E7C0009E420AD9012307F5C34084F85934294AE7
:10E7D000234B0221483070F0C1FA98F95D3F002BBD
:10E7E00094F855340DDC6FF3451384F8553402B0BA
:10E7F000BDE8F0811A4B204AC4F85C8484F859843F
:10E80000BAE7C3F34012AA42F1D065F3451384F886
:10E8100055349B06EBD5194BD3F83C0403681B69B0
:10E8200098470028E3D06CF04DFE01221F216CF0C8
:10E83000FBFB3846FFF71CFD48B107F5C14001223C
:10E840002121603002B0BDE8F041F8F7FBB898F83C
:10E850005D1F3222384602B0BDE8F041FFF79EBD91
:10E86000801A1508843F160800007A440000804F83
:10E87000000000008F1A15085F3F1608D093002093
:10E8800008B5044B01221A70D4F030F9024B18601D
:10E8900008BD00BF61CC002064CC0020014B0022E9
:10E8A0001A70704761CC00202DE9F0410446D4F085
:10E8B0001DF92A4BB4F8F6221988294E91420546D3
:10E8C0000ED01A80274B18603378A3B1002434701F
:10E8D0006CF0F8FD22461321BDE8F0416CF0A4BBBA
:10E8E0003378214FDBB93B782BB11E4B1F4A1B6895
:10E8F000C31A934201D8BDE8F0810123337004F5B7
:10E90000C043D3F8600490F8D53013B103689B6A14
:10E9100098476CF0D7FD012213216CF085FB3B7802
:10E92000002BE8D03378002BE5D00E4A104913684D
:10E93000EB1A8B42DFD904F5C0441560D4F86004AB
:10E9400090F8D530002BD6D00021C9F0BDFED4F808
:10E9500060040368BDE8F0415B6A184762CC0020A0
:10E9600060CC002064CC002061CC002080841E009C
:10E9700040420F002DE9F84300F5C04500F540582E
:10E980000446D5F83C0498F8087E0368DB6C984789
:10E99000014650B995F93034002BA5BFD5F8603445
:10E9A00093F8D500012180F0010104F5775909F1B0
:10E9B0000C09484697F080FFD5F8603493F8D530BD
:10E9C0000646002B7BD0002865D03E4B93F93034AF
:10E9D000002B04DB02463C49484697F047FB98F978
:10E9E000D27D57B195F93034002B0EDA04F5C140D1
:10E9F00001220F216030F8F725F86CF063FD3246F4
:10EA0000BDE8F84309216CF00FBBD5F83C0403685E
:10EA10005B69984758B195F93134002B07DA95F8BE
:10EA20005534DA0703D498F8083EDB07DED53146C3
:10EA3000484697F0A7FFDFED257AB4EEE70AF1EE3E
:10EA400010FA05DD0A220921204601F05BF8D4E71F
:10EA5000023F032F11D801A353F827F045EA00081D
:10EA60006DEA00088BEA000891EA00080A221521E5
:10EA7000204601F047F80028BFD10A22062120468F
:10EA800001F040F80028B8D1DCE70A221121F6E7AE
:10EA90000A221521F3E797B198F8083E7BB9094B94
:10EAA00093F93034002B06DB04F5C340084A0521F6
:10EAB000483070F053F96CF005FD0022A0E7BDE886
:10EAC000F88300BFD0930020AC1A15080000C8429C
:10EAD000B51A150870B500F5C04300F5FE45703550
:10EAE00086B093F88C1104462846C8F033FA02A881
:10EAF00019F0B2FB04F5105002A9303011F036FDC8
:10EB000004F5E043049AC3F8682F059AC3F86C2F04
:10EB10002846C8F071FA82061AD52846C8F07AFA53
:10EB200004F5FE45FDEEC07A603504F5005417EE9D
:10EB3000901A0222284617EE906A19F093FB94F877
:10EB4000AC36DB0706D401223146284619F08AFB91
:10EB500006B070BD0121284619F048FC0028F2D00B
:10EB6000F6E7000070B500F5004486B0B4F8BC3C90
:10EB70008B420D46164603D1D4F8B83C934221D0BF
:10EB8000D3F0C0FFD4F8B43CC31A132B1AD9C4F87D
:10EB9000B86CA4F8BC5CC4F8B40C6CF093FC0446EC
:10EBA000D3F0B8FF084B094A1B68CDE90453084B62
:10EBB0000193084B0093CDE90201074B074920461A
:10EBC0006CF0BCF806B070BD68CC0020CC1A1508FB
:10EBD000E41A150811ED1408E3CC1408DF1A15081F
:10EBE00038B500F5C0440D4694F83134C3F38013B2
:10EBF0008B420BD021B16CF065FC11216CF0F4F963
:10EC000094F8313465F3861384F8313438BD00004C
:10EC1000F0B52DED048B00F5C0468BB0D6F860340E
:10EC200093F8D530054600F5E044002B67D096F9FF
:10EC30003034002B63DBD6F83C0403685B699847EB
:10EC4000002861D1D4F88C0F9FED440A6C3039F064
:10EC50001DFD0AAACDED080A8DED091A8DED070AF2
:10EC600012E9070004AB01AF83E8070087E807005B
:10EC7000384639F0CFF8D4F88C3F05F5FE404030E7
:10EC8000D3ED368AB0EE409A6FF02CFA3AF01EF9C6
:10EC9000D4F8943FD6F83C04D3EDE49A0368DB6CD7
:10ECA000B0EE408A9847DFED2E7AB4EEE79AF1EEA7
:10ECB00010FA02DC96F838340BB100283AD0DFEDB8
:10ECC000297A68EEA78AF3EE0E7AF4EEE78AF1EE7F
:10ECD00010FA2FDCF0EE087AB4EEE78AF1EE10FAC3
:10ECE00028DCF5EEC09AF1EE10FA23DAD4F88C0F96
:10ECF00003689B6F98470BB0BDEC048BF0BDD4F854
:10ED00008C0F03689B6F0FE005F5A045D4F88C0FBE
:10ED1000D5F8C42F0368B2F90820002A03DCD6F81E
:10ED20003424022AEED1DB6F0BB0BDEC048BBDE8BE
:10ED3000F0401847D4F88C5FDFED0B0A2B68D3F84E
:10ED40008060D4F8943F40F2AB1093EDCC0AB7EE5C
:10ED5000001A34F097F82846B047CCE79F0CB3452B
:10ED60000080BB44E02E65420000000000F5C0407A
:10ED700090F83804704700002DE9F04100F5C045D7
:10ED8000064695F83034B1EBD31F0C4647D0254BDF
:10ED900000221A6000293ED06CF094FB12216CF026
:10EDA00023F995F8303464F3C71385F8303484F0D0
:10EDB0000108A8F03DFE4146A8F016FE06F5804782
:10EDC000B8F1000F05D097F8663013B9D3F09AFE6A
:10EDD000B86687F8668014B3B7F860325B071ED553
:10EDE000D5F8603493F8D530CBB1D5F83C0403683E
:10EDF0005B69984798B9D5F83C04036820219B6962
:10EE0000984760B106F5C1400122BDE8F0410D21EF
:10EE10006030F7F717BE6CF055FB1C21BFE7BDE86B
:10EE2000F08100BF68CC00202DE9F04F2DED0A8B5A
:10EE300000F5C0458DB0D5F8603493F8D56000F585
:10EE40000042044601921EB90121FFF795FF0BE035
:10EE500095F93024002A66DAD5F83C0403689B6CE7
:10EE600098470646002842D04FF0000B95F9302411
:10EE7000B44E002AC0F25981D6ED007AB4F9DC22F2
:10EE8000B8EE677A1AB9B4F8DA22A4F8DC22B4F83A
:10EE9000DC32DFEDAD6A07EE903AF8EEE77A67EE26
:10EEA000A67AB4EEE77AF1EE10FAACBF01210021A8
:10EEB0002046FFF795FE95F93024002A95F8312475
:10EEC000B8BF4BF0010B5306019B93F8A02C48BF31
:10EED0004BF0020B0AB14BF0080B32685946204642
:10EEE0000DB0BDEC0A8BBDE8F04FFFF73BBED5F887
:10EEF0006034204693ED0C8AF7F7DCFFB4EEC80AC5
:10EF0000F1EE10FAB0D5D5F8603493F8A130032BA8
:10EF1000AAD16AF05DFB4FF4801142226AF010FB27
:10EF20003146204691E7019A92F8A09CB9F1000F72
:10EF300003D0844A0023136096E700F5E04A93F873
:10EF40000780DAF88C0F03685B6F984707460090DC
:10EF5000D5F83C0403685B69984720B1D5F8343490
:10EF6000022B00F0E480B8F1000F0CBF4FF0000B53
:10EF70004FF4007BB7EE00BA17B14BF4806B0096EC
:10EF800004F501473C3738469DF0CEF80130DAF8F9
:10EF90008C0F9FED6E0A9FED6ECADFED6E8A0CBF7F
:10EFA000012302236C3008EE103A39F06FFB0CABF2
:10EFB000CDED0A0A8DED0B1A8DED090A13E9070054
:10EFC0000DF10C0E0DF1180C8CE807008EE807000F
:10EFD000704638F01FFF04F5E042DFED5F7AD2F8AB
:10EFE0008C2F92ED36AA2AEE27AAB4EECC0AF3EEC5
:10EFF0000EBAF1EE10FA04F5FE40B4EEEBAAC8BF6B
:10F000004BF4807B4030F1EE10FAC8BF4BF4807BAC
:10F01000F0EE40AA6FF066F839F058FFB8EEC88AF3
:10F0200004F5FE40B4EEC80AF1EE10FA00F17000EB
:10F0300098BF4BF0800BF0EE409AC7F0F7FF68EEF8
:10F04000288AB0EEC09AB4EEE89AF1EE10FA2046A3
:10F0500048BF4BF0400B0DF079FA002847D14BF038
:10F06000200BB24638469DF05FF8012850D14BF096
:10F07000100BB1463349B8F1000F54D0009B002B60
:10F0800051D0F4EECCAAF1EE10FA4CDCB4EEEBAABF
:10F09000F1EE10FA47DCF4EEC89AF1EE10FA42D81D
:10F0A000B4EEE89AF1EE10FA3DD5BAF1000F3AD07D
:10F0B000B9F1000F37D00A68B4F9DC0207EE902AE4
:10F0C000B8EE677A18B9B4F8DA02A4F8DC02B4F83A
:10F0D000DC3207EE903AF8EEE77A67EE8B7AB4EE20
:10F0E000E77AF1EE10FA19D501320A60BEE604F5AE
:10F0F000BF4060306EF09EFFDFED187A90ED007A31
:10F10000B4EEE77AF1EE10FAA9D44FF0000AA9E7BD
:10F1100038469DF009F80130ACD1A8E7012120461E
:10F12000FFF72AFEA2E60022DFE70121C0E6B8F1E0
:10F13000000FB0EE08BA0CBF4FF0000B4FF4007B8D
:10F140001BE700BF68CC0020CDCC4C3E9F0CB345E4
:10F150000080BB440000C842E02E654200004843E6
:10F1600010B500F51E52044607CA88B002AB83E80A
:10F1700007009FED1D7ADDED047A77EE877A9FED2B
:10F180001B7ACDED047AD4EDB97AF0EEE77AF4EE9D
:10F19000C77A04F5FE40F1EE10FA00F140000BD5FD
:10F1A000B4F9DA2207EE902AF8EEE77AF7EE006A71
:10F1B00086EEA77A84EDB97AD4F8E4220192194652
:10F1C00001AA6FF081F82046FFF72EFE2046FEF7D9
:10F1D00039F92046FEF716FA2046FDF7C7FF20460C
:10F1E000FEF77EF808B010BD0AE81C4100000034AC
:10F1F00010B504462DED028B1D207BF04DFB68B34E
:10F2000004F5C043D3F83C0400F0D8FA08EE100A25
:10F2100004F5BC501921183061F0A8F802281AD062
:10F220000338012808D804F5BF4060306EF002FFB3
:10F2300090ED008ABDEEC88AB8EEC88A9FED090A33
:10F2400028EE000ABDEC028B04F501403C30BDE81D
:10F2500010409CF0EFBF9FED048AEDE7BDEC028B00
:10F2600010BD00BF0AD7233C00000000104A026016
:10F27000104A426002F1740102F575524261243A6B
:10F2800082610D4AC2610D4A02620D4A4262A2F2D7
:10F29000A442826204328160C2620A49C1600432BF
:10F2A0000263043204314263074A0161826370479A
:10F2B000C835150824760020005800205CB30020D3
:10F2C0003098002068B30020203700201C2969D81E
:10F2D000DFE801F0130F171B27232F1F682B68335C
:10F2E0006868373B3F43474A4D5054595C606868F3
:10F2F000650000F50C40C430704700F5144038300C
:10F30000704700F50D400430704700F50D40403067
:10F31000704700F511403430704700F51240D83086
:10F32000704700F512404C30704700F512409030A5
:10F33000704700F51340AC30704700F51140743051
:10F34000704700F51140B030704700F50F40303085
:10F35000704700F513401830704700F51040F0304A
:10F36000704700F51540EAE700F51540EFE700F5B6
:10F370001540C0E700F516400830704700F5A04082
:10F38000D0F88C0C704700F51240BCE700F5174030
:10F390007830704700F5A040D0F8E40E704700F5D3
:10F3A0001740DCE70020704773B50B6805461B6CFF
:10F3B00008460C4616469847034605F5C3400F4AD3
:10F3C0000096042148306FF0C9FC6CF07BF823688C
:10F3D00005461B68204698470A21024628466BF0DE
:10F3E00023FE074B93F831349B0641BF054A13783F
:10F3F00043F00403137002B070BD00BFE81A150893
:10F40000D09300200CCF002038B50C4A18230546B5
:10F410000C4669F009FE78B121462846FFF756FFF1
:10F4200030B10146064A2846FFF7BEFF002038BD2E
:10F43000284669F087FCF9E70120F8E7681B150802
:10F44000081B150810B500F5C044002384F874307B
:10F45000084B00F5E04093F83014D0F88C0FC90940
:10F46000BFF00AFBD4F83C040368BDE81040DB6839
:10F47000184700BFD093002070B5054608680368A0
:10F480005B690C461646984790B1306803685B6923
:10F49000984768B905F5C043D3F8602492F8D520A1
:10F4A00032B193F93034002B02DB2846F7F718FD10
:10F4B00004480DF0ABFE20680368BDE870409B680F
:10F4C000184700BF60CD002070B500F5C045044668
:10F4D000D5F83C040B4E0368DB6998473074D5F8C7
:10F4E0003C0403681B689847F070D5F83C04036837
:10F4F0005B6C9847014604F50F502030BDE8704022
:10F5000059F042B8EDCE002070B52DED028B244BA2
:10F5100093F85534DB0782B006460D461446B0EE2C
:10F52000408AF0EE608A06D500232B60236002B08B
:10F53000BDEC028B70BD79F04BFB037F002BF3D049
:10F54000F36A9FED181A1B689FED170AB3F908308C
:10F5500007EE103AB36A1B68B3F9083007EE903A29
:10F56000B8EEC77AF8EEE77A67EE000A68EE811A1D
:10F5700027EE800A28EE011A01A9684634F052FDF0
:10F58000DFED0A6A9DED007ADDED017A27EE267A3D
:10F5900067EEA67A85ED007AC4ED007AC7E700BF72
:10F5A000D09300200AD7233C530469390000C84295
:10F5B00070B52DED028B88B0002302930393364B78
:10F5C00093F8553413F0010F0646B0EE408A06ADAD
:10F5D00002AC03D179F0FCFA037F5BB994E8030035
:10F5E00085E803009DED060ADDED070A08B0BDECD5
:10F5F000028B70BDB36ADFED296A1B68B3F908306E
:10F6000007EE903AF36A1B68B3F9083007EE103A38
:10F61000B8EEC77AF8EEE77A27EE267A67EEA67A92
:10F62000F1EE476ACDED026ADFED1D6ACDED037A9A
:10F63000B0EEC77AB4EEE67AF1EE10FA06D5F0EE47
:10F64000E77AF4EEE67AF1EE10FAC7D403AA21467F
:10F650001448F7F775FCDDED027A9DED037AF0EEC4
:10F66000E77AB0EEC77AF4EE477AF1EE10FACCBF43
:10F67000B0EE670AB0EE470A204638F019FB04A83E
:10F680008DED040ACDED050A38F0C4FB204688EE66
:10F69000000A38F03DFBA1E7D093002053046939FC
:10F6A00000000034D0330020094B93F93024002AA5
:10F6B0000CDAB5EEC00AF1EE10FA07D9D3F86034CF
:10F6C00093F8A100C31E584258417047002070476C
:10F6D000D0930020436A1B6893F8D53043B1054BA3
:10F6E00093F8300400F0A000203818BF01207047C4
:10F6F00001207047D093002010B5436A0446186873
:10F70000D1B10221C8F0F0FF236A9FED0C1A1868EE
:10F710000368F0EE410ADB6AB0EE410A9847236ABB
:10F72000074A1868D2ED970A03689FED040A5B6EDA
:10F73000BDE81040002118470121E3E70000000068
:10F74000D073002010B5436A04461868002930D0F1
:10F750000221C8F0C9FF236A1868BFF05DF9636A27
:10F760001B6893F8A130012B04D8236A0121186883
:10F77000BFF0ECFE63691868C3F006FA63691868A5
:10F78000C3F0B8FA63699FED0C0A1868C3F0EEFC89
:10F7900063691868C3F070FD236A9FED071A186843
:10F7A0000368BDE81040DB6AF0EE410AB0EE410AA2
:10F7B00018470121CDE700BF0000000013B5044643
:10F7C00001A90C480CF050FF10B1019802B010BD17
:10F7D00063691868C1F028FF18B9074BD3F8640FA4
:10F7E000F4E7064801AA032118F072FD0028F4D0BE
:10F7F000EBE700BFD0330020D0A3002030B30020BF
:10F80000F0B52DED048B044689B0002940F0FF804F
:10F810008368814E03F58053B3F9C259642DB8BF94
:10F820006425FFF7CBFF6268A842B2F93430AABF63
:10F8300096F831540125C5F38015002BDBBF6369B1
:10F840001B685B4293EDC78AC8BF07EE903AB2F9D6
:10F850003230C8BFB8EEE78A002BB8BF5B429BB21C
:10F860005B4207EE903AA368F8EEE77A03F580531F
:10F87000F4EEC87AB3F9C279F1EE10FAD8BFB0EE5F
:10F88000678A2046642FB8BF6427FFF797FF636934
:10F89000A26B1B68D2ED001A93EDC91AD3ED0E0AC4
:10F8A000391A00EE101AB8EEC00A33F093FF6368FD
:10F8B000B3F93230002BB8BF5B429BB25B4201EE22
:10F8C000103AF0EE480AB8EEC11A40F2972033F031
:10F8D000D9FA63691868B0EE408AC1F0A5FE96F8BF
:10F8E00032341A0707467FD44C48C4F01DFA00286A
:10F8F0007AD0002F78D09FED4A9A48488DED019A32
:10F9000001A98DED029AC4F097FA00287CD0A06975
:10F91000C7F07EFB03C803AB83E80300194601A8C8
:10F9200038F0AAF905A88DED050ACDED060A38F0E4
:10F9300071FAF0EE409A3B4EDFED3B7AD6ED008A4D
:10F940008DED059A68EEA78AA6F1240005A98DED34
:10F95000069A8DED079AC4F099FAF4EEE89AF1EE62
:10F9600010FAA6F6282608DDDFED307AF0EEE88AF8
:10F97000F4EEE78AF1EE10FA4AD5DDED077A9FED55
:10F980002C7AF4EEC77AF1EE10FA2DDD9FED297A8C
:10F99000F4EEC77AF1EE10FA26D5B6F8403A5B07D6
:10F9A00022D46368B3F93230002BB8BF5B429BB2FC
:10F9B00008EE103ABAEEEF8AF2EE0E7A88EE277A67
:10F9C00067EE297AF5EEC07AF1EE10FA48BFDFED66
:10F9D000147A37EEC88AFAEE047AB4EE678AF1EE4A
:10F9E00010FAC8BFB0EE678A636929461868B0EE9E
:10F9F000480AC1F0BDFE6369186809B0BDEC048B0C
:10FA0000BDE8F040C3F038BCF0EE499A93E700251A
:10FA10009FED038AE8E700BFD0930020D4BD00200B
:10FA200000000000F8BD00200000C84200000034C3
:10FA300000000C4200004843436A186803681B69D1
:10FA40001847000038B52DED028B03680446D3F843
:10FA500084309847236B2A481B68F0EE408AB3F93C
:10FA600008500CF0EBFC4FF47A72041E4FF00001CA
:10FA70002846D8BF4FF4FA7433F042FA8442B6EE07
:10FA8000000A2ADD07EE900AB8EEE77A07EE904A00
:10FA900027EE007AF8EEE77A87EE278A4FF46D704A
:10FAA00038EEC00AF5EE087AB1EE400A80EE270A79
:10FAB000B7EE001AFEEE000A33F0E4F9F7EE007A32
:10FAC00077EEC07A28EE000A20EE080A20EE080A37
:10FAD000A7EE880ABDEC028B38BD031B07EE103A77
:10FAE000C4F57A74B8EEC77A07EE904A27EE007A2A
:10FAF000F8EEE77A87EE278A38EE008ACEE700BF75
:10FB0000D03300202DE9F04F2DED028B00F5004998
:10FB100000F5C04899F8C04C89F8C02C0546D8F8C3
:10FB20003C04036883B01B680E4617469847B042F2
:10FB300023D105F580431A2F83F8647009D140B9A9
:10FB400005F5E04305F5BE45D3F88C3F6A6AC3F876
:10FB5000FC20944B93F831349D0606D401242046B2
:10FB600003B0BDEC028BBDE8F08FBC42F6D08E4AEC
:10FB7000137843F002031370F0E7022F0CD01B2E12
:10FB800012D105F50D403946403003B0BDEC028B73
:10FB9000BDE8F04F01F016BB31462846FFF734FCB4
:10FBA00004460028EBD1DAE731462846FFF78EFB02
:10FBB0000446019018B9284669F0C4F8CFE7D8F890
:10FBC000603493F8D5B003685B699847019A05F5EE
:10FBD000114374338BF0010A9A4208BF0120BBF134
:10FBE000000F08D10198036851465B6898470446A6
:10FBF00048BB6E4A22E098F93034002B80F2C48072
:10FC0000002800F0C180DFF89CB1DBF83C040368F9
:10FC10005B6998470446002840F0B6800198FFF7DA
:10FC200011FFABF5C040B0EE408AF7F743F9B4EEF0
:10FC3000C08AF1EE10FA40F3A7805D4A0199284688
:10FC4000FFF7B2FB8BE705F5C84101AA3C31284616
:10FC5000FFF712FC05F580430198C8F83C0483F8CF
:10FC6000647003681B689847014605F5D2503A4610
:10FC700008306AF0D7FD05F5C3400021483078F020
:10FC80002FF8F31E012B02D9B01F4442444105F561
:10FC9000405389F8BE4B93F9D23D23B105F5775017
:10FCA0000C3096F093FED8F83C0403681B68984724
:10FCB000C11E4842484105F5E04205F5A04389F8D8
:10FCC0001C0003F6F460D2F88C1F0068C1F8F8003D
:10FCD00003F62470D2F88C1F0068C1F8FC00012ED6
:10FCE00001D00B2E06D103F60C73D2F88C2F1B68B3
:10FCF000C2F8FC302846FFF7E7FB2A4B93F8313473
:10FD00009B063FF534AF29E705F5405393F8CC2D1A
:10FD1000002A3FF467AFB3F8E82DD4077FF562AF50
:10FD200093F8083E002B3FF45DAFD8F8603493F8A9
:10FD3000D530002B3FF456AF05F5804393F864307F
:10FD40000A2B7FF44FAF98F93034002BFFF64AAFFF
:10FD5000184A01992846FFF727FB0024FFE61648BA
:10FD60000CF046FE0028CFD1D8F83C0403685B694C
:10FD700098470028C8D0019803685B6998470446F3
:10FD80000028C1D10D4A59E7019803681B699847BB
:10FD90000028E4D008480CF019FE04460028DED103
:10FDA000074A4BE7D09300200CCF0020D4A81708B7
:10FDB000301B1508541B1508D0330020421B1508B2
:10FDC000A20C17080148FFF79DBE00BFD0330020EA
:10FDD00013B504468DED010A9AF0B6F96369A26B7A
:10FDE0001B6892ED001A93ED0E0AD3EDC90A01A922
:10FDF00098F0AEFF9DED010A02B010BD436A18688D
:10FE000003685B6A1847000038B5436A1C6894F8B9
:10FE1000D510054661B92046C8F066FC6B6A1B68C0
:10FE200093F8A10018B1012814BF0320022038BDA7
:10FE3000164803783BBBFFF737FC20BB144A92F807
:10FE4000303403F0A003202B17D0B5EEC00AF1EE3A
:10FE500010FA10D592F832345B070CD401212046F9
:10FE6000C8F042FC6B6A1B6893F8A130012B0CBFF1
:10FE700002200320DBE70221F1E720460221C8F03F
:10FE800033FC0420D3E70120D1E700BF60CD002080
:10FE9000D093002010B52DED028B124B93F8553402
:10FEA000DB07044604D59FED100ABDEC028B10BDA4
:10FEB00078F08EFE037F002BF5D0636B186879F025
:10FEC00049F8A368DFED097A03F5E35292ED008A61
:10FED000D2ED010A28EE278A34F05EF828EE000AF7
:10FEE000E3E700BFD0930020000000000000C842FC
:10FEF0000148F7F751B800BFD03300200148F7F7A9
:10FF0000C9BF00BFD03300200148FFF7FBBD00BFD1
:10FF1000D03300202DE9F04F5E4E2DED028B96F888
:10FF200055348FB013F0010F04460D4605AF5FD175
:10FF300043689B899A071CD557486EF07BF8DFED24
:10FF4000577A90ED007AB4EEE77AF1EE10FA10DD10
:10FF50006BF0B8FA3D216BF047F809220521A6F5B0
:10FF6000C040FFF7CFFD20B9092202212046FFF74C
:10FF7000CBFF636893F95430002B39D000230593ED
:10FF8000089323691868C6F099FD236A1868036806
:10FF90009B6EB0EE408A984708AAF0EE400A3946B8
:10FFA000B0EE480A2046FFF7AFFADDED057A9FED87
:10FFB0003C7AF0EEE77AF4EEC77AF1EE10FA08D563
:10FFC000DDED087AF0EEE77AF4EEC77AF1EE10FA9A
:10FFD0000ED496F832341B0704D46BF073FA49211F
:10FFE0006BF002F896F8323443F0080386F83234A6
:10FFF0002868F4F7C7FA824668688B46F4F7C2FAB5
:020000040801F1
:100000008046A86880F000408946F4F7BBFA9FED6F
:100010001F0BCDE90C0108A8CDE908ABCDE90A8991
:1000200039F052FA8DED0A1B8DED0C2B8DED080B7E
:100030006369DFED1C0A9FED1C0A186808A9C2F06D
:1000400001FC63691868C2F055FE63691868C3F063
:1000500013F9236A1D6863691868C1F029FE3846E0
:1000600012498DED020ACDED030A8DED041AFCF75D
:1000700049F8079B009397E80C0002A92846BEF0B8
:100080007DFD0FB0BDEC028BBDE8F08F00000000DD
:1000900000005940D093002024B3002000002F44DA
:1000A0000000003400007A44000000001CCC002056
:1000B0002DE9F043AA4D2DED028B95F8313493B024
:1000C00000265A0604460596069603D54369186825
:1000D000C1F002F995F85534DB0756D463689B8963
:1000E0009F071BD59F486DF0A5FFDFED9F7A90ED30
:1000F000007AB4EEE77AF1EE10FA0FDD6BF0E2F978
:100100003D216AF071FF994809220521FFF7FAFCA9
:1001100020B9092202212046FFF7F6FE636893F911
:10012000543093B391489FED928AF7F7B3FEE3689A
:100130009FED907A1B68D3ED0A7AF4EEC87AF1EE5F
:1001400010FAB8BFF0EE477AB6EE000A27EE800A42
:100150002046FFF72DFA8DED050AB0EEC00AB4EE89
:10016000C80AF1EE10FACDED060A40F1AC80F0EECF
:10017000E00AF4EEC80AF1EE10FA40F1A4807E4BDA
:10018000B3F8403A980700F1AE8095F833346FF336
:10019000820385F8333495F832341A0700F1A880C9
:1001A0007648C3F0C1FD95F8333460F3820313F051
:1001B000040F85F833340EAF40F09C8060690E96D2
:1001C0000F96006801233A4605A9C1F0FFF863695C
:1001D0001868C2F08FFD63691868C1F069FDA368F3
:1001E0008DED0B0ACDED0C0A8DED0D1AD3ED007AD5
:1001F000F5EEC07AF1EE10FA52DD614B9FED618AA7
:10020000B3F9503200EE903AF8EEE00A2046CDED18
:10021000030AFFF7D3FAA368DDED030AD3ED001A52
:100220009FED510AB7EE002A07EE900A31EE822ABE
:10023000B8EEE71A22EE082A61EE881A32F042FD83
:10024000DFED517A20EE270ADFED507A20EE270A03
:1002500033F130FDDFED4E7A20EE270A0BA820EEB9
:10026000088A37F0D7FDB4EEC08AF1EE10FA17D540
:10027000C8EE006A63699DED0B7ADDED0C7A27EE1E
:10028000267A67EEA67A8DED0B7ACDED0C7A1B6897
:10029000D3F8AC23C3F8B823D3F8B023C3F8BC23F6
:1002A000236A3C491C683846FBF72CFF109B0093DF
:1002B00097E80C000BA92046BEF060FC13B0BDEC23
:1002C000028BBDE8F08395F83234190704D46BF043
:1002D000F9F849216AF088FE95F8323443F00803B2
:1002E00085F8323451E795F832346FF3C303F7E7FA
:1002F000002058E70DF11C08204807964146089653
:1003000009960A96C3F098FD28B9A069C6F080FE48
:1003100003C888E80300A069C6F082FE09AA014666
:100320001648C3F0EFFD08980B960C96F4F72AF9DF
:10033000804607988946F4F725F9CDE91089CDE97B
:100340000E0101236069009300680BAB09AA3946CE
:10035000C1F074F895F833345B077FF52FAF36E7BB
:10036000D093002024B3002000002F44D03300207D
:100370000000003400007A43D0B30020D4BD002038
:10038000D07300200000C8420AD7233C35FA8E3CC7
:100390000AE81C411CCC002013B504460191FFF76C
:1003A00087FE0199204602B0BDE81040FFF728BA49
:1003B0001FB5194B93F832341B07044629D4002388
:1003C00001A91648019302930393C3F051FB03283C
:1003D00007D8DFE800F0150E020801A92046FFF754
:1003E00099FD04B010BD0D48C3F064FB30B1012885
:1003F000F7D100212046FFF7CFFFF2E70121F9E70F
:1004000069F0E6F840F286324FF4801169F098F80E
:10041000EFE70021EFE700BFD0930020C8BE002027
:1004200008B5034619B9064A92F9042A1AB91846BA
:10043000FFF7B2FF08BDBDE80840FFF7B9BF00BF36
:10044000D0B300200148FEF797BC00BFD033002096
:1004500000487047989500200148F6F789BD00BF15
:10046000D033002070B5174D8AB000230022044617
:1004700004A9D5F8940FCDE90423CDE90623CDE9ED
:100480000823C1F02DFCD5F8940F08A9C1F092FC07
:10049000DDE90601F4F7C6FB0646DDE90801F4F7DD
:1004A000C1FB0546DDE90401F4F7BCFB0222019023
:1004B00001A920460296039518F0A6FA20460AB034
:1004C00070BD00BFD0A30020014B01221A707047FD
:1004D0006CCC00200020704700207047002070473F
:1004E00000207047002070470020704700207047B0
:1004F0000020704700207047002070479FED010AE0
:10050000704700BF000000000020704700207047C7
:10051000002070470120704700207047002070477E
:10052000002070470120704700207047012070476D
:10053000012070470020704701207047012070475C
:100540000020704700487047801B1508004870471E
:10055000801B1508836803F5805393F8743CDB0710
:1005600006D5002380F83C30024B0222C3F8342425
:1005700001207047D093002090F83C3053B9836835
:1005800003F5805393F8743CDB0742BF034B012211
:10059000C3F83424002380F83C307047D093002007
:1005A000012380F83C3070472DE9F0432DED0C8B92
:1005B000F0EE409A20EE000A97B00025A0EEA00AC7
:1005C00004468946B0EE41CAF0EE60AA90461F4646
:1005D00001950295039504950595069533F1B6FDB1
:1005E000F7EE00CAB4EEEC0AF1EE10FAC8BFCCEE9A
:1005F000807AA36803F5805303F5436203F634431E
:10060000D3ED000A92ED009A9FEDC6DAC4BF69EE01
:10061000A79A6AEEA7AAB0EE690A33F0BDFCA368F8
:1006200029EE0D9A03F5805303F5436203F6344334
:10063000D3ED000AD2ED008A29EE009AB0EE6A0AE4
:1006400033F0AAFCA36868EE8D8A03F5805303F6A5
:10065000484203F64C43D3ED000A92ED008A68EE5F
:10066000808AB0EE4C0A33F097FC636828EE0D8A5E
:1006700093F9703028EE008A002B00F0D980236AAD
:100680009FEDA90A18686C3038F000F8B0EE60AA47
:10069000CDED080A8DED091A8DED070A32F090FBB9
:1006A000BDEEC0BAA14940F6B8321BEE100A32F0D6
:1006B00017FC434207EE903A6368F8EEE77A93ED51
:1006C0001A7A67EE877AB0EE4A0ACDED017A32F0F7
:1006D00077FBFDEEC0BA40F6B83294491BEE900AA3
:1006E00032F0FEFB42426368039507EE902A93EDD9
:1006F0001B7A93F97030F8EEE77A022B67EE877A6F
:10070000CDED027A6ED18A4BB3F950320AEE103A2F
:10071000B8EECBBAB8EECAAA236AB4EECABAF1EE02
:1007200010FA1A683DDDA368DFED820AA16B92ED35
:10073000051AD1ED001A03F5E15393ED047A27EE83
:100740000D7A3AEE4B0AC7EE200A33F043F8DDED9E
:10075000017A37EE800A8DED010AB8EEEB0A236AC2
:10076000B4EECA0AF1EE10FA1A6834DDA368A16B80
:1007700092ED061AD1ED001A03F5E153D3ED040A08
:1007800020EE8DDADFED6B0A3AEE400ACDEE200A5C
:1007900033F020F8DDED027A37EE800A8DED020AA3
:1007A00020E0B1EE4A0AB4EEC0BAF1EE10FAD4D5A8
:1007B000A368A16BDFED5F0AD1ED001A92ED051A77
:1007C00003F5E15393ED047A27EE0D7A30EE4B0AF0
:1007D000C7EE200AB9E7B1EE4AAAB4EECA0AF1EEB2
:1007E00010FAC3D4236AD3F800C00CF184030FCBF2
:1007F00012AD85E80F000EAE0AAD86E80F0085E861
:100800000F0004AB01AA29466046BEF053FE6368A0
:1008100093F97030022B16D1DDED047A39EE279A68
:10082000DDED057A78EEA78ADDED067A38EE278AC7
:1008300089ED009AC8ED008A87ED008A17B0BDECFB
:100840000C8BBDE8F083F0EEE99AF0EEEAAAF4EE44
:10085000E9AAF1EE10FA48BF6D46CDED009ACDED54
:100860000AAAD5ED007ADFED340AB0EECCCAF4EE78
:10087000CC7AF1EE10FAD8BF35468DED0ECA95ED63
:10088000007ADFED2E7A87EE270AAD20B7EE001A48
:100890003CEEC00A32F0F6FAE369D3ED937A04A88D
:1008A00020EE270A37F0F2FEF0EEC07A8DED061A40
:1008B000B0EEC91A31EE671A8DED040AB0EEC11A16
:1008C00039EE000ACDED050AB520F1EE410A32F00D
:1008D000D9FAB0EE409A9DED050AB0EEE81AF0EEB6
:1008E000C07A31EE671A38EE800AB0EEC11AF1EE26
:1008F000410ABA2032F0C6FAF0EE408A9DED060AAF
:10090000B0EEC81AF0EEC07A31EE671A38EE000A7F
:10091000B0EEC11ABF20F1EE410A32F0B3FAB0EEE8
:10092000408A85E70000C8429F0CB34548F4FFFFAA
:10093000D073002000007A440000000000A08C4525
:1009400010B52DED028B836A044686B0186878F0E6
:1009500001FBE36A1868B0EE408A78F0FBFA636B3B
:100960008DED010A186878F0F5FA05ABB0EE401A83
:1009700003A92046DDED010A04AAB0EE480AFFF7FC
:1009800013FE636A186890F8D51000293CD1C7F0AF
:10099000ABFE2046FFF756F8636A1B6893F8A11078
:1009A0000129B0EE408A3FD0032946D051B9236ACD
:1009B00001211868BFF09AFC236A1868BEF016F887
:1009C0009FED218A236A9DED030A1868A3680268D7
:1009D000DDED040A9DED051A03F5805393F8743C90
:1009E0009B074CBFD36B936B9847236A174A1868D1
:1009F000D2ED970A036800215B6EB0EE480A984773
:100A000006B0BDEC028B10BD114B93F93124002AC6
:100A100006DBD3F83434022B04D190F8A1300BB9A3
:100A20000121B4E70221B2E7236A1868BFF05EFC37
:100A3000236A1868BDF0F0FFC2E7D9790029C1D157
:100A40002046FFF7FFFCBDE700000000D073002048
:100A5000D0930020836803F6A82393ED000AB5EE37
:100A6000C00AF1EE10FA01DCFEF7E6BF70470000A5
:100A70007047000000207047012070470220704737
:100A80000020704700207047012070470020704709
:100A900081F001007047000001207047012070477D
:100AA000004870471C1C150800487047281C150892
:100AB00038B5436904461868C0F0E4FE18B96369A4
:100AC0001868C2F067FA636920461D68FFF7C4FC26
:100AD0006368B3F93820B3F9363000EE903A4342F8
:100AE00001EE102A00EE103AB8EEC11AF8EEE00A54
:100AF000B8EEC00A2846C0F0A5FD636920461D680F
:100B0000FFF7AAFC6368B3F93820B3F9363000EE7A
:100B1000903A434201EE102A00EE103A2846B8EE11
:100B2000C11AF8EEE00AB8EEC00AC0F005FE0120D6
:100B300038BD000030B52DED028B0446436985B009
:100B40001D68FFF789FC6368B3F93820B3F93630C4
:100B500000EE903A434201EE102A00EE103AB8EE51
:100B6000C11AF8EEE00AB8EEC00A28465B4DC0F0A4
:100B700069FD2046FFF7C2F9B5F9503208EE103A88
:100B8000236A186803689B6E9847B8EEC88AF0EE2F
:100B9000400A02AA01A9B0EE480A2046FEF7B4FCBA
:100BA0002046FFF777F9236B1B68B3F90830F0EEA6
:100BB000408A00EE103A2046B8EEC00AFFF798F9D6
:100BC0002046B0EE408A8DED030AFFF745FC6368CE
:100BD000B3F9363001EE103A434200EE903AB8EEE7
:100BE000C11AF8EEE00A2B20B0EE480A32F04AF9BA
:100BF00020468DED030AFFF707F9042813D8DFE834
:100C000000F0032F252A4B00236A1868BDF0EEFE82
:100C1000236A00211868BEF099FC63699FED300AD1
:100C20001868C2F0A3FA236ADDED020A18689DED88
:100C3000010A0368B0EE681ADB6A984763691868AE
:100C4000C2F01AFB05B0BDEC028B30BD236A012156
:100C50001868BEF07BFC236A1868BDF0DDFEDCE797
:100C6000204D2B7863B963689FED1F1ADFED1C0AD6
:100C700093ED040A452032F005F928460CF0A2FA5B
:100C800020469DED030AFFF7A3F816488DED030AF1
:100C900003A90CF0DDFAC6E7636A02211868C7F001
:100CA00023FDB5F95032114800EE103A02AA01A90D
:100CB000B8EEC00A99F0C2F920469DED030AFFF78D
:100CC00087F80B488DED030A0BF0ECFC63699DED92
:100CD000030A1868C0F03CFDA5E700BFD0730020F0
:100CE0000000000060CD002000007A4480B40020A5
:100CF000389400200020704790F8B931002B14BFC1
:100D00001B2003207047000000207047012070471F
:100D100090F89001062804D0A0F10A0358425841E7
:100D20007047012070470000012070470120704784
:100D300090F8B901034A044B002814BF1046184626
:100D4000704700BFC41C1508A522170890F8B90108
:100D5000034A044B002814BF10461846704700BFD2
:100D6000D01C1508A522170890F890010B3818BF61
:100D70000120704790F8B9312BB9044BD3F8400FDC
:100D800000F0010070470020704700BFD0830020B2
:100D9000024BD3F8400FC0F3C0107047D08300203F
:100DA00090F8903123B9034B187880F00100704718
:100DB0000020704738CD002038B590F89041012CC4
:100DC000054601D0002038BDC368186803681B6958
:100DD00098470028F6D1EB681B68204683F8B8488E
:100DE000F1E70000C3681B68002283F8B8280120DF
:100DF0007047000070B52DED028B002380F8B931EB
:100E0000B0F87030012B84B004460D4601D800299B
:100E100049D0636A264E1B6893F8D5308BBB2548B2
:100E2000072384F890310368022B02D10021FAF7DE
:100E30000BFF9FED218AE368F0EE480A1868B0EED8
:100E4000481AF0EE481AB0EE480A0125C5F088F8B5
:100E500084ED798A84ED7A8A84ED7B8A84F8B851AE
:100E600004F59A7038F09AFB144805F00FFB96F8D9
:100E7000323413486FF3C30386F83234C2F000FDF6
:100E800011E096F93034002BC9DA04F13C003AF055
:100E900077FE05460028C2D12046FFF7D9FA094A55
:100EA00002216DF05BFF284604B0BDEC028B70BDE3
:100EB000D09300201CCC0020000000001CC60020A5
:100EC000C8BE0020D81C150838B5094D95F8803DDE
:100ED000012B044603D105F67C5038F0C5FB95F88C
:100EE000A51004487BF096F8002384F8B93138BD8A
:100EF000D0B30020FCB3002010B52DED028B094BC0
:100F00000446D3F8980FB0EE408AC4F063FB9FED1F
:100F1000060A28EE008A012084ED7A8ABDEC028B55
:100F200010BD00BFD0A300200AD7233C10B52DED83
:100F3000028B094B0446D3F8980FB0EE408AC4F0F8
:100F400059FB9FED060A28EE008A012084ED7B8A7A
:100F5000BDEC028B10BD00BFD0A300200AD7233CFC
:100F600010B52DED028B094B0446D3F8980FB0EE67
:100F7000408AC4F04DFB9FED060A28EE008A01204E
:100F800084ED798ABDEC028B10BD00BFD0A3002098
:100F90000AD7233CC3681B681869C0F0EBBF000088
:100FA00038B5D0F8943104460D461BB9D1F0AAFDEE
:100FB000C4F89401D1F0A6FDD4F89431C01A4FF4CE
:100FC0007A73B0FBF3F0B4F89231984209D320461B
:100FD000FFF73EFA2B88044A06216DF0BFFE012080
:100FE00038BD0020FCE700BFF41C150890F89031D4
:100FF000052B05D1054BD3F8A03FD868C0F028BF1A
:10100000C36818680368DB68184700BFD0A30020D6
:1010100008B590F89031052B0BD1094BD3F8A03FC0
:10102000D868243036F0F6FEBCEEC00A10EE100A86
:1010300008BDC368186803689B689847F4E700BF59
:10104000D0A3002090F890318B4206D00B2B80F873
:10105000901102D10148FCF739BD7047D033002010
:1010600073B501231E4E80F87530D6F83C348342A8
:1010700005460A4614D1012485F8B941D6F83C0446
:10108000019203681B689847019A0146154869F068
:10109000C9FB96F831349A061BD4204602B070BDC5
:1010A00001910321FEF730FF019A04460028E2D1A6
:1010B00085F875006AF006FA1B220A2169F0B4FF70
:1010C00096F831349B06E8D5074A137843F00403B9
:1010D00003E0054A137843F002031370DDE700BF15
:1010E000D0930020184E00200CCF002030B585B0E2
:1010F00004460D4601466846FFF7B4F9694604F117
:101100003C003BF0ADF9C8B96AF0DCF91B220A21BA
:1011100069F08AFF0D4B93F831349B0604D50C4AD5
:10112000137843F0040313702046FFF791F9094A3E
:1011300004216DF013FE002005B030BD2946204685
:1011400005B0BDE83040FFF78BBF00BFD093002053
:101150000CCF0020081D150830B585B004460D469B
:1011600001466846FFF77EF9694604F13C003BF012
:101170009BF9C8B96AF0A6F91B220A2169F054FF4D
:101180000D4B93F831349B0604D50C4A137843F089
:10119000040313702046FFF75BF9094A04216DF040
:1011A000DDFD002005B030BD2946204605B0BDE874
:1011B0003040FFF755BF00BFD09300200CCF002078
:1011C000441D15087FB505460E4605F13C04014651
:1011D0006846FFF747F9694620463BF065F9C0B914
:1011E000204669463BF03CF9044690B96AF06AF93A
:1011F0001B220A2169F018FF0D4B93F831349B062E
:101200000FD42846FFF724F90A4A04216DF0A6FD01
:1012100004E031462846FFF723FF0446204604B089
:1012200070BD054A137843F004031370E9E700BF6B
:10123000D09300207C1D15080CCF002010B590F82D
:1012400090410A2C16D1B0F8BE410C8090F8C41120
:101250001170D0F8C8211A60029BD0F8CC211A6016
:10126000039BB0F9D0211A80049BB0F9D2211A80D7
:10127000012010BD0020FCE790F890310A2B06D128
:10128000B0F8BE318B4204BF012380F8BC317047F7
:1012900030B5044685B00F480BF098FB0546B0B159
:1012A000072384F890310023019302930393E368AA
:1012B00001A91868C4F018F9E3681868036801A95F
:1012C0005B680022984704480021FAF7BDFC2846D5
:1012D00005B030BDD03300201CCC0020F0B5424F0B
:1012E000D7F86C2FD7F8683F2DED028B1343D7F852
:1012F000642F134387B005460C460CD168F068F99B
:1013000040F275124FF4801107B0BDEC028BBDE8BE
:10131000F04068F015B98069C5F07CFE2046B0EE5B
:10132000408A16F0C9FF03283AD1EB6801A9186872
:10133000C4F0E4F9064698B3DDED017A63680093E2
:1013400038EE678A294BDFED2A7A93F930349FED26
:10135000290A2948002BA8BFB0EE670A38EE008A98
:10136000009BBDEEC88A002118EE102A9342ACBF44
:1013700000930092FAF768FC6B691868C1F00AFEE6
:10138000DDED007A1D48B8EEE70A31460CF0F2F9BF
:1013900000212846FFF756FE07B0BDEC028BF0BDDA
:1013A00094E80F0002AE86E80F00D7F8683F049378
:1013B0006A46D7F86C3F05930221304616F088FF45
:1013C00078B96AF07FF80222152169F02DFEDDED73
:1013D000037AF8EEE77A77EE887AFDEEE77ACDEDDC
:1013E000007A0026AEE700BFD0A30020D0930020F3
:1013F000000000000000C8421CCC002038CD0020B6
:10140000F0B52DED028BC3688BB0044618680D460D
:10141000C4F04AF900285BD100230193029303939F
:1014200094F89031EBB900220023384804A9CDE9A3
:101430000423CDE90623CDE908230CF0CDF980B1D2
:10144000DDE90601F3F7EEFB0746DDE90801F3F7F6
:10145000E9FB0646DDE90401F3F7E4FB029701909E
:10146000039694ED790A9FED2A8AE368DDED010A7F
:101470009DED021ADDED031A1868B4EEC80AF1EE0C
:1014800010FAAABFDFED237A9FED230A20EE270A88
:10149000C4F066FDD4ED7A7AF4EEC87AF1EE10FA73
:1014A00007DBE3689FED1B0A186827EE800AC4F08B
:1014B00091F8D4ED7B7AF4EEC87AF1EE10FA07DBFE
:1014C000E3689FED140A186827EE800AC4F092F8CA
:1014D000E36829461868C4F06BFC054688B10F4BD9
:1014E0001B68022B09D0032B03D10D4B93F98132DA
:1014F0001BB10A480021FAF7C7FB01212046FFF77C
:10150000A1FD28460BB0BDEC028BF0BD38CD00200C
:10151000000000340000C842000000001CCC002085
:10152000D073002010B52DED028BC368DFED348A37
:101530001B684269D3ED0A0A9FED328A93ED060AD1
:10154000F4EEE80A0446F1EE10FA1068B8BFF0EEC7
:10155000480ABFF041FEE36862691B681068D3ED7A
:101560000A0A93ED060AF4EEE80AF1EE10FAB8BFA3
:10157000F0EE480ABFF0A8FE63691868C0F054F89E
:1015800018B963691868C1F05FFAE36862691B689B
:10159000106893ED080A93ED0C1AD3ED070AB0EE2C
:1015A000C00AC0F04FF8E36862691B68106893EDE9
:1015B000080A93ED0C1AD3ED070AB0EEC00AC0F08A
:1015C000BBF863691868C0F05DF918B963691868F9
:1015D000C1F0E0FC00210C48FAF736FB0B489AF00A
:1015E000C1FE0B4AB2F8323423F48163A2F83234DC
:1015F000BDEC028B20460221BDE81040FFF722BD62
:101600000000003400007A431CCC00200CB5002000
:10161000D093002010B50C4B0446D3F8A00F90EDEA
:101620000F0A90F8602000F12001C3F01FFC07486A
:101630000368022B02D00821FAF706FB2046052199
:10164000BDE81040FFF7FEBCD0A300201CCC00205A
:101650002DE9F0432DED028B524DDFED538AB0EEB4
:10166000408A93B00446D5F8A00F0E461746C3F043
:101670000FFAF0EEC87AF4EEE87AF1EE10FA07D439
:101680009FED4A0AD5F8A00F28EE000AC3F062FACF
:10169000D5F8A00F90ED0F0AB0EEC00A0FB1B1EE71
:1016A000400AC3F047FA0023D5F8A00F039302AA1B
:1016B00003A904930593C3F069FADFED3D7A9DED2C
:1016C000027AB4EEE77AF1EE10FA66DD022203A99F
:1016D0000EA817F099F971680191304616F0ECFDEB
:1016E000019902460EA816F0BDFDE3680EA9186820
:1016F000C4F05EFB10B92F48FCF7E8FDA069C5F007
:1017000087FC06464068F2F73DFF80463068894610
:10171000F2F738FFCDE90601D5F8A00F06A9203071
:10172000CDE9088936F08EFE0AA88DED0A0B8DED05
:101730000C1B36F0F5FE204B1B68022B51EC100BF6
:101740001FD0D5F8A03F93ED0E8AB4EEE88AF1EEF3
:1017500010FAB8BF93ED048AF3F764FA07EE900A23
:10176000B4EEE78AF1EE10FA13484FF0000111D5FC
:101770009FED127AF4EEC77AF1EE10FA0ADDFAF76D
:1017800083FA04212046FFF75DFC13B0BDEC028B09
:10179000BDE8F083FAF758FAF3E72046FFF73AFF7F
:1017A000F3E700BFD0A30020000000340000C842CF
:1017B00000009643D03300201CCC00200000FA43E8
:1017C00070B52DED028B294BDFED298AD3F8984FA8
:1017D000D3F8945FD4ED0A0A9FED268A94ED060AA9
:1017E000F4EEE80AF1EE10FAB8BFF0EE480A064649
:1017F0002846BFF0F1FCD4ED0A0A94ED060AF4EE97
:10180000E80AF1EE10FAB8BFF0EE480A2846BFF039
:101810005BFD2846BFF008FF10B92846C1F014F957
:1018200094ED080A94ED0C1AD4ED070AB0EEC00A44
:101830002846BFF007FF94ED080A94ED0C1AD4ED8A
:10184000070A2846B0EEC00ABFF076FF2846C0F06F
:1018500019F810B92846C1F09DFB07480021FAF796
:10186000F3F9BDEC028B0123337070BDD0A30020CF
:101870000000003400007A431CCC002008B5074863
:10188000D0F8403F9B0704D50121A0F5A040F5F713
:10189000CFF9BDE8084002480BF0C2BDD08300205C
:1018A00038CD002030B589B00446FDF713FF30B1C4
:1018B0000021204609B0BDE83040FDF743BF636A10
:1018C00002211868C6F010FFE368186803685B69B6
:1018D000984701461048FCF7E3FB63691868C1F0BC
:1018E000CBFC236A1D6863691868C0F0E1F905AC98
:1018F00020460A498DED020ACDED030A8DED041A4A
:10190000FAF700FC079B009394E80C0002A9284614
:10191000BDF034F909B030BDD03300201CCC00201C
:1019200038B50446FDF7D6FE054628B1204600210D
:10193000BDE83840FDF706BF636A02211868C6F0AB
:10194000D3FE29462046BDE83840FEF769BD0000B9
:101950000148002107F0F8B97CC7002030B5174DC9
:101960009FED170A05F5E04389B00446D3F8A00FB0
:10197000C3F030FB01462846FCF792FB6369186808
:10198000C1F07AFC236A1D6863691868C0F090F999
:1019900005AC20460B498DED020ACDED030A8DED15
:1019A000041AFAF7AFFB079B009394E80C0002A916
:1019B0002846BDF0E3F809B030BD00BFD0330020A9
:1019C000000000001CCC002030B589B00446FDF7B3
:1019D00081FE30B10021204609B0BDE83040FDF75E
:1019E000B1BE636A02211868C6F07EFEE36818681B
:1019F00003685B69984701461048FCF751FB63692F
:101A00001868C1F039FC236A1D6863691868C0F062
:101A10004FF905AC20460A498DED020ACDED030AC7
:101A20008DED041AFAF76EFB079B009394E80C0007
:101A300002A92846BDF0A2F809B030BDD03300207D
:101A40001CCC002030B52DED028B83B00446FDF791
:101A500041FE20B9636A1B6893F8D63043B9002170
:101A6000204603B0BDEC028BBDE83040FDF76ABEF6
:101A700094F89831DA071DD4E3681D682B6828466E
:101A80009B689847D5ED097A94F89831B4EEE70A47
:101A9000F1EE10FA4CBF0122002262F3000384F839
:101AA000983107D4204603B0BDEC028BBDE830402E
:101AB000FFF7F8BE94F898319B0734D4E368DFED64
:101AC000458A1B686269D3ED0A0A9FED438A93ED4C
:101AD000060A1068F4EEE80AF1EE10FAB8BFF0EE6C
:101AE000480ABFF079FBE36862691B681068D3EDB0
:101AF0000A0A93ED060AF4EEE80AF1EE10FAB8BF0E
:101B0000F0EE480ABFF0E0FB63691868BFF08CFD97
:101B100018B963691868C0F097FF94F8983143F0DA
:101B2000020384F898312D4BD4F8A021D3F8643FF8
:101B30009B1A07EE903AB8EEE78AF1EE047AB0EE1F
:101B4000C87AB4EEE77AF1EE10FA38D594F8983105
:101B500043F0040384F89831204684ED678AFEF749
:101B6000A7FA6369A26B1B68D2ED001A93EDC91A3C
:101B7000D3ED0E0AB1EE480A31F02CFE63691B6802
:101B800040F2AA4093EDC61AD3EDC70A31F07AF9B4
:101B90002046FEF71DF912488DED010A0AF082FD7C
:101BA00063699DED010A1868BFF0D2FD636918688A
:101BB00003B0BDEC028BBDE83040C1F05DBBD4ED9D
:101BC000677A68EE277AF5EEC07AF1EE10FAC3D59F
:101BD000BCE700BF0000003400007A43D0A300201F
:101BE0003894002030B52DED028B83B00446FDF70C
:101BF00071FD20B9636A1B6893F8D63043B90021A0
